:100000000C94C51F0C94F01F0C94F01F0C94F01F5F
:100010000C94F01F0C94F01F0C94F01F0C94F01F24
:100020000C94F01F0C94A6D10C94F01F0C94F01FAC
:100030000C94F01F0C94A6900C94F01F0C94F01FDD
:100040000C94F01F0C944B990C94BCCE0C94F01FA4
:100050000C94F03B0C94F01F0C94F01F0C94F01FC8
:100060000C94F01F0C94F01F0C9421C70C94F01FFB
:100070000C94F01F0C94F01F0C94F01F0C94F01FC4
:100080000C94E78E0C94F01F0C94F01F084AD73B99
:100090003BCE016E84BCBFFDC12F3D6C74319ABD57
:1000A00056833DDA3D00C77F11BED9E4BB4C3E917B
:1000B0006BAAAABE000000803F05A84CCDB2D44E6A
:1000C000B93836A9020C50B9918688083CA6AAAA6C
:1000D0002ABE000000803F4D383420582059205A55
:1000E0002045006563686F3A0043616E6E6F74204F
:1000F000656E746572207375626469723A20004D92
:100100003234004D3233202573006175746F2569D8
:100110002E67004572726F723A006572726F7220BC
:1001200077726974696E6720746F2066696C650008
:100130004E6F74205344207072696E74696E67004C
:100140002F005344207072696E74696E6720627963
:10015000746520002E0044656C6574696F6E2066BE
:1001600061696C65642C2046696C653A20004669BB
:100170006C652064656C657465643A002E006F7070
:10018000656E206661696C65642C2046696C653A11
:10019000200057726974696E6720746F2066696CFD
:1001A000653A20002E006F70656E206661696C658F
:1001B000642C2046696C653A20002E006F70656ED5
:1001C000206661696C65642C2046696C653A200084
:1001D00046696C652073656C6563746564002053C3
:1001E000697A653A200046696C65206F70656E65B6
:1001F000643A20002E006F70656E206661696C6540
:10020000642C2046696C653A20004E6F7720667238
:100210006573682066696C653A20004E6F772064CC
:100220006F696E672066696C653A20002220706FE6
:1002300073002220706172656E743A220053554239
:10024000524F5554494E452043414C4C20746172E5
:100250006765743A2200747279696E6720746F2042
:1002600063616C6C207375622D67636F64652066D3
:10027000696C6573207769746820746F6F206D6195
:100280006E79206C6576656C732E204D4158206C1C
:100290006576656C2069733A002E0A0044656C65CA
:1002A00074696F6E2862696E29206661696C656485
:1002B0000046696C652862696E292064656C657406
:1002C00065640057726974696E6720746F2066698F
:1002D0006C653A20002E0A006F70656E20666169B9
:1002E0006C65642C2046696C653A20005344206399
:1002F000617264206F6B006F70656E526F6F742057
:100300006661696C656400766F6C756D652E696EEB
:100310006974206661696C656400534420696E6984
:1003200074206661696C006563686F3A00486172A9
:1003300064636F6465642044656661756C74205302
:10034000657474696E6773204C6F61646564002026
:1003500044002049002020204D33303120500050EF
:1003600049442073657474696E67733A00205A00BB
:1003700020590020204D323036205800486F6D65DE
:10038000206F666673657420286D6D293A002045DC
:1003900000205A0020580020420020540020204D08
:1003A000323035205300416476616E636564207697
:1003B00061726961626C65733A20533D4D696E20CC
:1003C000666565647261746520286D6D2F73292CD4
:1003D00020543D4D696E2074726176656C206665AF
:1003E00065647261746520286D6D2F73292C20421D
:1003F0003D6D696E696D756D207365676D656E74B1
:100400002074696D6520286D73292C20583D6D611D
:1004100078696D756D205859206A65726B20286D5A
:100420006D2F73292C20205A3D6D6178696D756D93
:10043000205A206A65726B20286D6D2F73292C203D
:1004400020453D6D6178696D756D2045206A657246
:100450006B20286D6D2F73290020540020204D3211
:100460003034205300416363656C65726174696F59
:100470006E3A20533D616363656C65726174696FA8
:100480006E2C20543D7265747261637420616363E5
:10049000656C65726174696F6E00204500205A00BA
:1004A00020590020204D3230312058004D617869AC
:1004B0006D756D20416363656C65726174696F6E03
:1004C00020286D6D2F7332293A00204500205A00F4
:1004D00020590020204D3230332058004D6178697A
:1004E0006D756D2066656564726174657320286D35
:1004F0006D2F73293A00204500205A002059002012
:10050000204D393220580053746570732070657225
:1005100020756E69743A006563686F3A00457272BF
:100520006F723A0053544F505045442E2000507281
:10053000696E7465722073746F7070656420647581
:100540006520746F206572726F72732E2046697811
:1005500020746865206572726F7220616E64207508
:100560007365204D39393920746F20726573746159
:1005700072742E202854656D706572617475726591
:100580002069732072657365742E20536574206929
:100590007420616674657220726573746172746927
:1005A0006E6729004B494C4C45442E20005072691F
:1005B0006E7465722068616C7465642E206B696C62
:1005C0006C28292063616C6C656421006F6B00529C
:1005D0006573656E643A20002200556E6B6E6F770E
:1005E0006E20636F6D6D616E643A20220043686116
:1005F0006E67652066696C616D656E74006C63641E
:1006000020636F6E74726173742076616C75653AE5
:1006100020007A5F6D696E3A2000795F6D696E3AED
:100620002000785F6D696E3A20005A3A00593A000E
:1006300020436F756E7420583A2000453A005A3AAC
:1006400000593A00583A004649524D574152455FC9
:100650004E414D453A4D61726C696E2056313B20DA
:10066000537072696E7465722F6772626C206D616F
:100670007368757020666F722067656E3620464914
:10068000524D574152455F55524C3A687474703A16
:100690002F2F7777772E6D656E64656C2D70617284
:1006A00074732E636F6D2050524F544F434F4C5F05
:1006B00056455253494F4E3A312E30204D41434812
:1006C000494E455F545950453A7777772E637265A6
:1006D000616C69747933642E636E204558545255A9
:1006E0004445525F434F554E543A31205555494485
:1006F0003A30303030303030302D303030302D30F6
:100700003030302D303030302D30303030303030EF
:1007100030303030300A007777772E637265616C45
:1007200069747933642E636E204F66662E004265CD
:100730006420646F6E652E0020423A0020453A0026
:10074000543A004265642048656174696E672E0002
:1007500048656174696E6720646F6E652E00204580
:100760003A00543A0048656174696E672E2E2E0077
:100770002042403A0020403A00202F003A00205406
:1007800000202F0020423A00202F006F6B20543AA7
:10079000002569206D696E2C202569207365630032
:1007A000456E642066696C65206C697374004265EF
:1007B00067696E2066696C65206C697374004E6FA2
:1007C000206D6F76652E00526573756D696E6720BA
:1007D0007072696E74005761697420666F7220755B
:1007E0007365722E2E2E00536C6565702E2E2E00B2
:1007F000FFFFFF00006B4300006B430000824300DB
:1008000000A0400000A0400000803F000000000069
:1008100000000000000000000000000000000000D8
:1008200000000000006B4300006B43000082432582
:100830006920686F757273202569206D696E757403
:10084000657300446F6E65207072696E74696E67BF
:100850002066696C650053544F505045442E20006B
:100860005072696E7465722073746F707065642065
:1008700064756520746F206572726F72732E2046E6
:10088000697820746865206572726F7220616E6489
:1008900020757365204D39393920746F2072657366
:1008A000746172742E202854656D70657261747560
:1008B00072652069732072657365742E20536574A8
:1008C0002069742061667465722072657374617248
:1008D00074696E6729006F6B004E6F204C696E65FE
:1008E000204E756D62657220776974682063686553
:1008F000636B73756D2C204C617374204C696E654D
:100900003A20004E6F20436865636B73756D2077E6
:10091000697468206C696E65206E756D6265722CF5
:10092000204C617374204C696E653A2000636865E1
:10093000636B73756D206D69736D617463682C20D2
:100940004C617374204C696E653A20004C696E6589
:10095000204E756D626572206973206E6F74204C35
:10096000617374204C696E65204E756D6265722BE3
:10097000312C204C617374204C696E653A20004D17
:1009800031313000446F6E6520736176696E672087
:1009900066696C652E006F6B004D32390020205067
:1009A0006C616E6E657242756666657242797465D9
:1009B000733A20002046726565204D656D6F72792F
:1009C0003A20004D617220323820323031380043F5
:1009D0006F6D70696C65643A200028456E646572BD
:1009E000332900207C20417574686F723A20004DD5
:1009F000617220323820323031382030393A31318A
:100A00003A333800204C617374205570646174650A
:100A1000643A2000312E302E30004D61726C696EC8
:100A2000200020536F66747761726520526573658C
:100A30007400205761746368646F67205265736542
:100A400074002042726F776E206F75742052657348
:100A50006574002045787465726E616C2052657310
:100A6000657400506F7765725570007374617274AD
:100A70000062696E004D31313720494E56414C4974
:100A80004420444154412E004D3131372050726989
:100A90006E74696E672E2E2E004730205A25730023
:100AA000473238205830205930004730205A2573BB
:100AB00000473932205A2573204525730062696E3C
:100AC000002200656E717565696E672022007C3CAE
:100AD0003E5E2B3D3F2F5B5D3B2C2A225C00453167
:100AE0003A200045303A20005A3A2000593A200076
:100AF000583A20004D53312C4D53322050696E73BB
:100B00000A0024F404D9201BC40C5C0E9804C40908
:100B10005F0265077101F405F900FB04B3004804A6
:100B20008700C10369005803550003034500BE0256
:100B30003A008402310053022A00290225000402EF
:100B40002000E4011C00C8011900AF011700980142
:100B500014008401130071011000610110005101A3
:100B60000E0043010D0036010B002B010B0020018C
:100B70000B00150109000C01090003010800FB002E
:100B80000800F3000800EB000700E4000600DE00A8
:100B90000600D8000600D2000600CC000500C70001
:100BA0000500C2000500BD000400B9000400B50046
:100BB0000400B1000400AD000400A9000400A50079
:100BC0000300A20003009F0004009B0003009800A4
:100BD00003009500020093000300900003008D00C5
:100BE00002008B00030088000200860002008400DF
:100BF0000300810002007F0002007D0002007B00F4
:100C00000200790002007700010076000200740003
:100C1000020072000100710002006F0002006D000E
:100C200001006C0002006A00010069000200670018
:100C3000010066000100650001006400020062001E
:100C4000010061000100600001005F0002005D0022
:100C500001005C0001005B0001005A000100590026
:100C60000100580001005700010056000100550026
:100C70000100540001005300000053000100520025
:100C8000010051000100500001004F0001004E0022
:100C900000004E0001004D0001004C0001004B001F
:100CA00000004B0001004A0001004900010048001B
:100CB0000000480001004700010046000000460017
:100CC0000100450000004500010044000100430010
:100CD000000043000100420000004200010041000A
:100CE000000041000100400001003F0000003F0003
:100CF00001003E0000003E0001003D0000003D00FC
:100D000001003C0000003C0000003C0001003B00F2
:100D100000003B0001003A0000003A0001003900E9
:100D200000003900010038000000380000003800E1
:100D300001003700000037000100360000003600D7
:100D400000003600010035000000350000003500CD
:100D500001003400000034000000340001003300C2
:100D600000003300000033000100320000003200B8
:100D700000003200010031000000310000003100AD
:100D800001003000000030000000300001002F00A2
:100D900000002F0000002F0000002F0001002E0097
:100DA00000002E0000002E0001002D0000002D008C
:100DB00000002D0000002D0001002C0000002C0080
:100DC00000002C0000002C0001002B0000002B0074
:100DD00000002B0000002B0001002A0000002A0068
:100DE00000002A0000002A0001002900000029005C
:100DF000000029000000290000002900010028004F
:100E00000000280000002800000028000000280042
:100E10000100270000002700000027000000270035
:100E20000000270001002600000026000000260028
:100E3000000026000000260001002500000025001B
:100E4000000025000000250000002500000025000E
:100E50000100240000002400000024000000240001
:100E600000002400010023000000230000002300F4
:100E700000002300000023000000230000002300E6
:100E800001002200000022000000220000002200D9
:100E900000002200000022000100210000002100CB
:100EA00000002100000021000000210000002100BE
:100EB00000002100010020000000200000002000B0
:100EC00000002000000020000000200000002000A2
:100ED0000000200001001F0000001F0000001F0094
:100EE00000001F0000001F0000001F0000001F0086
:100EF00001001E0000001E0000001E0000001E0079
:100F0000000024F4D43050C38E20C2A24017828B3C
:100F10007011127A910D816CD90AA861E108C75845
:100F20006607615143061E4B5D05C145A7041A4182
:100F30001104093D9803713931034036DB026533F2
:100F40009102D4305402802E1D02632CEE01752ACA
:100F5000C501B028A001102781018F2564012B2431
:100F60004B01E0223401AC211F018D200D01801FB7
:100F7000FC00841EED00971DDF00B81CD200E61BAC
:100F8000C600201BBC00641AB200B219A8000A19DE
:100F9000A0006A189900D117910040178B00B51670
:100FA000840031167E00B31579003A157300C7141A
:100FB0006F0058146A00EE1366008813630025134F
:100FC0005E00C7125B006C12570015125400C1116D
:100FD000510070114F0021114B00D61049008D10A7
:100FE00047004610440002104200C00F4000800F2E
:100FF0003E00420F3C00060F3B00CB0E3800930E24
:1010000037005C0E3500270E3400F30D3200C10DA1
:101010003100900D3000600D2E00320D2D00050DB9
:101020002C00D90C2B00AE0C2900850C29005C0C7F
:101030002700350C27000E0C2600E80B2400C40BFB
:101040002400A00B23007D0B23005A0B2100390B39
:101050002100180B2000F80A1F00D90A1E00BB0A45
:101060001E009D0A1D00800A1D00630A1C00470A1D
:101070001B002C0A1B00110A1A00F7091A00DD09CF
:101080001900C4091900AB091900920917007B095E
:101090001800630917004C091600360916002009CC
:1010A00016000A091500F5081500E0081400CC0820
:1010B0001400B8081400A4081400900813007D0858
:1010C00012006B081300580812004608120034087A
:1010D0001100230811001208110001081100F00787
:1010E0001000E0071000D0071000C0071000B00784
:1010F0000F00A107100091070E0083070F0074076F
:101100000F0065070E0057070E0049070E003B074A
:101110000D002E070E0020070D0013070D00060717
:101120000D00F9060C00ED060D00E0060C00D406DB
:101130000C00C8060C00BC060C00B0060C00A4068F
:101140000B0099060C008D060B0082060B0077063B
:101150000B006C060B0061060A0057060B004C06DC
:101160000A0042060A0038060A002E060A00240673
:101170000A001A060A001006090007060A00FD0503
:101180000900F4050900EB050900E2050900D9058D
:101190000900D0050900C7050900BE050900B5050D
:1011A0000800AD050800A50509009C050800940588
:1011B00008008C050800840508007C0508007405FB
:1011C00008006C050700650508005D050700560569
:1011D00008004E05070047050700400508003805D0
:1011E0000700310507002A050700230507001C0535
:1011F0000600160507000F05070008050600020592
:101200000700FB040600F5040700EE040600E804EE
:101210000600E2040700DB040600D5040600CF0444
:101220000600C9040600C3040600BD040600B70496
:101230000600B1040500AC040600A6040600A004E4
:1012400005009B04060095040500900406008A042E
:10125000050085040500800406007A040500750475
:101260000500700405006B040500660405006104B8
:1012700005005C04050057040500520405004D04F8
:10128000050048040500430405003E0404003A0438
:10129000050035040500300404002C040500270473
:1012A0000400230405001E0404001A0404001604AC
:1012B0000500110404000D040400090405000404E1
:1012C000040000040400FC030400F8030400F40319
:1012D0000400F0030400EC030400E8030400E4034A
:1012E0000400E0030400DC030400D8030400D4037A
:1012F0000400D0030400CC030400C8030300C503AA
:1013000003006563686F3A00656E6473746F707391
:10131000206869743A205A00205A3A00656E647356
:10132000746F7073206869743A20590020593A002C
:10133000656E6473746F7073206869743A20580026
:1013400020583A00656E6473746F70732068697416
:101350003A20004572726F723A004572723A204D1F
:10136000415854454D50204245440054656D7065C8
:101370007261747572652068656174656420626568
:1013800064207377697463686564206F66662E20D5
:101390004D415854454D50207472696767657265B8
:1013A00064202121004572723A204D494E54454D2A
:1013B00050003A20457874727564657220737769BD
:1013C0007463686564206F66662E204D494E5445EF
:1013D0004D5020747269676765726564202100450D
:1013E00072723A204D415854454D50003A2045788C
:1013F00074727564657220737769746368656420BC
:101400006F66662E204D415854454D5020747269C8
:10141000676765726564202100202D20496E766122
:101420006C6964206578747275646572206E756D80
:1014300062657220210070012C0190012701B0012A
:101440002201C0011D01F001180110021301300238
:101450000E016002090190020401C002FF000003B6
:10146000FA004003F5008003F000D003EB002004F5
:10147000E6007004E100E004DC004005D700C00590
:10148000D2004006CD00D006C8008007C300300857
:10149000BE00F008B900C009B400B00AAF00B00B3C
:1014A000AA00D00CA500000EA000500F9B00C01099
:1014B00096005012910000148C00C0158700B017E0
:1014C0008200B0197D00D01B7800001E7300402000
:1014D0006E0090226900F024640040275F0090298C
:1014E0005A00E02B5500102E500020304B001032D7
:1014F0004600E033410090353C001037370070382B
:101500003200A0392D00B03A2800A03B2300603CF7
:101510001E00103D1900903D1400103E0F00703E5B
:101520000A00C03E0500003F0000504944204175BC
:10153000746F74756E652066696E69736865642181
:101540002050757420746865204B702C204B6920E6
:10155000616E64204B6420636F6E7374616E74738C
:1015600020696E746F20436F6E666967757261746F
:10157000696F6E2E6800504944204175746F747510
:101580006E65206661696C6564212074696D656FA4
:1015900075740020403A006F6B20543A006F6B2046
:1015A000423A00504944204175746F74756E65204D
:1015B0006661696C6564212054656D706572617443
:1015C00075726520746F6F206869676800204B64CE
:1015D0003A2000204B693A2000204B703A2000202E
:1015E000436C617369632050494420002054753A6C
:1015F0002000204B753A2000206D61783A200020B1
:101600006D696E3A200020643A200020626961739F
:101610003A20000000000000000000000000000070
:101620003FFFF0000000000000000000000000008C
:101630003800700000000000000000000000000002
:1016400033873000000000000000000000000000B0
:10165000278790000000000000000000000000004C
:101660002F87D000000000000000000000000000F4
:101670002F87D000000000000000000000000000E4
:101680002F03D0F80180000C1FE00000082080002C
:1016900020301048008000123FF00000041040008D
:1016A00020781043C38CD0023FF0000004104000AB
:1016B00020781071249267CC3FF000000820800051
:1016C00020301041249E40021FE000001041000025
:1016D0002F03D049249040121FE000002082000018
:1016E0002F87D0FBB3CEE00C3FF00000208200003B
:1016F0002F87D000000000003FF0000010410000E4
:1017000027879000000000003FF0000008208000C4
:1017100033873000000000000FC000000000000010
:10172000380070000000000007800000FFFFC000CC
:101730003FFFF0000000000003000000FFFFC000BA
:101740000000000000000000000000000000000099
:101750003FFFF0000000000000000000000000005B
:1017600038007000000000000000000000000000D1
:1017700030FC30000000000000000000000000000D
:1017800020FC10000000000000000000000000002D
:1017900020781000000000000000000000000000A1
:1017A00020301000000000000000000000000000D9
:1017B0002C00D0F80180000C1FE000001041000058
:1017C0002E31D048008000123FF000000820800039
:1017D0002F7BD043C38CD0023FF000000820800054
:1017E0002F7BD071249267CC3FF0000010410000A5
:1017F0002E31D041249E40021FE0000020820000D4
:101800002C00D049249040121FE000004104000049
:10181000203010FBB3CEE00C3FF00000410400008C
:1018200020781000000000003FF00000208200003F
:1018300020FC1000000000003FF0000010410000FC
:1018400030FC3000000000000FC00000000000006D
:10185000380070000000000007800000FFFFC0009B
:101860003FFFF0000000000003000000FFFFC00089
:101870000000005900B02000B02000B02000B020CF
:10188000002D2D3A2D2D004D323100496E69742EF8
:101890002053442D43617264004E6F204361726493
:1018A000004D3231004368616E67652053442D431B
:1018B000617264005072696E742066726F6D20539D
:1018C000440053746F70205072696E7400526573D7
:1018D000756D65205072696E740050617573652076
:1018E0005072696E7400436F6E74726F6C00507248
:1018F00065706172650054756E6500496E666F2093
:1019000073637265656E00F92E2E00F8526566727B
:10191000657368004D61696E004D3234004D32339D
:10192000202573004D383420582059205A20450076
:10193000473238205830205930004D31303620534E
:10194000323535004D31303920532569004D31395C
:101950003020532569004732382058302059300054
:10196000526573746F7265204661696C7361666558
:101970000054656D7065726174757265004D6169C2
:101980006E0046616E2073706565640046616E206E
:1019900073706565640042656400426564004E6F63
:1019A0007A7A6C65004E6F7A7A6C6500436F6E745C
:1019B000726F6C004D6F7665204178697300436FDC
:1019C0006F6C646F776E005072656865617420415A
:1019D0004253005072656865617420504C41004765
:1019E0003238004175746F20486F6D65004D383492
:1019F0000044697361626C65205374657070657230
:101A000073004D61696E004D6F766520302E316D2B
:101A10006D004D6F766520316D6D004D6F766520E0
:101A200031306D6D0050726570617265004578747B
:101A30007275646572004D6F7665205A004D6F7641
:101A4000652059004D6F76652058004D6F766520F2
:101A500041786973004578747275646572005A0044
:101A6000590058004D363030004368616E6765207C
:101A700066696C616D656E7400466C6F7700466CCC
:101A80006F770046616E2073706565640046616E15
:101A90002073706565640042656400426564004EB1
:101AA0006F7A7A6C65004E6F7A7A6C650053706558
:101AB0006564005370656564004D61696E004E6F2A
:101AC0000059657300526573756D65205072696EBB
:101AD000743F00FFFFFFFFFFFFFFFFFFFFFFFFFF60
:101AE000FFFFFFFFFFFFFFFFFFFFFFFFFFFFFFFF06
:101AF000FFFFFFFFFFFFFFFFFFFFFFFFFFFFFFFFF6
:101B0000FFFFFFFFFFFFFFFFFFFFEFFFFFFFFFFFF5
:101B1000FFFFFFFFFFFFFFFFFFFFEFEFFFFFFFFFF5
:101B2000FFFFFFFFFFFFFFFFFFFFE7DFFFFFFFFFFD
:101B3000FFFFFFFFFFFFFFFFFFFFE7DFFFFFFFFFED
:101B4000FFFFFFFFFFFFFFFFFFFFE3DFFFFFFFFFE1
:101B5000FFFFFFFFFFFFFFFFFFFFF3CFFFFFFFFFD1
:101B6000FFFFFFFFFFFFFFFFFFE1E1CFFFFFFFFFF1
:101B7000FFFFFFFFFFFFFFFE78000003DDFFFFFF19
:101B8000FFFFFFFFFFFFFEFF807E0001EEFFFFFF74
:101B9000FFFFFFFFFFFFFE7DCFFC0000F77FFFFF91
:101BA000FFFFFFFFFFFFFF8E060000007BBFFFFF70
:101BB000FFFFFFFFFFFFFFC0000000007DDFFFFF12
:101BC000FFFFFFFFFFFFFFFC01FE00003EE7FFFFFE
:101BD000FFFFFFFFFFFFFFFFFFFC00031F73FFFF7F
:101BE000FFFFFFFFFFFFFFFFFFF800018F81FFFFF7
:101BF000FFFFFFFFFFFFFFFFFFE0000083F9FFFF94
:101C0000FFFFFFFFFFFFFFFFFF00FC0000F0FFFFF3
:101C1000FFFFFFFFFFFFFFFFE00FFFC00000FFFF20
:101C2000FFFFFFFFFFFFFFFE03FFFFC00000FFFFFE
:101C3000FFFFFFFFFFFFFFFFFFFFF9000000FFFFB7
:101C4000FFFFFFFFFFFFFFFFFFFFFC0007C0FFFFDD
:101C5000FFFFFFFFFFFFFFFFFFFFFF0007E0FFFFAA
:101C6000FFFFFFFFFFFFFFFFFFFFFFE007F1FFFFA9
:101C7000FFFFFFFFFFFFFFFFFFFFFFFC07F9FFFF75
:101C8000FFFFFFFFFFFFFFFFFFFFFFFF03F9FFFF66
:101C9000FFFFFFFFFFFFFFFFFFFFFFFF83F9FFFFD6
:101CA000FFFFFFFFFFFFFFFFFFFFFFFFC3FFFFFF80
:101CB000FFFFFFFFFFFFFFFFFFFFFFFFE1FFFFFF52
:101CC000FFFFFFFFFFFFFFFFFFFFFFFFF0BFFFFF73
:101CD000FFFFFFFFFFFFFFFFFFFFFFFBF83FFFFFDF
:101CE000FFFFFFFFFFFFFFFFFFFFFFF9F83FFFFFD1
:101CF000FFFFFFFFFFFFFFFFFFFFFF7EF0FFFFFF84
:101D0000FFFFFFFFFFFFFFFFFFFFFF8E03FFFFFF50
:101D1000FFFFFFFFFFFFFFFFFFFFFFE01FFFFFFFD2
:101D2000FFFFFFFFFFFFFFFFFFFFFFFFFFFFFFFFC3
:101D3000FFFFFFFFFFFFFFFFFFFFFFFFFFFFFFFFB3
:101D4000FFFFFFFFFFFFFFFFFFFFFFFFFF7FFFFF23
:101D5000FFFFFFFFFFFFFF00007FFFFFF87FFFFF98
:101D6000FFFFFFFFFFFFFF80007FFFFFE07FFFFF20
:101D7000FFFFFFFFFFFFFFC3FCFFFFFFF8FFFFFFB9
:101D8000FFFFFFFFFFFFFFC3FCFFFFFFF8FFFFFFA9
:101D9000FFFFFFFFFFFFFF87FDFFFFFFF1FFFFFFDB
:101DA000FFFFFFFFFFFFFF87FFFFFFFFF1FFFFFFC9
:101DB000FFFFFFFFFFFFFF0FE7F30FFC23FC3FFFD9
:101DC000FFFFFFFFFFFFFF0FEF8007F003F01E0094
:101DD0007FFFFFFFFFFFFE1FCF8187C787C70C0074
:101DE0007FFFFFFFFFFFFE001FC7C78FC79F0F0CBE
:101DF000FFFFFFFFFFFFFE001F878F1F8F1F0F1FBB
:101E0000FFFFFFFFFFFFFC3F9F8F8F1F8E001E3FD6
:101E1000FFFFFFFFFFFFFC7F3F0F1E3F1E3FFE3F08
:101E2000FFFFFFFFFFFFF87FFF1F1C3F1C7FFC7FB2
:101E3000FFFFFFFFFFFFF8FFFF1E1C7E1C7FFC7FE4
:101E4000FFFFFFFFFFFFF0FFCE3E3C7E3C7FB8FF71
:101E5000FFFFFFFFFFFFF0FF9E3C387C387E78FFDE
:101E6000FFFFFFFFFFFFE1FF3C7C787C783CF1FF48
:101E7000FFFFFFFFFFFFE1F8387878101801F1FF4E
:101E8000FFFFFFFFFFFF000060203C007C07807F1A
:101E9000FFFFFFFFFFFFFFFFFFFFFE1FFE1FFFFF14
:101EA000FFFFFFFFFFFFFFFFFFFFFFFFFFFFFFFF42
:101EB000FFFFFFFFFFFFFFFFFFFFFFFFFFFFFFFF32
:101EC000FFFFFFFFFFFFFFFFFFFFFFFFFFFFFFFF22
:101ED000FFFFFF00060900FE06018902FE20FFFE4B
:101EE00007FE06FE000000060007010606060200C7
:101EF000808080800080030303060103A0A0A0056A
:101F000007070600FF5050F850F850500509090621
:101F100000FE2070A8A07028A870200608080600FF
:101F2000FF40A84810204854080507070600FF6036
:101F300090906098906801030306020380808002FD
:101F400007070602FF408080808080400207070666
:101F500002FF8040404040408005050506000088A3
:101F600050F850880505050600002020F8202002C2
:101F700004040602FEC0404080050101060002F88C
:101F8000020202060200C0C004060606010010108C
:101F900020408080040606060100609090909060CA
:101FA00003060606010040C0404040E00406060665
:101FB00001006090102040F0040606060100F020A9
:101FC000601010E005060606000010305090F81072
:101FD000040606060100F080E01010E00406060684
:101FE00001006080E0909060040606060100F01099
:101FF000102040400406060601006090609090604A
:102000000406060601006090907010600205050647
:102010000200C0C000C0C00207070602FEC0C00028
:10202000C040408005050506000018608060180566
:102030000303060001F800F8050505060000C0309E
:102040000830C0040707060100609010604000409F
:102050000506060600007090A8B08070050606060A
:102060000000205088F88888050606060000F088E1
:10207000F08888F004060606010060908080906079
:10208000040606060100E090909090E00406060623
:102090000100F080E08080F0040606060100F08078
:1020A000E0808080040606060100609080B09060A9
:1020B0000406060601009090F09090900306060634
:1020C0000100E040404040E00506060600003810F0
:1020D0001010906004060606010090A0C0A0909029
:1020E0000406060601008080808080F00506060652
:1020F000000088D8A8A8888804060606010090D0A9
:10210000B090909005060606000070888888887058
:10211000040606060100E09090E0808004070706B0
:1021200001FF609090D0B06010040606060100E048
:102130009090E09090040606060100609040209088
:1021400060050606060000F8202020202004060670
:1021500006010090909090906004060606010090A1
:102160009090F060600506060600008888A8A8D850
:1021700088050606060000885020205088050606BF
:10218000060000888850202020040606060100F082
:1021900010204080F0030606060100E08080808069
:1021A000E0040606060100808040201010030606A9
:1021B000060100E020202020E005030306000320A4
:1021C00050880501010600FEF802020206020480A2
:1021D0004004040406010070909070040606060195
:1021E000008080E09090E00404040601007080808C
:1021F000700406060601001010709090700404042C
:1022000006010060B0C070040606060100205040C0
:10221000E040400406060601FE60909070106004E5
:1022200006060601008080E09090900306060601F5
:10223000004000C04040E00308080601FE200060A6
:10224000202020A0400406060601008080A0C0A037
:1022500090030606060100C040404040E00504042B
:10226000060000D0A8A888040404060100E09090AD
:1022700090040404060100609090600406060601C4
:10228000FEE09090E080800406060601FE709090CB
:10229000701010040404060100A0D080800404041F
:1022A00006010070C030E00406060601004040E070
:1022B000405020040404060100909090700404042F
:1022C0000601009090606005040406000088A8A83C
:1022D00050040404060100906060900406060601A4
:1022E000FE909090709060040404060100F020407D
:1022F000F00307070601002040408040402001070E
:10230000070602FF80808080808080030707060127
:10231000008040402040408004020206010350A09B
:10232000FFFFFFFFFFFFFFFFFFFFFFFFFFFFFFFFBD
:10233000FFFFFFFFFFFFFFFFFFFFFFFFFFFFFFFFAD
:10234000FF0000000600070106060602008000806C
:102350008080800406060601FF2070A0A070200582
:1023600007070600FF304840F04040F80505050625
:102370000000A8508850A80506060600008850F8FE
:1023800020F8200107070602FF80808000808080FF
:102390000407070601FF708060906010E0030101F0
:1023A000060105A0060707060000788494A494841B
:1023B0007803050506010160A06000E0050505063B
:1023C00000002850A05028040303060100F010105C
:1023D000040101060102F00607070600007884B434
:1023E000A4A48478040101060105F0040303060196
:1023F000026090600507070600FF2020F8202000FB
:10240000F803050506010140A02040E0030505068C
:102410000101C0204020C0020202060204408004E4
:1024200005050601FF9090B0D08005060606000065
:1024300078E8E86828280101010602028002020209
:102440000602FE408003050506010140C04040E051
:1024500003050506010140A04000E0050505060052
:1024600000A0502850A00508080600FF40C04050BA
:10247000703078100508080600FF40C0405068081A
:1024800010380508080600FFC0204030F0307810F2
:102490000407070601002000206080906005070700
:1024A00006000040202050708888050707060000BD
:1024B0001020205070888805070706000020502053
:1024C0005070888805070706000028502050708843
:1024D000880507070600005000205070888805070F
:1024E0000706000020502050708888050606060068
:1024F0000078A0F0A0A0B80408080601FE60908053
:1025000080906020400407070601004020F080E032
:1025100080F00407070601002040F080E080F0040E
:1025200007070601002050F080E080F0040707064E
:1025300001005000F080E080F003070706010080F2
:1025400040E0404040E00307070601002040E04033
:102550004040E003070706010040A0E0404040E0A3
:10256000030707060100A000E0404040E005060622
:102570000600007048E8484870040707060100504C
:10258000A090D0B090900407070601004020609012
:1025900090906004070706010020406090909060D2
:1025A0000407070601002050609090906004070720
:1025B00006010050A060909090600407070601009B
:1025C000500060909090600505050600008850203E
:1025D00050880408080601FF1070B0B0D0D0E08029
:1025E00004070706010040209090909060040707C0
:1025F00006010020409090909060040707060100BB
:1026000020509090909060040707060100500090C1
:102610009090906005070706000010208850202049
:102620002004060606010080E09090E08004060683
:102630000601006090A0A090A004070706010040DA
:102640002000709090700407070601002040007081
:102650009090700407070601002050007090907061
:1026600004070706010050A0007090907004060651
:1026700006010050007090907004070706010020CA
:1026800050207090907005040406000070A8B07887
:102690000406060601FE70808070204004070706CD
:1026A000010040200060B0C0700407070601002050
:1026B000400060B0C07004070706010020500060B1
:1026C000B0C070040606060100500060B0C0700380
:1026D0000707060100804000C04040E003070706EE
:1026E0000100204000C04040E00307070601004011
:1026F000A000C04040E0030606060100A000C04064
:1027000040E00407070601003060107090906004FC
:10271000070706010050A000E0909090040707060C
:10272000010040200060909060040707060100202F
:102730004000609090600407070601002050006090
:1027400090906004070706010050A0006090906020
:10275000040606060100500060909060050505061D
:1027600000002000F8002004040406010070B0D02E
:10277000E0040707060100402000909090700407D5
:1027800007060100204000909090700407070601A2
:102790000020500090909070040606060100500042
:1027A000909090700409090601FE204000909090DE
:1027B0007090600408080601FE8080E09090E08040
:1027C000800408080601FE50009090907090600010
:1027D000060900FE070199032B20FFFE08FE07FEF5
:1027E00000000006000001070706020080808080CC
:1027F000800080030303060104A0A0A005070706CC
:1028000000005050F850F85050050707060000200F
:1028100070A07028702005070706000048A8502007
:1028200050A89005070706000040A0A040A89068A7
:1028300001030306020480808003070706010020CD
:102840004080808040200307070601008040202050
:102850002040800505050600018850F850880505D0
:10286000050600012020F820200303030601FF6075
:102870004080050101060003F80303030601FF4041
:10288000E04005070706000008081020408080058A
:102890000707060000205088888850200507070693
:1028A00000002060A0202020F80507070600007027
:1028B0008808304080F8050707060000F808103047
:1028C00008887005070706000010305090F81010B7
:1028D000050707060000F880B0C8088870050707DC
:1028E000060000304080B0C8887005070706000069
:1028F000F80810102040400507070600007088887F
:1029000070888870050707060000708898680810AE
:10291000600307070601FF40E0400040E040030776
:10292000070601FF40E04000604080040707060101
:102930000010204080402010050303060002F8002C
:10294000F80407070601008040201020408005079A
:1029500007060000708810202000200507070600E9
:1029600000708898A8B08070050707060000205006
:102970008888F88888050707060000F048487048EE
:1029800048F0050707060000708880808088700581
:102990000707060000F04848484848F005070706C2
:1029A0000000F88080F08080F8050707060000F836
:1029B0008080F08080800507070600007088808096
:1029C000988870050707060000888888F888888836
:1029D000030707060100E04040404040E0050707CC
:1029E0000600003810101010906005070706000060
:1029F0008890A0C0A090880507070600008080800E
:102A0000808080F80507070600008888D8A8888895
:102A1000880507070600008888C8A89888880507E1
:102A200007060000708888888888700507070600F8
:102A300000F08888F08080800508080600FF708814
:102A4000888888A87008050707060000F08888F0C5
:102A5000A0908805070706000070888070088870BD
:102A6000050707060000F820202020202005070782
:102A70000600008888888888887005070706000097
:102A800088888850505020050707060000888888ED
:102A9000A8A8D88805070706000088885020508815
:102AA0008805070706000088885020202020050799
:102AB00007060000F80810204080F8030707060109
:102AC00000E08080808080E00507070600008080AD
:102AD0004020100808030707060100E020202020FE
:102AE00020E00503030600042050880501010600CC
:102AF000FFF80202020602068040050505060000F6
:102B000070087888780507070600008080B0C888BC
:102B1000C8B00505050600007088808870050707A5
:102B200006000008086898889868050505060000F2
:102B30007088F88070050707060000304840F040B4
:102B400040400507070600FE7888887808887005E9
:102B500007070600008080B0C8888888030707063A
:102B600001004000C0404040E00409090601FE1099
:102B7000003010101090906005070706000080805C
:102B80008890E09088030707060100C0404040405D
:102B900040E0050505060000D0A8A8A888050505A1
:102BA000060000B0C8888888050505060000708802
:102BB0008888700507070600FEB0C888C8B0808006
:102BC0000507070600FE6898889868080805050547
:102BD000060000B0C88080800505050600007080F2
:102BE0007008F00507070600004040F040404830FC
:102BF0000505050600008888889868050505060013
:102C00000088885050200505050600008888A8A87F
:102C10005005050506000088502050880507070666
:102C200000FE88889868088870050505060000F889
:102C3000102040F8040707060100304020C0204063
:102C400030010707060200808080808080800407B2
:102C500007060100C02040304020C00503030600E5
:102C60000448A890000000010000000000010000DE
:102C70000000000100000000000100000000000151
:102C80000000000000010000000000010000000042
:102C90000001000000000001000000000001000031
:102CA0000000000100000000000100000000000121
:102CB0000000000000010000000000010000000012
:102CC0000001000000000001000000000001000001
:102CD00000000001000000000001000000000001F1
:102CE00000000000000100000000000100000000E2
:102CF00000010000000000010000000000010000D1
:102D000000000001000000000001000000000001C0
:102D100000000000000100000000000100000000B1
:102D2000000100000000000100000000000600009B
:102D30000107070602008000808080808005070769
:102D40000600FF2078A0A0A0782005070706000055
:102D5000304840E04048B005050506000088705046
:102D600070880508080600FF88885020F820202079
:102D70000107070602008080800080808005080827
:102D80000600FF7080E090483808700301010601DA
:102D900007A00507070600007088A8C8A888700467
:102DA00006060601017090B05000F0060505060009
:102DB000002448904824040202060102F010040195
:102DC00001060103F00507070600007088E8C8C87F
:102DD0008870050101060007F8030303060104409B
:102DE000A0400506060600002020F82020F8040573
:102DF0000506010360902040F0040505060103E08C
:102E0000106010E002020206020640800506060677
:102E100000FF888888C8B08005070706000078E8AA
:102E2000E868282828010101060203800202020640
:102E300002FE408003050506010340C04040E00457
:102E400006060601016090906000F0060505060088
:102E50000090482448900609090600FF40C0404001
:102E6000E40C143C040609090600FF40C04040E899
:102E70001404081C0509090600FFC0204020C818DA
:102E800028780805070706000020002020408870E9
:102E90000508080600004020708888F88888050822
:102EA000080600001020708888F888880508080641
:102EB00000002050708888F88888050808060000FF
:102EC00048B0708888F88888050808060000500017
:102ED000708888F8888805080806000020507088E7
:102EE00088F888880607070600003C50909CF09000
:102EF0009C0509090600FE7088808080887020404B
:102F000005080806000040F88080F08080F8050879
:102F10000806000010F88080F08080F80508080698
:102F2000000020F88080F08080F805080806000086
:102F300050F88080F08080F8030808060100804087
:102F4000E040404040E00308080601002040E04027
:102F5000404040E003080806010040A0E040404037
:102F600040E0030808060100A000E040404040E0C7
:102F7000050707060000F04848E84848F00508083B
:102F8000060000285088C8A8988888050808060008
:102F900000402070888888887005080806000010A6
:102FA0002070888888887005080806000020507006
:102FB000888888887005080806000028507088886E
:102FC0008888700508080600005000708888888886
:102FD0007005050506000088502050880507070683
:102FE0000000709898A8C8C870050808060000403E
:102FF00020888888888870050808060000102088C6
:103000008888888870050808060000205000888895
:10301000888870050808060000500088888888881D
:103020007005080806000010208888502020200520
:10303000070706000080F088F080808005070706FB
:103040000000708890A09088B00508080600004035
:103050002000700878887805080806000010200015
:10306000700878887805080806000020500070086D
:1030700078887805080806000028500070087888CD
:103080007805070706000050007008788878050862
:10309000080600002050207008788878060505068C
:1030A000000078147C907C0507070600FE7088807D
:1030B000887020400508080600004020007088F84D
:1030C00080700508080600001020007088F88070E5
:1030D0000508080600002050007088F88070050779
:1030E0000706000050007088F88070030808060189
:1030F00000804000C0404040E00308080601004056
:103100008000C0404040E003080806010040A000E5
:10311000C0404040E0060A0A0600FEA4A800FC8465
:1031200080808084FC060A0A0600FE549400FC8419
:1031300004040484FC050808060000285000B0C8F8
:103140008888880508080600004020007088888864
:1031500070040A0A0602FE30408090909090909091
:1031600090040A0A0600FEC0201090909090909063
:1031700090060707060001448C8C8480403C0607BB
:103180000706000188C4C4840408F005050506008C
:10319000012000F8002005080806000040F0C8885B
:1031A00088987810050808060000E0F88888888864
:1031B00088F80505050600012030F83020050808CC
:1031C0000600002070F820202020E00509090600F4
:1031D000FF2070A8A8B8888850200509090600FFBC
:1031E000E080C0B0A8A83028280509090600FFF82B
:1031F000A88888888888A8F8050A0A0600FE205052
:1032000050505088A8A8887000091200FC0A01E8F4
:1032100003D720FFFD0EFD0BFD00000009000E018D
:103220000B0B0904008080808080808000008080FB
:1032300004040409030790909090080A0A0900000A
:10324000242424FF2424FF242424070B0B0901FF3A
:10325000107C929050381412927C10070A0A0901CF
:103260000042A4A4481010244A4A84070A0A09010B
:103270000060909090606294889462010404090454
:103280000780808080030C0C0903FF204040808071
:1032900080808080404020030C0C0903FF80404068
:1032A000202020202020404080070707090103102C
:1032B000925438549210070707090101101010FEAC
:1032C0001010100204040904FEC0C0408007010170
:1032D000090104FE020202090400C0C0070A0A092B
:1032E000010002040408101020404080070A0A0967
:1032F000010038448282828282824438070A0A09A5
:103300000100103050901010101010FE070A0A092A
:103310000100384482020408102040FE070A0A090E
:103320000100FE020408180402028478070A0A0950
:103330000100040C14244484FE040404070A0A094E
:103340000100FE808080F80402028478070A0A09DE
:1033500001003C408080B8C482824438070A0A09D0
:103360000100FE020404080810101010070A0A09E0
:10337000010038448244384482824438070A0A09EA
:10338000010038448282463A0202047802070709A3
:103390000400C0C0000000C0C00209090904FEC04A
:1033A000C0000000C0C040800509090902000810E3
:1033B00020408040201008070404090102FE00009C
:1033C000FE050909090200804020100810204080F5
:1033D000070A0A090100384482020408101000108C
:1033E000070A0A09010038449AAAAAAAAA9C403CE2
:1033F000070A0A09010010282828447C4482828296
:10340000070A0A090100F8848284F884828284F819
:10341000070A0A0901003C42808080808080423C8B
:10342000070A0A090100F88482828282828284F873
:10343000070A0A090100FE808080F880808080FEF3
:10344000070A0A090100FE808080F8808080808061
:10345000070A0A09010038448280808E828244383B
:10346000070A0A09010082828282FE8282828282A7
:10347000050A0A090200F82020202020202020F838
:10348000070A0A0901003E08080808080888887029
:10349000070A0A09010082848890A0D08884828269
:1034A000070A0A090100808080808080808080FE79
:1034B000070A0A0901008282C6AA92828282828257
:1034C000070A0A0901008282C2A2928A8682828247
:1034D000070A0A0901007C82828282828282827CBF
:1034E000070A0A090100F884828284F880808080BB
:1034F000080B0B0901FF384482828282828A443A97
:1035000001070A0A090100F884828284F8908884FD
:1035100082070A0A0901007C8280807C0202028202
:103520007C070A0A090100FE10101010101010107C
:1035300010070A0A09010082828282828282824402
:1035400038070A0A09010082828244444428282854
:1035500010070A0A0901008282828292929292AA3C
:1035600044070A0A09010082824428101028448274
:1035700082070A0A090100828244281010101010E4
:1035800010070A0A090100FE02040810204080808A
:10359000FE040C0C0903FFF0808080808080808016
:1035A0008080F0070A0A09010080404020101008BE
:1035B000040402040C0C0902FFF01010101010108B
:1035C00010101010F00704040901061028448208A6
:1035D00001010900FFFF03030309030A80402007DC
:1035E00007070901007C02027E82867A070A0A091F
:1035F0000100808080BCC2828282C2BC07070709AA
:1036000001007C82808080827C070A0A0901000216
:1036100002027A86828282867A0707070901007C85
:103620008282FE80827C070A0A0901001C22222075
:1036300020F820202020070A0A0901FD7A848484CA
:1036400078807C82827C070A0A090100808080BC25
:10365000C28282828282050A0A090200600000E0BA
:103660002020202020F8050D0D0902FD180000384B
:10367000080808080808888870070A0A09010080F5
:103680008080848890B0C88482050A0A090200E01C
:103690002020202020202020F8070707090100EC27
:1036A000929292929282070707090100BCC282821D
:1036B0008282820707070901007C82828282827CE3
:1036C000070A0A0901FDB8C4828282C4B8808080DA
:1036D000070A0A0901FD3A46828282463A0202023C
:1036E0000707070901009C62424040404007070766
:1036F0000901007C82807C02827C070909090100A3
:103700002020FC20202020221C070707090100821E
:1037100082828282867A07070709010082824444F6
:103720002828100707070901008282929292AA4472
:1037300007070709010082442810284482070A0A63
:103740000901FD424224242418181090600707073D
:10375000090100FE0408102040FE060B0B090200C0
:103760001C20202020C0202020201C010C0C09043B
:10377000FF808080808080808080808080060B0B2E
:10378000090100E0101010100C10101010E00703D9
:103790000309010762928CFFFFFFFFFFFFFFFFFF9E
:1037A000FFFFFFFFFFFFFFFFFFFFFFFFFFFFFFFF29
:1037B000FFFFFFFFFFFFFFFF00000009000E010BEE
:1037C0000B0904008080000080808080808080065B
:1037D000080809010008789490A0A47840070A0A14
:1037E0000901001C222020F8202060A25C070606A8
:1037F000090103827C44447C82070A0A0901008291
:103800008244287C107C101010010B0B0904FF80EF
:1038100080808080008080808080040B0B0902FF04
:1038200060908060909090601090600302020903A5
:103830000BA0A00809090900013C4299A5A1A5997E
:10384000423C050707090103609070907800F80773
:103850000808090101122448909048241206040423
:10386000090102FC040404050101090204F8080925
:10387000090900013C42B9A5BDA9A5423C060101C8
:10388000090109FC0404040903066090906007091B
:1038900009090101101010FE10101000FE040606A8
:1038A0000901046090106080F004060609010460BC
:1038B000902010906003030309030A204080070949
:1038C000090901FE8282828282C6BA8080070A0AC2
:1038D0000901007E8A8A8A7A0A0A0A0A0A02020210
:1038E000090404C0C00403030902FD20906003061C
:1038F0000609010440C0404040E0050606090104F5
:103900007088887000F8070808090101904824129F
:1039100012244890070A0A09010040C0404042E6CC
:103920000A121A06070A0A09010040C040404CF278
:10393000020C101E070A0A0901006090201092660E
:103940000A121A06070A0A09010010001010204086
:103950008082827C070E0E090100201008001028CA
:103960002828447C44828282070E0E090100081038
:10397000200010282828447C44828282070E0E09E9
:1039800001001028440010282828447C44828282A8
:10399000070D0D09010034580010282828447C44E4
:1039A000828282070D0D090100282800102828288E
:1039B000447C44828282070E0E09010010282810E0
:1039C00010282828447C44828282070A0A090100C0
:1039D0001E2828284E784888888E070D0D0901FD7D
:1039E0003C42808080808080423C082418070E0E74
:1039F00009010020100800FE808080F8808080800F
:103A0000FE070E0E09010008102000FE808080F8DD
:103A100080808080FE070E0E09010010284400FE01
:103A2000808080F880808080FE070D0D09010028CD
:103A30002800FE808080F880808080FE050E0E09C0
:103A4000020040201000F82020202020202020F814
:103A5000050E0E09020010204000F8202020202032
:103A6000202020F8050E0E09020020508800F820C2
:103A700020202020202020F8050D0D0902005050A4
:103A800000F82020202020202020F8070A0A090121
:103A90000078444242F24242424478070D0D090147
:103AA000003458008282C2A2928A86828282070EE5
:103AB0000E090100201008007C82828282828282AC
:103AC000827C070E0E090100081020007C82828291
:103AD00082828282827C070E0E0901001028440037
:103AE0007C82828282828282827C070D0D090100A3
:103AF0003458007C82828282828282827C070D0D11
:103B00000901002828007C82828282828282827C53
:103B100007070709010182442810284482070C0C7A
:103B20000901FF027C868A8A9292A2A2C27C800747
:103B30000E0E090100201008008282828282828299
:103B4000824438070E0E090100081020008282828C
:103B500082828282824438070E0E090100102844B6
:103B60000082828282828282824438070D0D09019E
:103B70000028280082828282828282824438070E54
:103B80000E09010008102000828244281010101035
:103B90001010070A0A0901008080FC828282FC80E2
:103BA0008080060A0A09010038444448D048444449
:103BB0004458070B0B090100201008007C02027E0C
:103BC00082867A070B0B090100081020007C020294
:103BD0007E82867A070B0B090100102844007C02C4
:103BE000027E82867A070A0A0901003458007C02A4
:103BF000027E82867A070A0A0901002828007C02D0
:103C0000027E82867A070C0C090100102828100019
:103C10007C02027E82867A0707070901006C121275
:103C20007E90926C070A0A0901FD7C828080808266
:103C30007C104830070B0B090100201008007C8223
:103C400082FE80827C070B0B090100081020007C9B
:103C50008282FE80827C070B0B0901001028440041
:103C60007C8282FE80827C070A0A090100282800E3
:103C70007C8282FE80827C050C0C09020080402040
:103C80000000E02020202020F8050C0C0902001084
:103C900020400000E02020202020F8050C0C090224
:103CA000002050880000E02020202020F8050B0B89
:103CB00009020050500000E02020202020F8070BCF
:103CC0000B090100483050083C4482828244380786
:103CD0000A0A090100345800BCC28282828282072B
:103CE0000B0B090100201008007C82828282827CFA
:103CF000070B0B090100081020007C82828282825F
:103D00007C070B0B090100102844007C8282828210
:103D1000827C070A0A0901003458007C8282828270
:103D2000827C070A0A0901002828007C828282829C
:103D3000827C07090909010010381000FE001038C4
:103D4000100709090901FF027C8A8A92A2A27C80DD
:103D5000070B0B09010040201000828282828286BC
:103D60007A070B0B090100081020008282828282F0
:103D7000867A070B0B090100102844008282828298
:103D800082867A070A0A0901002828008282828234
:103D900082867A070E0E0901FD04081000424224B3
:103DA00024241818109060070B0B0901FE8080B8BE
:103DB000C4828282C4B88080070D0D0901FD2424CD
:103DC000004242242424181810906000002100248E
:103DD0000027002A0000002200250028002B0000F8
:103DE0000020002300260029000202020202020233
:103DF000020404040404040404030303030303038C
:103E00000301010101010101010102040810204028
:103E100080010204081020408001020408102040A4
:103E20008080402010080402010000000102000010
:103E3000000000000004030706000000000000006E
:103E400000000000000000000002494E46494E49B3
:103E500054594E414ECDCCCC3D0AD7233C17B7D157
:103E60003877CC2B329595E6241FB14F0A000020FD
:103E7000410000C84200401C4620BCBE4CCA1B0E7C
:103E80005AAEC59D7400407A10F35A00A0724E18C5
:103E9000090010A5D4E80000E87648170000E40BFC
:103EA00054020000CA9A3B000000E1F505000080C2
:103EB000969800000040420F000000A0860100001C
:103EC00000102700000000E803000000006400006C
:103ED0000000000A00000000000100000000002CAB
:103EE00076D888DC674F0823DFC1DFAE59E1B1B770
:103EF00096E5E3E453C63AE651997696E8E6C2843D
:103F000026EB898C9B62ED407C6FFCEFBC9C9F4054
:103F1000F2BAA56FA5F490055A2AF75C936B6CF979
:103F2000676DC11BFCE0E40D47FEF520E6B500D04F
:103F3000ED902E0300943577050080841E08000064
:103F4000204E0A000000C80C333333330F986E1232
:103F5000831141EF8D2114893BE65516CFFEE6DB38
:103F600018D1844B381BF77C1D901DA4BBE4242082
:103F70003284725E228100C9F124ECA1E53D270064
:103F8000843C673F7BBF8EC6603F11241FBECFEFCE
:103F9000D0E4DEBFCDBF14E0A0E0B1E0E4ECF4EB90
:103FA00001E00BBF02C007900D92A838B107D9F706
:103FB0001BBE1BE1A8E8B4E001C01D92A531B1070A
:103FC000E1F71FE3C8E8DFE304C02297FE010E9487
:103FD00007DAC038D107C9F70E9411D10C9455DA1D
:103FE0000C940000EF92FF920F931F93F22FF02E8C
:103FF00047FD02C0E4E001C0E4E1242F332727FDA0
:10400000309537FF03C0309521953F4F4F2D512FED
:104010000F2FEE2E0E9495258F2D912F1F910F911E
:10402000FF90EF900895A0E0B0E0E9E1F0E20C9499
:1040300026DAEC01A880B980CA80DB80A114B10423
:10404000C104D10441F484E2A82E89EDB82E8BE599
:10405000C82E87E0D82EC601B5012DE133EF41E02F
:1040600050E00E94EAD927EA31E440E050E00E94A3
:1040700082D97B018C01C601B5012DE133EF41E00E
:1040800050E00E94EAD9CA01B9012CEE34EF4FEF9B
:104090005FEF0E9482D96E0D7F1D801F911F97FFD9
:1040A00004C06150704080409048688379838A835F
:1040B0009B839B01AC015F77B901CA01CDB7DEB725
:1040C000EAE00C9442DA0E94132008958EE593E012
:1040D0000E941320089560935E0370935F038093A2
:1040E0006003909361030895A0E0B0E0EAE7F0E296
:1040F0000C9424DAEC015B016115710519F0FB01E8
:1041000091838083F9908F2D90E00E940BDA892BA8
:10411000C9F7FDE2FF1621F4F990EE24E39405C0FF
:104120002BE2F21609F4F990EE248E0101501040B2
:10413000C8016AE47EE343E050E00E940323892B38
:1041400001F58E010E5F1F4FC8016DE47EE345E06F
:1041500050E00E940323892B19F48E01095F1F4F41
:10416000A114B10419F0F50111830083E0FC04C02F
:1041700070E090E080E814C070E090E080E86FEFBD
:1041800008C1C80162E57EE343E050E00E940323DA
:10419000892B69F4A114B10429F470E090E080EC5B
:1041A0006FE7F7C02296F501D183C083F6CF88244C
:1041B000992440E050E060E070E0EF2DE053EA30F9
:1041C000A0F5F2E0EF2A8E2D90E09C01287030706F
:1041D000E2FE06C0232B79F50894811C911C2BC0AC
:1041E000232B19F0089481089108DB01CA0112E021
:1041F000880F991FAA1FBB1F1A95D1F7480F591F87
:104200006A1F7B1F440F551F661F771F4E0F511DDE
:10421000611D711D483929E9520729E9620729E121
:10422000720748F084E0E82A06C0EE3F31F4E3FC70
:1042300039C098E0E92AF990C0CFE53311F0E531B3
:1042400089F529912D3219F4E0E1EE2A05C02B32CF
:1042500019F081E090E003C0299182E090E0E22F24
:10426000E053EA3018F0C81BD90B1CC020E030E046
:10427000FCE020383F075CF4C901880F991F880FC4
:10428000991F280F391F220F331F2E0F311DE9915F
:10429000E053EA3068F3E4FE03C0309521953F4FC8
:1042A000820E931ECE2CDD24E1FE07C0A114B104C2
:1042B00021F02197F501D183C083CB01BA010E947F
:1042C00070D67B018C01F3E0CF22DD2423E0C216FF
:1042D000D10421F417FB109517F9109557016801C7
:1042E000C801B70120E030E040E050E00E94D0D5A6
:1042F000882309F44AC097FE0DC029E6E22E2EE37A
:10430000F22E9094819491089394C0E2D0E000E062
:1043100010E012C091E8E92E9EE3F92EF6CFF701E6
:104320002591359145915491C601B5010E94B0D8AF
:104330005B016C018C1A9D0A8C169D0684F7D5953D
:10434000C7950F5F1F4F0630110529F08CEF9FEFC7
:10435000E80EF91EF1CFC501D6017C018D018C2D2F
:10436000880F8D2D881F8F3F51F0C601B50120E0C9
:1043700030E040E050E00E94D0D5882331F482E262
:1043800090E09093141B8093131B7E2D9F2D802F04
:10439000612F272F392F482F562FB901CA01CDB7CA
:1043A000DEB7ECE00C9440DA2F923F925F926F926E
:1043B0007F928F929F92AF92BF92CF92DF92EF92B5
:1043C000FF920F931F93CF93DF938C011B01EA01A0
:1043D0006115710519F0FB0191838083209749F0E5
:1043E000CE010297839728F020E030E040E050E0D3
:1043F000F6C0F801A1908F018A2D90E00E940BDA9F
:10440000892BB9F7FDE2AF1631F4F801A1908F01C5
:104410005524539407C0FBE2AF1619F4F801A1909C
:104420008F015524209719F0C031D105C1F4F0E374
:10443000AF1679F4F8018081883711F0883549F496
:10444000F801A1800E5F1F4FF2E05F2AC0E1D0E0CB
:1044500006C0209721F480E3A816E9F427C0C830ED
:10446000D10531F1C930D10524F4C230D10531F57F
:104470000CC0CA30D10589F0C031D105F9F4C12C86
:10448000D12CE12CB8E0FB2E28C0C12CD12CE12C82
:10449000A0E4FA2E22C0CAE0D0E0FCECCF2EFCEC67
:1044A000DF2EFCECEF2EFCE0FF2E17C0C8E0D0E0C2
:1044B000C12CD12CE12CE0E1FE2E0FC09E0144273F
:1044C00037FD4095542F60E070E080E090E80E9456
:1044D000C8D9C901DA016C017D0120E030E040E07B
:1044E00050E060E03E01882477FC8094982C70EDC9
:1044F000B72EBA0CE9E0EB1570F48A2D81548A319D
:1045000018F499ECB92E06C08A2D81568A3150F5DF
:1045100089EAB82EBA0C8B2D90E08C179D0714F504
:104520006F3FE1F0C216D306E406F506B0F0CA010B
:10453000B901A40193010E9482D99B01AC012B0D0A
:10454000311D411D511D2130F0E03F07F0E04F07C4
:10455000F0E85F0710F461E001C06FEFF801A1908F
:104560008F01C5CF2114310481F0662331F0015051
:104570001040F1011183008308C051FE1AC002509F
:104580001040F1011183008314C067FF12C050FC7A
:1045900005C02FEF3FEF4FEF5FE704C020E030E0B2
:1045A00040E050E882E290E09093141B8093131B4C
:1045B00016C050FE08C050954095309521953F4F4C
:1045C0004F4F5F4F0CC057FF0AC082E290E09093BC
:1045D000141B8093131B2FEF3FEF4FEF5FE7B901E1
:1045E000CA01DF91CF911F910F91FF90EF90DF9063
:1045F000CF90BF90AF909F908F907F906F905F9083
:104600003F902F900895FB01DC014150504088F00D
:104610008D9181341CF08B350CF4805E6591613492
:104620001CF06B350CF4605E861B611171F3990B05
:104630000895881BFCCFFB01DC014150504048F03D
:1046400005900D920020C9F701C01D9241505040C5
:10465000E0F70895FB0155915523A9F0BF01DC0156
:104660004D9145174111E1F759F4CD010590002016
:1046700049F04D9140154111C9F3FB014111EFCFB4
:1046800081E090E001970895FB01DC0104C08D9169
:104690000190801921F441505040C8F7881B990BB4
:1046A0000895FB01DC0102C001900D924150504081
:1046B000D8F70895FB01DC010D900020E9F7119770
:1046C00001900D920020E1F70895FC018191861779
:1046D00021F08823D9F7992708953197CF010895BC
:1046E000FB01DC0101900D920020E1F70895FB0130
:1046F000DC014150504030F08D910190801919F447
:104700000020B9F7881B990B0895FB01DC0141508B
:10471000504048F001900D920020C9F701C01D9251
:1047200041505040E0F70895AEE0B0E0EAE9F3E22E
:104730000C942CDA0D891E898EE08C831A830983F0
:104740008FEF9FE79E838D839E01275E3F4FCE01B3
:1047500001966F89788DA9010E94B8232F81388531
:10476000020F131FF80110822E96E4E00C9448DA31
:10477000ABE0B0E0EEEBF3E20C941EDA3C012B016F
:104780005A01FC0117821682838181FD03C06FEFFD
:104790007FEFC6C19AE0892E1E010894211C311CAE
:1047A000F3012381F20123FD859123FF81912F01E4
:1047B000882309F4B2C1853239F423FD859123FFA2
:1047C00081912F01853229F490E0B3010E94E52701
:1047D000E7CF982FFF24EE249924FFE1FF15D0F0B6
:1047E0009B3269F09C3228F4903259F0933291F464
:1047F0000EC09D3249F0903369F441E024C052E08C
:10480000F52A84E0F82A28C098E0F92A25C0E0E1DA
:10481000FE2A22C0F7FC29C0892F80538A3070F409
:10482000F6FE05C0989C902C1124980E15C0E89CAB
:10483000E02C1124E80EF0E2FF2A0EC09E3229F48B
:10484000F6FC6BC140E4F42A07C09C3619F450E82A
:10485000F52A02C0983649F4F20123FD959123FF11
:1048600091912F01992309F0B8CF892F8554833076
:1048700018F08052833038F444E050E0A40EB51EA6
:104880005FE359830FC0933631F0933779F0933556
:1048900009F056C020C0F5018081898342E050E0D4
:1048A000A40EB51E610101E010E012C0F501C08048
:1048B000D180F6FC03C06FEF7FEF02C0692D70E07E
:1048C00042E050E0A40EB51EC6010E94DA278C011A
:1048D0005FE7F52214C0F501C080D180F6FC03C06B
:1048E0006FEF7FEF02C0692D70E042E050E0A40E50
:1048F000B51EC6010E94CF278C0150E8F52AF3FEB1
:1049000007C01AC080E290E0B3010E94E527EA9454
:104910008E2D90E008171907A8F30EC0F601F7FCDA
:104920008591F7FE81916F0190E0B3010E94E52728
:10493000E110EA94015010400115110579F7EAC021
:10494000943611F0993669F5F7FE08C0F50120811B
:1049500031814281538184E090E00AC0F501808179
:1049600091819C01442737FD4095542F82E090E0CF
:10497000A80EB91E9FE6F92257FF09C05095409531
:10498000309521953F4F4F4F5F4FE0E8FE2ACA0117
:10499000B901A1012AE030E00E941128D82ED218D6
:1049A00040C0953729F41F2D1F7E2AE030E01DC03E
:1049B0001F2D197F9F3661F0903720F4983509F04C
:1049C000ACC00FC0903739F0983709F0A6C004C0CA
:1049D00028E030E00AC0106114FD146020E130E0EE
:1049E00004C014FD166020E132E017FF08C0F50195
:1049F000608171818281938144E050E008C0F501BB
:104A000080819181BC0180E090E042E050E0A40E02
:104A1000B51EA1010E941128D82ED2188FE7F82EBA
:104A2000F122F6FE0BC05EEFF522D91438F4F4FE45
:104A300007C0F2FC05C08FEEF82202C01D2D01C098
:104A4000192DF4FE0DC0FE01ED0DF11D80818033A6
:104A500019F499EEF92208C01F5FF2FE05C003C0E9
:104A60008F2D867809F01F5F0F2DF3FC14C0F0FE28
:104A70000FC01E1510F09D2C0BC09D2C9E0C911A82
:104A80001E2D06C080E290E0B3010E94E5271F5F63
:104A90001E15C0F304C01E1510F4E11A01C0EE2467
:104AA00004FF0FC080E390E0B3010E94E52702FFFE
:104AB0001DC001FD03C088E790E00EC088E590E0CE
:104AC0000BC0802F867891F001FF02C08BE201C0FD
:104AD00080E2F7FC8DE290E0B3010E94E52706C07A
:104AE00080E390E0B3010E94E5279A94D914C0F3C3
:104AF000DA94F101ED0DF11D808190E0B3010E9487
:104B0000E527DD20A9F706C080E290E0B3010E940E
:104B1000E527EA94EE20C1F743CEF3016681778161
:104B2000CB012B96E2E10C943ADAA9E0B0E0EBE994
:104B3000F5E20C9422DA6A01122FA02EBE2C2BE390
:104B4000201718F42CE3922E02C0902E9394AE01FD
:104B50004F5F5F4F27E0092D0E94F726BC01898136
:104B6000E82EFF24C70189709070019711F4ADE21F
:104B700009C0B1FE02C0ABE205C0B0FC02C0A0E0BB
:104B800001C0A0E2E3FE3BC0AA2311F423E001C070
:104B900024E0211710F020E002C0121B212FEB2C83
:104BA000B4FE02C0322F0AC0F601322F80E202C0EA
:104BB000819331503323E1F7C20ED11CAA2319F09F
:104BC000F601A1936F01F6013196E2FE05C09EE465
:104BD000D6019C9381E404C09EE6D6019C9381E6B5
:104BE00011968C9391833296DF01832F90E202C05D
:104BF0009D9381508823E1F7E30FF11D40C0E2FE51
:104C000042C0AA2311F423E001C024E0211710F0D0
:104C100020E002C0121B212FEB2CB4FE02C0922F09
:104C20000AC0F601922F80E202C08193915099232D
:104C3000E1F7C20ED11CAA2319F0F601A1936F016E
:104C4000F6013196E2FE08C089E4D6018C938EE429
:104C500011968C9386E407C089E6D6018C938EE684
:104C600011968C9386E681833296DF01892F20E2AC
:104C700002C02D9381508823E1F7E90FF11D1082C6
:104C80002EEF3FEFAFC0161617061CF041E050E0C4
:104C900003C0AB014F5F5F4FAA2019F480E090E0A2
:104CA00003C08A2D90E0019620E030E0AA2311F0A5
:104CB00021E030E0240F351F280F391F812F90E0AD
:104CC0002817390714F020E002C0121B212F4B2DAA
:104CD00050E0CA0180719070B4FC0DC0B3FC0BC0F1
:104CE000F601322F40E202C0419331503323E1F705
:104CF000C20ED11C01C0322FAA2319F0F601A193D4
:104D00006F01892B11F0132F0AC0F601132F80E3D6
:104D100002C0819311501123E1F7C30ED11C092D5C
:104D2000060FBA8090E1892E912C8E209F20E4FE00
:104D300004C0F1E3BF1609F40150101614F001E0AD
:104D400003C0093008F008E09B0177FF02C020E0B3
:104D500030E0CB010196821B930BFE013196E80FE8
:104D6000F91F8EE2F82E3B01601A71088A2D90E03F
:104D700044275527481B590B8FEF2F3F380719F44D
:104D8000D601FD926D01621773072CF0621673064F
:104D900014F4808101C080E3215030403196241703
:104DA000350724F0D6018D936D01E6CF261737071E
:104DB00049F4B5E3BB1528F0BB1621F48114910426
:104DC00009F481E3F6018193D601812F90E202C0BC
:104DD0009C93815011968823D9F7E10FF11D108221
:104DE00020E030E0C9012996EEE00C943EDA28304C
:104DF00008F027E03327DA01990F311D87FD916014
:104E000000966105710539F432602E5F3D9330E301
:104E10002A95E1F708959F3F30F0803871056105CC
:104E200009F03C5F3C5F3D93913008F08068911D34
:104E3000DF93CF931F930F93FF92EF92192F987FD9
:104E40009695E92F96959695E90FFF27E152F14C3B
:104E500099273327EE24FF24A701E7010590089442
:104E6000079428F4360FE71EF81E491F511D660FE0
:104E7000771F881F991F0694A1F70590079428F4BF
:104E8000E70EF81E491F561FC11D770F881F991F77
:104E9000661F0694A1F70590079428F4F80E491FA1
:104EA000561FC71FD11D880F991F661F771F0694B5
:104EB000A1F70590079420F4490F561FC71FD81F6C
:104EC000990F661F771F881F0694A9F78491109584
:104ED000177041F0D695C79557954795F794E79485
:104EE0001A95C1F7E5E8FEE36894159015913591A0
:104EF0006591959105907FE27395E118F10A430B56
:104F0000560BC90BD009C0F7E10CF11E431F561F09
:104F1000C91FD01D7EF4703311F48A95E6CFE89452
:104F2000015030F0080F0AF40027021708F4202F70
:104F30002395022F7A3328F079E37D932A95E9F7B8
:104F400010C07D932A9589F60694979567953795B5
:104F500017951794E118F10A430B560BC90BD009AA
:104F600098F023957E9173957A3308F070E37C93E3
:104F70002013B8F77E9170617D9330F0839571E3D3
:104F80007D9370E32A95E1F71124EF90FF900F9144
:104F90001F91CF91DF91992787FD90950895FC018E
:104FA0000590615070400110D8F7809590958E0F54
:104FB0009F1F0895FC016150704001900110D8F7C7
:104FC000809590958E0F9F1F08950F931F93CF93F9
:104FD000DF938C01EB018B8181FF1BC082FF0DC031
:104FE0002E813F818C819D812817390764F4E881E7
:104FF000F9810193F983E88306C0E885F985802F5C
:105000000995892B31F48E819F8101969F838E8330
:1050100002C00FEF1FEFC801DF91CF911F910F91D9
:105020000895FA01AA27283051F1203181F1E8943E
:105030006F936E7F6E5F7F4F8F4F9F4FAF4FB1E08B
:105040003ED0B4E03CD0670F781F891F9A1FA11D86
:10505000680F791F8A1F911DA11D6A0F711D811D87
:10506000911DA11D20D009F468943F912AE0269F4C
:1050700011243019305D3193DEF6CF010895462FAB
:105080004770405D4193B3E00FD0C9F7F6CF462F8C
:105090004F70405D4A3318F0495D31FD40524193F5
:1050A00002D0A9F7EACFB4E0A695979587957795B2
:1050B0006795BA95C9F700976105710508959B0139
:1050C000AC010A2E06945795479537952795BA95C2
:1050D000C9F7620F731F841F951FA01D0895FC015F
:1050E000128213820895FC018381882311F081E0EC
:1050F00082830895FC018281811112820895CF93E9
:10510000DF93DC01FC01EB55FE4F8081918100971C
:10511000C9F1019791838083ED01CC5ADF4FFD01E6
:10512000ED58FF4F8BE1019009928150E1F7FD01AD
:10513000EE5AFF4FAF58BF4F8D919C911197A157D9
:10514000B04091838083FD01ED58FF4F20E030E0B7
:10515000AD014B555E4F10C02F5F3F4FEF01DF0198
:105160005F968BE10D9009928150E1F7858D968DC8
:10517000329791838083B196DA018D919C912817A3
:10518000390750F3DF91CF910895FC0181E694E057
:10519000918380838781882321F0CF0104960E9428
:1051A000CF80089583519E4F0E94CF800895CF9263
:1051B000DF92EF92FF920F931F93DF93CF93CDB7C0
:1051C000DEB76F970FB6F894DEBF0FBECDBF8C0170
:1051D0006B01095A1F4FD8018C9107551040882345
:1051E00021F42FE2E22EF12C03C090E5E92EF12C00
:1051F000E00EF11E81E694E09A8389831C821B8273
:1052000018861D82B7016C5F7F4FCE010596A601FF
:1052100021E00E94DD87882391F5E3EEF0E0949190
:1052200008C08091C00085FFFCCF9093C6003196E6
:1052300094919923B1F7E9EEF0E0949108C0809140
:10524000C00085FFFCCF9093C600319694919923BE
:10525000B1F709C08091C00085FFFCCF0894C11C44
:10526000D11C9093C600F6019081992399F7809103
:10527000C00085FFFCCF8AE08093C6005AC0F801C9
:10528000EB55FE4F208131812A30310508F040C0B6
:105290002F5F3F4F3183208321503040F90185E05B
:1052A000EE0FFF1F8A95E1F7E21BF30BED58FF4F5E
:1052B000E00FF11F13C0AF01415E5F4FBF018BE1F3
:1052C000DB010D90BD01DA010D92AD018150C1F7F6
:1052D000929182913296968F858F7F9721503040A0
:1052E000BFEF2E3F3B0739F7D801AD58BF4FF7014D
:1052F00034968BE101900D928150E1F70F581F4FCA
:10530000F70182819381D8018D939C9301571040BE
:10531000D801AC5ABF4FFE0135968BE101900D923A
:105320008150E1F70E5A1F4F8B819C81F8019183C8
:105330008083CE0101960E94C5286F960FB6F8941F
:10534000DEBF0FBECDBFCF91DF911F910F91FF90B8
:10535000EF90DF90CF9008959C01AB0183519E4F59
:105360002D5C3F4FB90121E00E94DD8708950F9326
:105370001F93FC01162F072F242F8381882309F404
:1053800063C0E051FE4F8081E05FF140882309F067
:105390005BC0CF0183519E4FF396BF01412F502F29
:1053A0000E94DD87882361F5E8EDF2E0949108C062
:1053B0008091C00085FFFCCF9093C60031969491F8
:1053C0009923B1F7812F902F9C01F90107C080919B
:1053D000C00085FFFCCF31969093C6009081992341
:1053E000B1F7E5EDF2E0949108C08091C00085FF2F
:1053F000FCCF9093C600319694919923B1F724C0C5
:10540000E3ECF2E0949108C08091C00085FFFCCFEE
:105410009093C600319694919923B1F7812F902FE4
:105420009C01F90107C08091C00085FFFCCF319637
:105430009093C60090819923B1F78091C00085FFB9
:10544000FCCF8AE08093C6001F910F910895EF92E0
:10545000FF920F931F938C013EECE32E31E0F32E6D
:10546000E80EF91EC7010E948180C7010E94CF800B
:10547000F801108211821F910F91FF90EF90089513
:10548000CF92DF92EF92FF920F931F93CF93DF9310
:105490007C016B01DB010D900020E9F78D010150CB
:1054A0001040061B170BEEECF1E0EE0EFF1ED701CD
:1054B0001C92E2E3FEEFEE0EFF1ECB016EE470E005
:1054C0000E946523EC01009731F4F8013197EC0D4F
:1054D000FD1D86010EC060E270E00E9465238C0114
:1054E0000F5F1F4FCE016AE270E00E946523FC014E
:1054F00031978DE081838AE082831382C7018653CE
:105500009E4FB8010E94DF888EEC91E0E80EF91EF4
:10551000D7018C91882319F1E3E1F1E0949108C05F
:105520008091C00085FFFCCF9093C6003196949186
:105530009923B1F7EAE1F1E0949108C08091C000AD
:1055400085FFFCCF9093C600319694919923B1F7D3
:105550008091C00085FFFCCF8AE08093C600DF9178
:10556000CF911F910F91FF90EF90DF90CF90089512
:10557000CF93DF93EC018B81882309F43BC0E2E4F5
:10558000F1E0949108C08091C00085FFFCCF90931A
:10559000C600319694919923B1F7CE55DD4F4881DD
:1055A00059816A817B81C25AD2408CE095E02AE021
:1055B00030E00E941F3DE0E4F1E0949108C080914A
:1055C000C00085FFFCCF9093C6003196949199233B
:1055D000B1F7C656DD4F488159816A817B818CE0E5
:1055E00095E02AE030E00E941F3D8091C00085FFD9
:1055F000FCCF12C0E0E3F1E0949108C08091C000BC
:1056000085FFFCCF9093C600319694919923B1F712
:105610008091C00085FFFCCF8AE08093C600DF91B7
:10562000CF9108952F923F924F925F926F927F9207
:105630008F929F92AF92BF92CF92DF92EF92FF92A2
:105640000F931F93DF93CF93CDB7DEB7AC970FB611
:10565000F894DEBF0FBECDBF5C014B01FC0183811E
:10566000882309F438C1C50182539E4F0E94CF8020
:10567000F50112821A8A1D8A198A188A81E694E035
:105680009F878E875EE4C52ED12CCA0CDB1C2FE2CF
:1056900030E0A20EB31EF601B182A08221ED3FEFF1
:1056A000A20EB31EF40180818F3209F090C0C401B4
:1056B0006FE270E00E9465237C010894E11CF11CFC
:1056C0003E010894611C711C260142E1242E312CFC
:1056D0002C0E3D1E77C0C7016FE270E00E9465236B
:1056E0006C01009709F481C0E816F90608F07DC046
:1056F0008C010E191F09C301B701A8010E9485235F
:10570000060D171DF8011082F30107C08091C0003B
:1057100085FFFCCF31969093C60090819923B1F715
:105720008091C00085FFFCCFFAE0F093C600F20143
:10573000608171816115710519F460E070E002C04B
:105740006C5F7F4FC101A30121E00E94DD878823A8
:1057500071F5EEE7F1E0949108C08091C00085FFFB
:10576000FCCF9093C600319694919923B1F7FE0136
:10577000319607C08091C00085FFFCCF3196909391
:10578000C60090819923B1F7ECE7F1E0949108C04D
:105790008091C00085FFFCCF9093C6003196949114
:1057A0009923B1F78091C00085FFFCCF8DC02EE01A
:1057B00030E02C0F3D1FF2013183208376010894E5
:1057C000E11CF11CE114F10409F085CF0BC080E568
:1057D00090E0A80EB91EF601B182A08220EB3FEF47
:1057E000A20EB31ED82C092D02C0DE2C0F2D8EE484
:1057F00090E0A80EB91EF5018081918122EB3FEF68
:10580000A20EB31E009719F480E090E001C0049648
:105810006D2D702F0E94AF88882339F1EEE6F1E0FC
:10582000949108C08091C00085FFFCCF9093C60082
:10583000319694919923B1F78D2D902F9C01F90108
:1058400007C08091C00085FFFCCF31969093C600C1
:1058500090819923B1F782EA92E0A80EB91EF50172
:10586000108211821282138232C0E6E5F1E0949137
:1058700008C08091C00085FFFCCF9093C600319690
:1058800094919923B1F78D2D902F9C01F90107C0B8
:105890008091C00085FFFCCF31969093C600908127
:1058A0009923B1F7E4E5F1E0949108C08091C0003C
:1058B00085FFFCCF9093C600319694919923B1F760
:1058C0008091C00085FFFCCF8AE08093C600CE01A6
:1058D0000E960E94C528AC960FB6F894DEBF0FBE98
:1058E000CDBFCF91DF911F910F91FF90EF90DF908F
:1058F000CF90BF90AF909F908F907F906F905F9070
:105900004F903F902F900895C3966BE37AE00E94EA
:10591000AF88882379F0E1EBF2E0949108C08091A0
:10592000C00085FFFCCF9093C600319694919923D7
:10593000B1F70EC0ECE9F2E0949108C08091C0008C
:1059400085FFFCCF9093C600319694919923B1F7CF
:10595000E9E9F2E0949108C08091C00085FFFCCF96
:105960009093C600319694919923B1F70895BF9210
:10597000CF92DF92EF92FF920F931F93CF93DF931B
:105980008C01EB018FE28993FF24EE24E39475EA06
:10599000C72E71E0D72EC00ED11E6FE1B62E14C0F7
:1059A000FB9CC00111248D589F4F800F911FBE0199
:1059B0000E94E18002C02196E3948881882319F037
:1059C0008CE88E15C0F7F3942F2D30E0F60180811E
:1059D00091812817390720F3E7FC07C0C8018253DB
:1059E0009E4FBE010E94E18001C01882DF91CF91DD
:1059F0001F910F91FF90EF90DF90CF90BF9008958F
:105A00002F923F924F925F926F927F928F929F92CE
:105A1000AF92BF92CF92DF92EF92FF920F931F93BC
:105A2000DF93CF93CDB7DEB7AD970FB6F894DEBF57
:105A30000FBECDBF6C014B014DA7DC0113968C91BD
:105A4000882309F44AC3E1EDF1E0CE0EDF1ED60152
:105A50008C91EFE2FEEFCE0EDF1E882309F419C110
:105A6000222309F0E1C028E032E0C20ED31ED601A5
:105A70008C91E8EFFDEFCE0EDF1E882371F1E3E19C
:105A8000F1E0949108C08091C00085FFFCCF909315
:105A9000C600319694919923B1F7E6E5F2E094912E
:105AA00008C08091C00085FFFCCF9093C60031965E
:105AB00094919923B1F78CE095E061E070E04AE0C1
:105AC00050E00E94843D8091C00085FFFCCF8AE0B9
:105AD0008093C6000E94B03F00C3E3EEF0E09491D3
:105AE00008C08091C00085FFFCCF9093C60031961E
:105AF00094919923B1F7EDE3F2E0949108C080917D
:105B0000C00085FFFCCF9093C600319694919923F5
:105B1000B1F7F40107C08091C00085FFFCCF31963A
:105B20009093C60090819923B1F7E2E3F2E094915B
:105B300008C08091C00085FFFCCF9093C6003196CD
:105B400094919923B1F7C6012DE032E0C20ED31E25
:105B5000B6010E94B72C4BEF5FEFC40ED51ED601E5
:105B60009C91E8EFFDEFCE0EDF1E8DE8989FF001CF
:105B70001124E35FFD4FEC0DFD1D07C08091C000B7
:105B800085FFFCCF31969093C60090819923B1F7A1
:105B9000ECE2F2E0949108C08091C00085FFFCCF58
:105BA0009093C600319694919923B1F722EA32E09E
:105BB000C20ED31ED6014D915D916D917C91EEE5A3
:105BC000FDEFCE0EDF1E8CE095E02AE030E00E9473
:105BD0001F3D8091C00085FFFCCF8AE08093C60006
:105BE000A601485F5D4FDA012C91E22FF0E0EE0F45
:105BF000FF1FEE0FFF1FEC0DFD1DE75FFD4F82EA5B
:105C000092E0C80ED91ED6014D905D906D907C90AB
:105C10008EE59DEFC80ED91E40825182628273824A
:105C20002F5FDA012C932FC0E3EEF0E0949108C0CF
:105C30008091C00085FFFCCF9093C600319694916F
:105C40009923B1F7EBE1F2E0949108C08091C00094
:105C500085FFFCCF9093C600319694919923B1F7BC
:105C6000F40107C08091C00085FFFCCF319690936E
:105C7000C60090819923B1F78091C00085FFFCCFC9
:105C80008AE08093C600C60182539E4F0E94CF8057
:105C900039C0E8E0F2E0CE0EDF1ED6011C92E8EF3C
:105CA000FDEFCE0EDF1EE3EEF0E0949108C0809190
:105CB000C00085FFFCCF9093C60031969491992344
:105CC000B1F7EAE0F2E0949108C08091C00085FF4E
:105CD000FCCF9093C600319694919923B1F7F401CB
:105CE00007C08091C00085FFFCCF31969093C6001D
:105CF00090819923B1F78091C00085FFFCCF8AE0A5
:105D00008093C600D60112961C921A8A1D8A198A9F
:105D1000188A81E694E09F878E87FEE4AF2EB12C2F
:105D2000AC0CBD1CEFE2F0E0CE0EDF1ED501CD9233
:105D3000DC92E1EDFFEFCE0EDF1ED4018C918F32AD
:105D400009F090C0C4016FE270E00E9465237C01FD
:105D50000894E11CF11C3E010894611C711C250192
:105D6000E2E12E2E312C2C0E3D1E77C0C7016FE2D2
:105D700070E00E9465235C01009709F481C0E81679
:105D8000F90608F07DC08C010E191F09C301B70187
:105D9000A8010E948523060D171DF8011082F3014A
:105DA00007C08091C00085FFFCCF31969093C6005C
:105DB00090819923B1F78091C00085FFFCCFFAE074
:105DC000F093C600D2016D917C916115710519F4B3
:105DD00060E070E002C06C5F7F4FC101A30121E071
:105DE0000E94DD87882371F5E6EFF1E0949108C009
:105DF0008091C00085FFFCCF9093C60031969491AE
:105E00009923B1F7FE01319607C08091C00085FF4C
:105E1000FCCF31969093C60090819923B1F7E4EFBF
:105E2000F1E0949108C08091C00085FFFCCF909371
:105E3000C600319694919923B1F78091C00085FFF7
:105E4000FCCF1BC12EE030E02C0F3D1FF20131834F
:105E5000208375010894E11CF11CE114F10409F0A0
:105E600085CF0BC040E550E0C40ED51ED501CD92C4
:105E7000DC92E0EBFFEFCE0EDF1E082DF92C01C007
:105E80000E2DF601E25BFF4F2DA5222309F4B1C0D0
:105E9000608171816115710519F460E070E002C0E4
:105EA0006C5F7F4FC60182539E4F402F5F2D21E0D4
:105EB0000E94DD87882309F46CC04FED51E0C40EC9
:105EC000D51ED6014D915D916D917C91EBEBF0E08B
:105ED000CE0EDF1ED6014D935D936D937C93139789
:105EE000E6E6FDEFCE0EDF1EE6EEF1E0949108C08F
:105EF0008091C00085FFFCCF9093C60031969491AD
:105F00009923B1F7802F9F2D9C01F90107C0809143
:105F1000C00085FFFCCF31969093C60090819923F5
:105F2000B1F7EEEDF1E0949108C08091C00085FFDB
:105F3000FCCF9093C600319694919923B1F78CE0F1
:105F400095E02AE030E00E941F3D8091C00085FF6F
:105F5000FCCF8AE08093C60022EA32E0C20ED31E54
:105F6000D6011D921D921D921C921397E0EDF1E057
:105F7000949108C08091C00085FFFCCF9093C6002B
:105F8000319694919923B1F78091C00085FFFCCFA1
:105F900099C0ECEBF1E0949108C08091C00085FFBE
:105FA000FCCF9093C600319694919923B1F7802F3E
:105FB0009F2D9C01F90107C08091C00085FFFCCF97
:105FC00031969093C60090819923B1F7EAEBF1E006
:105FD000949108C08091C00085FFFCCF9093C600CB
:105FE000319694919923B1F78091C00085FFFCCF41
:105FF00044C0608171816115710519F460E070E041
:1060000002C06C5F7F4FC60182539E4F402F5F2DB1
:1060100026E50E94DD87882309F033C0E6EAF1E037
:10602000949108C08091C00085FFFCCF9093C6007A
:10603000319694919923B1F7802F9F2D9C01F901FE
:1060400007C08091C00085FFFCCF31969093C600B9
:1060500090819923B1F7E4EAF1E0949108C080912E
:10606000C00085FFFCCF9093C60031969491992390
:10607000B1F78091C00085FFFCCF8AE08093C60015
:1060800028C081E0F6018083E2E9F1E0949108C044
:106090008091C00085FFFCCF9093C600319694910B
:1060A0009923B1F7F40107C08091C00085FFFCCFB0
:1060B00031969093C60090819923B1F78091C000EA
:1060C00085FFFCCF8AE08093C600802F9F2D0E9421
:1060D000E3BFCE010E960E94C528AD960FB6F89488
:1060E000DEBF0FBECDBFCF91DF911F910F91FF900B
:1060F000EF90DF90CF90BF90AF909F908F907F9068
:106100006F905F904F903F902F900895FC0181E039
:106110008183CF0140E021E00E94002D089583514A
:106120009E4F0E94E7810895CF92DF92EF92FF92F7
:106130000F931F938C017B016A0183519E4F40E0B6
:1061400050E060E070E00E94B77FC80187519E4F29
:10615000B701A6010E94FD881F910F91FF90EF905B
:10616000DF90CF900895EF92FF920F931F93CF93FC
:10617000DF93EC010E948B908E01085F1D4FD801C8
:106180008C919EECE92E91E0F92EEC0EFD1E8823F9
:10619000A9F1C7010E94CF80F8016081615060833E
:1061A0008DE8689FB0011124635F7D4F6C0F7D1FE8
:1061B000CE0141E021E00E94002DD801EC91F0E0F9
:1061C000EE0FFF1FEE0FFF1FEC0FFD1FE75FFD4FF0
:1061D0004081518162817381CE55DD4F488359835F
:1061E0006A837B83C25AD240C7010E94B77F8B81EA
:1061F000882309F462C081E08A835FC00E946890AE
:10620000C7010E94CF801A82CE016BE37AE04AE593
:106210000E94B7291092FD0710924B0ACE016DEF34
:1062200077E04FE452E00E9494308F5F9F4FA1F4DB
:10623000E0E0F1E007C08091C00085FFFCCF31961F
:106240009093C60090819923B1F78091C00085FF9B
:10625000FCCF8AE08093C60010924D0A10924C0A3F
:10626000CE0183519E4F0E94CF8087ED90E00E9427
:10627000AF478091ED0F882301F11092ED0F8091CF
:10628000EB07C82FD0E0CC0FDD1FCD5AD84E688168
:106290007981882777FD8095982F0E9472D620916A
:1062A000A7033091A8034091A9035091AA030E942B
:1062B000DED7181614F419821882DF91CF911F913E
:1062C0000F91FF90EF900895EF92FF920F931F931D
:1062D000CF93DF938C01FC01138286A9882321F0E0
:1062E000C801C3960E94CF8027EAE22E21E0F22E59
:1062F000E00EF11EC70160E04FE10E94757E882329
:1063000009F5E3EEF0E0949108C08091C00085FFAC
:10631000FCCF9093C600319694919923B1F7EAE1AE
:10632000F3E0949108C08091C00085FFFCCF90936A
:10633000C600319694919923B1F78091C00085FFF2
:10634000FCCF7DC0E801C455DE4FCE01B70141E06E
:106350000E947889882341F5CE01B70140E00E9470
:106360007889882309F5E3E1F1E0949108C08091F0
:10637000C00085FFFCCF9093C6003196949199237D
:10638000B1F7E7E0F3E0949108C08091C00085FF89
:10639000FCCF9093C600319694919923B1F78091E8
:1063A000C00085FFFCCF4BC0C801C396BE010E9450
:1063B000D083882309F5E3E1F1E0949108C080914E
:1063C000C00085FFFCCF9093C6003196949199232D
:1063D000B1F7E7EFF2E0949108C08091C00085FF2B
:1063E000FCCF9093C600319694919923B1F7809198
:1063F000C00085FFFCCF23C081E0F8018383E3EE7A
:10640000F0E0949108C08091C00085FFFCCF90938C
:10641000C600319694919923B1F7ECEEF2E0949195
:1064200008C08091C00085FFFCCF9093C6003196D4
:1064300094919923B1F78091C00085FFFCCF8AE049
:106440008093C600D801AC5ABF4FF801F3968BE198
:1064500001900D928150E1F7F80181A992A90E5A9D
:106460001F4FF8019183808302551040C8018F9619
:10647000025B1F4FF80191838083DF91CF911F91C1
:106480000F91FF90EF9008952F923F924F925F925D
:106490006F927F929F92AF92BF92CF92DF92EF92D4
:1064A000FF920F931F93DF93CF93CDB7DEB7CC55F9
:1064B000D0400FB6F894DEBF0FBECDBF6C0166238F
:1064C00011F526EA32E0C20ED31ED6018C91EAE520
:1064D000FDEFCE0EDF1E882309F4E6C02EE932E080
:1064E000C20ED31ED601ED90FD900D911C91E2E6F7
:1064F000FDEFCE0EDF1E0E9404CFE616F70608075A
:10650000190708F4D1C026EA32E0C20ED31ED60124
:106510001C92EAE5FDEFCE0EDF1ED60113968C919C
:10652000882341F4C6010E946431F60183818823E7
:1065300009F4BAC000D000D000D0EDB7FEB7319654
:106540007E010894E11CF11CADB7BEB71296FC9217
:10655000EE9211978AE091E093838283D6019D9613
:106560008D919C919E97958384830E9494238701AB
:10657000EDB7FEB736960FB6F894FEBF0FBEEDBF6F
:1065800057010AC0D8018C91992787FD90950E94E8
:1065900013DAF80181938F01F50101900020E9F7EA
:1065A0003197EA19FB09802F8E198E175CF363E38C
:1065B000A62EB12CAC0CBD1CC50140E050E060E043
:1065C00070E00E94B77F99245DE3E52EF12CEC0E7C
:1065D000FD1E2E010894411C511C4FE1642E712CAC
:1065E0006C0E7D1E33E0232E31E0332E43C0D801E4
:1065F0008C9190E00E9413DAF80181938F01D7010A
:106600000D900020E9F71197AE19BF09802F8E1960
:106610008A176CF327968FAD27978E3759F1C701EC
:10662000B20145E050E00E947723009719F500D0B1
:1066300000D000D0EDB7FEB73196ADB7BEB7129619
:106640007C926E92119733822282558244820E94FC
:106650009423EDB7FEB736960FB6F894FEBF0FBE83
:10666000EDBFC3010E94DA468FEF90E00E94AF4772
:1066700099249394C501B70140E050E00E94EC8258
:10668000181614F48701BBCF992041F48FEF9FEFC8
:10669000D6019E969C938E939D9706C0F60185A584
:1066A00096A5019696A785A7C45ADF4F0FB6F89412
:1066B000DEBF0FBECDBFCF91DF911F910F91FF9035
:1066C000EF90DF90CF90BF90AF909F907F906F90B2
:1066D0005F904F903F902F9008952F923F924F924E
:1066E0005F926F927F928F929F92AF92BF92CF9262
:1066F000DF92EF92FF920F931F93DF93CF93CDB76B
:10670000DEB7CF58D0400FB6F894DEBF0FBECDBF76
:106710008C013B016A0184E090E0C80ED91EF801AB
:106720007196C757DF4FF983E883C958D040C80135
:106730000496CA57DF4F99838883C658D040C857FC
:10674000DF4F1882C858D040B6E6EB2EF12CEC0E85
:10675000FD1EF7013B96C557DF4FF983E883CB5801
:10676000D040A7EA8A2EA2E09A2E800E911EF9EA66
:10677000AF2EF2E0BF2EA00EB11EEEE02E2E312C79
:106780002C0E3D1E77E4472E512C4C0E5D1EC2018F
:106790000496C357DF4F99838883CD58D040E3EEEA
:1067A000F0E09491C157DF4F9883CF58D0404FC14C
:1067B000F7018385482F50E0BA016871707060312D
:1067C000710509F052C1F401208131812130310578
:1067D00009F44BC12230310509F447C1F701DE014C
:1067E00011969081903239F08E2F8E19883011F4E5
:1067F0008EE28D939D933196C557DF4F88819981A5
:10680000CB58D040E817F90761F71C921E86F301B8
:106810008081882329F4C10165E271E00E945A2336
:10682000C101B3010E945A23C101BE016F5F7F4FB6
:106830000E945A23C10165E271E00E945A231CA6FE
:106840001FA61BA61AA681E694E099A788A7CE01E9
:106850008C96B601AE014F5F5F4F21E00E94DD874D
:10686000882309F03FC0F40180819181892BD1F503
:10687000C157DF4F9881CF58D040E3EEF0E008C019
:106880008091C00085FFFCCF9093C6003196949113
:106890009923B1F7E7E2F1E007C08091C00085FFDE
:1068A000FCCF31969093C60090819923B1F78091E7
:1068B000C00085FFFCCFFAE0F093C600FE013196E0
:1068C00007C08091C00085FFFCCF31969093C60031
:1068D00090819923B1F78091C00085FFFCCF8AE0B9
:1068E0008093C600C357DF4FA881B981CD58D040EF
:1068F000FE01BC968BE101900D928150E1F78AA5D3
:106900009BA5F2019383828381E694E09183808347
:10691000C801B101A2010E946D33C2010E94C528C5
:10692000CE0188960E94C52892C0953E09F48FC07A
:106930009E3209F48CC09F3509F489C0F801918911
:10694000992331F09E3209F482C09F3509F47FC04B
:1069500043FD7DC080E06031710509F481E0F801FC
:1069600084A7882349F4F7018085873409F06FC034
:1069700081858E3709F46BC0CA57DF4FA881B98172
:10698000C658D040F7018081803241F08E2F8E1999
:10699000883011F48EE28D9380818D933196C557A6
:1069A000DF4F88819981CB58D040E817F90759F714
:1069B0001C92F40180819181009729F5F30107C0B1
:1069C0008091C00085FFFCCF31969093C6009081E6
:1069D0009923B1F7CA57DF4FE881F981C658D040F3
:1069E00007C08091C00085FFFCCF31969093C60010
:1069F00090819923B1F78091C00085FFFCCFFAE028
:106A0000F093C60024C08130910539F4F5018081EE
:106A100091810196918380831AC00297C1F4C8576F
:106A2000DF4FF881C858D0402F2F30E0F50180812A
:106A3000918128173907F1F0C857DF4FF881C858FE
:106A4000D040FF5FC857DF4FF883C858D040C60119
:106A5000B701C757DF4F48815981C958D0400E94BC
:106A6000EC8218160CF4A4CE05C0F701908199238E
:106A700009F05BCFC157DF4F0FB6F894DEBF0FBEF2
:106A8000CDBFCF91DF911F910F91FF90EF90DF90DD
:106A9000CF90BF90AF909F908F907F906F905F90BE
:106AA0004F903F902F900895EF92FF920F931F9376
:106AB000DF93CF93CDB7DEB76F970FB6F894DEBFF5
:106AC0000FBECDBF7C018C01025B1F4F805B9F4FCF
:106AD000F8019183808327EA32E0E20EF31E21E081
:106AE00030E0F701219331937F011182108227E575
:106AF0003DEFE20EF31E049640E050E060E070E0EF
:106B00000E94B77FF80120813181DE011596F901DD
:106B100034968BE101900D928150E1F7F901828169
:106B200093819C838B8381E694E09A838983C70158
:106B30006AE371E08E010F5F1F4FA8010E946D3361
:106B4000C8010E94C528F701E755FD4F808191815A
:106B50006F960FB6F894DEBF0FBECDBFCF91DF9119
:106B60001F910F91FF90EF900895EF92FF920F9376
:106B70001F93DF93CF93CDB7DEB76F970FB6F8941F
:106B8000DEBF0FBECDBF7C018C01025B1F4F805B5F
:106B90009F4FF8019183808327EA32E0E20EF31ED3
:106BA00022E030E0F7013183208329E53DEFE20E5A
:106BB000F31EF701E755FD4F60831182049640E014
:106BC00050E060E070E00E94B77FF80120813181E1
:106BD000DE011596F90134968BE101900D928150FA
:106BE000E1F7F901828193819C838B8381E694E0B4
:106BF0009A838983C7016AE371E08E010F5F1F4F9B
:106C0000A8010E946D33C8010E94C5286F960FB677
:106C1000F894DEBF0FBECDBFCF91DF911F910F91D2
:106C2000FF90EF900895EF92FF920F931F93DF93E1
:106C3000CF93CDB7DEB76F970FB6F894DEBF0FBE18
:106C4000CDBF7C0187EA92E0E80EF91EF7011182C0
:106C5000108289E59DEFE80EF91E87010D5C1F4F3C
:106C6000C80140E050E060E070E00E94B77FDE01C4
:106C70001596F8018BE101900D928150E1F7F70133
:106C800081A992A99C838B8381E694E09A8389836E
:106C9000C7016AE371E08E010F5F1F4FA8010E94D8
:106CA0006D33C8010E94C5286F960FB6F894DEBFF9
:106CB0000FBECDBFCF91DF911F910F91FF90EF904D
:106CC00008950F931F93CF93DF93DC01D3961C920B
:106CD000D397D6961C92D697D2961C921E92D19795
:106CE00081E694E0D0969C938E939F97AC5ABF4FC9
:106CF0001C9213961C92A755B040FD01E05BFF4F1C
:106D0000AE5ABF4F11961C921E92A255B04091836D
:106D10008083ED01C159DF4FFE0120E030E0482FB4
:106D2000148217821382128240839183215E3F4F27
:106D30007F9681E02633380799F7A855BE4F89E141
:106D40008C9313961C9258961C921B961C92139629
:106D50001C92A15DB140FD01E653FE4FA453BE4F0E
:106D600011961C921E924083918391961C921396C9
:106D70001C92A05FB140FD01E751FE4FA551BE4FEF
:106D800011961C921E9240839183A155BF4F1D9274
:106D90001D921D921C92139718961D921D921D9282
:106DA0001C921397A25AB24012961C9212971396F5
:106DB0001C9213971C9211961C9211978D010256EA
:106DC0001D4FF8011082118212821382AB55BE4F03
:106DD00011961C921E92AD59BF4F1C92FE01C90123
:106DE00011920197E9F7A256BF4F81E08C93A65A02
:106DF000B2409E961C921E929D970E9404CF6857A7
:106E00007C4E8F4F9F4FF801608371838283938301
:106E1000DF91CF911F910F910895DF93CF93CDB75D
:106E2000DEB7E0970FB6F894DEBF0FBECDBFDE0130
:106E30001196E1E1F4E080E101900D928150E1F7DB
:106E4000DE015196E1E0F4E080E101900D92815085
:106E5000E1F7DE019196E1EFF3E080E101900D9220
:106E60008150E1F789819A81AB81BC818093910F38
:106E70009093920FA093930FB093940F89899A895E
:106E8000AB89BC898093810F9093820FA093830F6D
:106E9000B093840F89A19AA1ABA1BCA18093A10F4B
:106EA0009093A20FA093A30FB093A40F8D819E8106
:106EB000AF81B8858093950F9093960FA093970F0D
:106EC000B093980F8D899E89AF89B88D8093850F77
:106ED0009093860FA093870FB093880F8DA19EA1EA
:106EE000AFA1B8A58093A50F9093A60FA093A70F6D
:106EF000B093A80F89859A85AB85BC858093990F3F
:106F000090939A0FA0939B0FB0939C0F898D9A8DAD
:106F1000AB8DBC8D8093890F90938A0FA0938B0FBC
:106F2000B0938C0F89A59AA5ABA5BCA58093A90F9A
:106F30009093AA0FA093AB0FB093AC0F8D859E8555
:106F4000AF85B88980939D0F90939E0FA0939F0F5C
:106F5000B093A00F8D8D9E8DAF8DB8A180938D0FB6
:106F600090938E0FA0938F0FB093900F8DA59EA539
:106F7000AFA5B8A98093AD0F9093AE0FA093AF0FBC
:106F8000B093B00F0E94A46B80E090E0AAEFB3E44E
:106F90008093B50F9093B60FA093B70FB093B80F2F
:106FA0008093B90F9093BA0FA093BB0FB093BC0F0F
:106FB00020E030E040E050E02093B10F3093B20F7A
:106FC0004093B30F5093B40F80E29EE4A0E0B0E092
:106FD00080937D0F90937E0FA0937F0FB093800FCF
:106FE0002093C90F3093CA0F4093CB0F5093CC0F0F
:106FF00080E090E0A0EAB1E48093BD0F9093BE0FD3
:10700000A093BF0FB093C00F8DEC9CECACECBEE333
:107010008093C10F9093C20FA093C30FB093C40F7E
:1070200080E090E0A0EAB0E48093C50F9093C60F93
:10703000A093C70FB093C80F2093D8073093D907F8
:107040004093DA075093DB072093D4073093D5079A
:107050004093D6075093D7072093D0073093D1079A
:107060004093D2075093D30789EB90E09093A617F3
:107070008093A5171092A8171092A7172FEF30E052
:107080003093AA172093A91780EF90E09093AC1744
:107090008093AB171092AE171092AD173093B017C4
:1070A0002093AF1780E290E09093B3198093B219C8
:1070B0008AE097EDADEAB1E48093B4039093B50311
:1070C000A093B603B093B70368EB7EE185EC9FE332
:1070D0000E947A986093B8037093B9038093BA03BF
:1070E0009093BB036AE979E189E992E40E94889868
:1070F0006093BC037093BD038093BE039093BF0362
:107100000E94989780E090E0A0E8BFE38093C003DE
:107110009093C103A093C203B093C303E7E2F3E0EB
:10712000949108C08091C00085FFFCCF9093C60069
:10713000319694919923B1F7EDE2F3E0949108C070
:107140008091C00085FFFCCF9093C600319694914A
:107150009923B1F78091C00085FFFCCF8AE080932E
:10716000C600E0960FB6F894DEBF0FBECDBFCF913C
:10717000DF910895CF93DF93C7E2D3E0FE019491AE
:1071800008C08091C00085FFFCCF9093C600319667
:1071900094919923B1F7E7E0F5E0949108C08091CC
:1071A000C00085FFFCCF9093C6003196949199233F
:1071B000B1F78091C00085FFFCCF8AE08093C600C4
:1071C000FE019491E7E2F3E008C08091C00085FFE2
:1071D000FCCF9093C600319694919923B1F74091DA
:1071E000910F5091920F6091930F7091940F8FEFC8
:1071F00094E00E9441424091950F5091960F60910A
:10720000970F7091980F8CEF94E00E94414240914B
:10721000990F50919A0F60919B0F70919C0F89EF7D
:1072200094E00E94414240919D0F50919E0F6091C9
:107230009F0F7091A00F86EF94E00E944142EBE314
:10724000F1E007C08091C00085FFFCCF319690939C
:10725000C60090819923B1F78091C00085FFFCCFD3
:107260008AE08093C600FE019491E7E2F3E008C053
:107270008091C00085FFFCCF9093C6003196949119
:107280009923B1F7ECEDF4E0949108C08091C0002F
:1072900085FFFCCF9093C600319694919923B1F766
:1072A0008091C00085FFFCCF8AE08093C600FE017C
:1072B0009491E7E2F3E008C08091C00085FFFCCF25
:1072C0009093C600319694919923B1F74091810F24
:1072D0005091820F6091830F7091840F83ED94E041
:1072E0000E9441424091850F5091860F6091870F17
:1072F0007091880F80ED94E00E9441424091890F87
:1073000050918A0F60918B0F70918C0F8DEC94E0EF
:107310000E94414240918D0F50918E0F60918F0FCE
:107320007091900F8AEC94E00E944142EBE3F1E00F
:1073300007C08091C00085FFFCCF31969093C600B6
:1073400090819923B1F78091C00085FFFCCF8AE03E
:107350008093C600FE019491E7E2F3E008C08091BB
:10736000C00085FFFCCF9093C6003196949199237D
:10737000B1F7ECEAF4E0949108C08091C00085FF79
:10738000FCCF9093C600319694919923B1F78091E8
:10739000C00085FFFCCF8AE08093C600FE01949177
:1073A000E7E2F3E008C08091C00085FFFCCF909336
:1073B000C600319694919923B1F74091A10F509155
:1073C000A20F6091A30F7091A40F83EA94E00E9432
:1073D000C6464091A50F5091A60F6091A70F7091DE
:1073E000A80F80EA94E00E94C6464091A90F5091F0
:1073F000AA0F6091AB0F7091AC0F8DE994E00E94E1
:10740000C6464091AD0F5091AE0F6091AF0F709195
:10741000B00F8AE994E00E94C646EBE3F1E007C0B2
:107420008091C00085FFFCCF31969093C60090817B
:107430009923B1F78091C00085FFFCCF8AE080934B
:10744000C600FE019491E7E2F3E008C08091C0001D
:1074500085FFFCCF9093C600319694919923B1F7A4
:10746000E5E6F4E0949108C08091C00085FFFCCF70
:107470009093C600319694919923B1F78091C00002
:1074800085FFFCCF8AE08093C600FE019491E7E27D
:10749000F3E008C08091C00085FFFCCF9093C60048
:1074A000319694919923B1F74091B50F5091B60F51
:1074B0006091B70F7091B80F8CE594E00E94414243
:1074C0004091B90F5091BA0F6091BB0F7091BC0FF2
:1074D00089E594E00E944142EBE3F1E007C080912E
:1074E000C00085FFFCCF31969093C6009081992310
:1074F000B1F78091C00085FFFCCF8AE08093C60081
:10750000FE019491E7E2F3E008C08091C00085FF9E
:10751000FCCF9093C600319694919923B1F7E6EA97
:10752000F3E0949108C08091C00085FFFCCF909358
:10753000C600319694919923B1F78091C00085FFE0
:10754000FCCF8AE08093C600FE019491E7E2F3E06D
:1075500008C08091C00085FFFCCF9093C600319693
:1075600094919923B1F74091B10F5091B20F60916E
:10757000B30F7091B40F8DE993E00E9441424091A6
:10758000C90F5091CA0F6091CB0F7091CC0F8AE94F
:1075900093E00E94414240917D0F50917E0F609197
:1075A0007F0F7091800F87E993E00E94C64640915B
:1075B000BD0F5091BE0F6091BF0F7091C00F84E955
:1075C00093E00E9441424091C10F5091C20F6091DF
:1075D000C30F7091C40F81E993E00E944142409132
:1075E000C50F5091C60F6091C70F7091C80F8EE8FC
:1075F00093E00E944142EBE3F1E007C08091C000BC
:1076000085FFFCCF31969093C60090819923B1F706
:107610008091C00085FFFCCF8AE08093C600FE0108
:107620009491E7E2F3E008C08091C00085FFFCCFB1
:107630009093C600319694919923B1F7ECE7F3E06B
:10764000949108C08091C00085FFFCCF9093C60044
:10765000319694919923B1F78091C00085FFFCCFBA
:107660008AE08093C600FE019491E7E2F3E008C04F
:107670008091C00085FFFCCF9093C6003196949115
:107680009923B1F74091D0075091D1076091D2076B
:107690007091D30783E793E00E9441424091D40761
:1076A0005091D5076091D6077091D70780E793E096
:1076B0000E9441424091D8075091D9076091DA0762
:1076C0007091DB078DE693E00E944142EBE3F1E02D
:1076D00007C08091C00085FFFCCF31969093C60013
:1076E00090819923B1F78091C00085FFFCCF8AE09B
:1076F0008093C600FE019491E7E2F3E008C0809118
:10770000C00085FFFCCF9093C600319694919923D9
:10771000B1F7EFE5F3E0949108C08091C00085FFD8
:10772000FCCF9093C600319694919923B1F7809144
:10773000C00085FFFCCF8AE08093C600FE019491D3
:10774000E7E2F3E008C08091C00085FFFCCF909392
:10775000C600319694919923B1F74091B4035091AA
:10776000B5036091B6037091B70385E593E00E947D
:1077700041426091B8037091B9038091BA0390912E
:10778000BB030E948198AB01BC0182E593E00E949B
:1077900041426091BC037091BD038091BE03909102
:1077A000BF030E948F98AB01BC018FE493E00E945D
:1077B0004142EBE3F1E007C08091C00085FFFCCFC0
:1077C00031969093C60090819923B1F78091C000C3
:1077D00085FFFCCF8AE08093C600DF91CF910895AA
:1077E0001F920F920FB60F920BB60F9211242F9388
:1077F0003F934F938F939F93EF93FF934091C600D6
:10780000E0910805F091090531969F012F773070BE
:10781000319780910A0590910B052817390739F0A7
:10782000E857FB4F40833093090520930805FF91EB
:10783000EF919F918F914F913F912F910F900BBEA0
:107840000F900FBE0F901F9018959A01AB0120303A
:1078500081EE380780E0480780E0580749F182E070
:107860008093C00060E079E08DE390E00E94EAD967
:107870002150304040405040CA01B90122E030E080
:1078800040E050E00E94EAD93093C5002093C40044
:107890008091C10080618093C1008091C1008860A7
:1078A0008093C1008091C10080688093C1000895D9
:1078B0001092C00020E130E0E7CF20910A0530911E
:1078C0000B0580910805909109058217930719F41B
:1078D0002FEF3FEF0EC0F901E857FB4F80812F5F7C
:1078E0003F4F2F77307030930B0520930A05282FD8
:1078F00030E0C901089580910A0590910B0590939D
:10790000090580930805089508952F923F924F929C
:107910005F926F927F928F929F92AF92BF92CF921F
:10792000DF92EF92FF920F931F93DF93CF93CDB728
:10793000DEB7A0970FB6F894DEBF0FBECDBF1C0117
:107940006A017B01411551056105710549F440E368
:1079500050E060E070E020E030E00E944F3D56C013
:10796000882499245401422E55246624772401E06A
:1079700010E00C0F1D1F080D191DC701B601A30152
:1079800092010E94C8D9F80160830894811C911C5F
:10799000A11CB11CC701B601A30192010E94C8D964
:1079A000C901DA016C017D01C114D104E104F104C3
:1079B000F1F681E0E82EF12CEC0EFD1EE80CF91C2E
:1079C0003E010894611C711CD501C4010197A109F5
:1079D000B1096C01C818D90816C0F601EE0DFF1DDB
:1079E00040814A3010F4405D01C0495C552747FD95
:1079F0005095652F752FC10120E030E00E944F3D6A
:107A00000894E108F1086E147F0439F7A0960FB6C8
:107A1000F894DEBF0FBECDBFCF91DF911F910F91C4
:107A2000FF90EF90DF90CF90BF90AF909F908F909E
:107A30007F906F905F904F903F902F900895211509
:107A4000310539F48091C00085FFFCCF4093C6001A
:107A500008950E94853C0895EF92FF920F931F9323
:107A60009A017B0100E010E0B801A7010E941F3DD0
:107A70001F910F91FF90EF900895EF92FF920F9357
:107A80001F939A01E62EFF2400E010E0B801A70141
:107A90000E941F3D1F910F91FF90EF900895EF926C
:107AA000FF920F931F93CF93DF93EC017A018B0129
:107AB0002115310539F48091C00085FFFCCFE0929B
:107AC000C6001BC02A303105B1F477FF10C04DE26B
:107AD00050E060E070E020E030E00E944F3D109503
:107AE0000095F094E094E11CF11C011D111DCE01E4
:107AF000B801A7012AE00E94853CDF91CF911F9138
:107B00000F91FF90EF900895EF92FF920F931F93C4
:107B10007B019A010027F7FC0095102FB801A701FF
:107B20000E944F3D1F910F91FF90EF9008950F938A
:107B30001F938C014DE050E060E070E020E030E009
:107B40000E944F3DC8014AE050E060E070E020E054
:107B500030E00E944F3D1F910F910895CF92DF9228
:107B6000EF92FF920F931F938C019A016B01EE2409
:107B7000FF24B701A6010E941F3DC8010E94973D46
:107B80001F910F91FF90EF90DF90CF9008959F92FB
:107B9000AF92BF92CF92DF92EF92FF920F931F931B
:107BA000CF93DF93EC017A018B01922ECB01BA01C6
:107BB00020E030E040E050E00E94D0D588236CF413
:107BC000CE014DE250E060E070E020E030E00E9445
:107BD0004F3D17FB109517F91095AA2420E030E0CF
:107BE00040E05FE30BC0CA01B90120E030E040E2B1
:107BF00051E40E94D7D59B01AC01A394A91498F33A
:107C0000C801B7010E94F7D47B018C010E9444D6C1
:107C10005B016C010E9470D69B01AC01C801B701E9
:107C20000E94F6D47B018C01CE01B601A5012AE0A9
:107C300030E00E941F3D9920A1F1ECE3F1E007C084
:107C40008091C00085FFFCCF31969093C600908153
:107C50009923B1F726C0C801B70120E030E040E227
:107C600051E40E94B0D87B018C010E943FD65B0199
:107C70006C01CC24B7FCC094DC2CCE01B601A5016C
:107C80002AE030E00E944F3DC601B5010E9472D645
:107C90009B01AC01C801B7010E94F6D47B018C01A5
:107CA0009A949920C1F6DF91CF911F910F91FF9087
:107CB000EF90DF90CF90BF90AF909F9008950E947B
:107CC000C73D0895EF92FF920F931F93CF93DF93D9
:107CD000EC01E090DC07F090DD070091DE071091E9
:107CE000DF07688179818A819B81A80197010E94C1
:107CF000D0D5882324F4E882F9820A831B83E0909C
:107D0000E007F090E1070091E2071091E3076C8132
:107D10007D818E819F81A80197010E94D0D5882303
:107D200024F4EC82FD820E831F83E090E407F09040
:107D3000E5070091E6071091E707688579858A8550
:107D40009B85A80197010E94D0D5882324F4E8865A
:107D5000F9860A871B87E0907A03F0907B030091F5
:107D60007C0310917D03688179818A819B81A801C0
:107D700097010E94DED7181624F4E882F9820A835C
:107D80001B83E0907E03F0907F03009180031091AD
:107D900081036C817D818E819F81A80197010E9462
:107DA000DED7181624F4EC82FD820E831F83E09048
:107DB0008203F0908303009184031091850368850A
:107DC00079858A859B85A80197010E94DED71816C0
:107DD00024F4E886F9860A871B87DF91CF911F91EB
:107DE0000F91FF90EF9008958091F80708950F93F9
:107DF0001F93CF93DF938130910569F46F5F7F4FBD
:107E000009F059C08DE095E00E94613689EF97E056
:107E10000E94B58D50C0892B09F04DC06F5F7F4F18
:107E200009F049C081E694E09093F7068093F60646
:107E30008091FD06882321F08AEF96E00E94CF8092
:107E400081E694E09093D8068093D7068091DE0671
:107E5000882321F08BED96E00E94CF80C3E9D6E025
:107E600001E614E005C06F9785E0CD35D80751F0E5
:107E7000198308838F818823B1F3CE0104960E9471
:107E8000CF80F1CF81E694E0998388838F81882326
:107E900021F0CE0104960E94CF8081E694E0909379
:107EA0003D0580933C0580914305882321F080E4C3
:107EB00095E00E94CF80DF91CF911F910F9108959F
:107EC00080E090E06FEF7FEF0E94F73E089581E041
:107ED00090E06FEF7FEF0E94F73E08950E946B984D
:107EE0008091F807882309F03AC081E08093F80771
:107EF0008091510A9091520AA091530AB091540A6C
:107F00008093550A9093560AA093570AB093580A43
:107F1000EDE1F5E0949108C08091C00085FFFCCFB1
:107F20009093C600319694919923B1F7EEE2F5E073
:107F3000949108C08091C00085FFFCCF9093C6004B
:107F4000319694919923B1F78091C00085FFFCCFC1
:107F50008AE08093C60084E295E00E94C0BF089545
:107F6000F8940E946B985E9A1092E8075E9A1092BD
:107F7000E907159A1092EA075E9AEDE1F5E094910F
:107F800008C08091C00085FFFCCF9093C600319659
:107F900094919923B1F7EDEAF5E0949108C08091AE
:107FA000C00085FFFCCF9093C60031969491992331
:107FB000B1F78091C00085FFFCCF8AE08093C600B6
:107FC00084EA95E00E94CFBFFFCF0E9404CF609368
:107FD000590A70935A0A80935B0A90935C0AE09165
:107FE000820AF091830AEC57F54F80818823A9F427
:107FF000ECECF5E0949108C08091C00085FFFCCFC7
:108000009093C600319694919923B1F78091C00066
:1080100085FFFCCF8AE08093C6000895EF92FF921F
:108020000F931F930E9404CFE0905D0AF0905E0AC8
:1080300000915F0A1091600A2091590A30915A0A02
:1080400040915B0A50915C0A621B730B840B950B89
:10805000E616F7060807190738F4E114F1040105DC
:10806000110511F00E94B03F80919A0390919B03FB
:10807000A0919C03B0919D030097A105B10559F112
:108080000E9404CF2091590A30915A0A40915B0A0C
:1080900050915C0A621B730B840B950B20919A0321
:1080A00030919B0340919C0350919D032617370705
:1080B0004807590780F49091BE148091BF14981717
:1080C00051F45E9A1092E8075E9A1092E907159AA9
:1080D0001092EA075E9A0E94146E1F910F91FF9012
:1080E000EF9008956F927F928F929F92AF92BF927E
:1080F000CF92DF92EF92FF920F931F93F82E609131
:10810000610A7091620A8091630A9091640A2091D9
:10811000650A3091660A4091670A5091680A0E9488
:10812000EBD73B014C0100D000D000D00DB71EB7FB
:108130000F5F1F4F6091720370917303882777FD63
:108140008095982F0E9472D620919E0330919F03B4
:108150004091A0035091A1030E94B0D820E030E0EC
:1081600040E752E40E94D7D520E030E048EC52E4EA
:108170000E94D7D55B016C01F80160827182828216
:108180009382F4828091EB07858380EC97E06DE623
:108190007AE041E65AE020E001E032E0E32E0E947E
:1081A000006780916D0A90916E0AA0916F0AB0915C
:1081B000700A8093C0079093C107A093C207B09341
:1081C000C3078091710A9091720AA091730AB091CD
:1081D000740A8093C4079093C507A093C607B09311
:1081E000C7078091750A9091760AA091770AB0919D
:1081F000780A8093C8079093C907A093CA07B093E1
:10820000CB078091790A90917A0AA0917B0AB0916C
:108210007C0A8093CC079093CD07A093CE07B093B0
:10822000CF078DB79EB706960FB6F8949EBF0FBEC8
:108230008DBF0E9404CF6093590A70935A0A8093AD
:108240005B0A90935C0A1F910F91FF90EF90DF9073
:10825000CF90BF90AF909F908F907F906F90089538
:10826000CF92DF92EF92FF920F931F938DE69AE0E9
:108270000E94623E0E9404CF6093590A70935A0A8A
:1082800080935B0A90935C0A6091C0077091C1076C
:108290008091C2079091C30720916D0A30916E0AB8
:1082A00040916F0A5091700A0E94D0D5882309F03E
:1082B0007AC06091C4077091C5078091C6079091FC
:1082C000C7072091710A3091720A4091730A509148
:1082D000740A0E94D0D5882309F065C060919E037E
:1082E00070919F038091A0039091A10320E030E062
:1082F00040E752E40E94D7D57B018C018DE69AE0DD
:1083000061E77AE045E75AE029E73AE0EBEECE2E66
:10831000E7E0DE2E0E94FD7080916D0A90916E0A5A
:10832000A0916F0AB091700A8093C0079093C10723
:10833000A093C207B093C3078091710A9091720A0B
:10834000A091730AB091740A8093C4079093C507F3
:10835000A093C607B093C7078091750A9091760ADB
:10836000A091770AB091780A8093C8079093C907C3
:10837000A093CA07B093CB078091790A90917A0AAB
:10838000A0917B0AB0917C0A8093CC079093CD0793
:10839000A093CE07B093CF071F910F91FF90EF905E
:1083A000DF90CF90089560917203709173038827D6
:1083B00077FD8095982F0E9472D620919E03309170
:1083C0009F034091A0035091A1030E94B0D820E0E8
:1083D00030E040E752E40E94D7D520E030E048EC9E
:1083E00052E488CF8CE095E00E947B3CEFECF5E016
:1083F000949108C08091C00085FFFCCF9093C60087
:10840000319694919923B1F74091510A5091520AB3
:108410006091530A7091540A4F5F5F4F6F4F7F4FC7
:108420008CE095E02AE030E00E944F3D8091C00052
:1084300085FFFCCF8AE08093C6000E94E53F089547
:108440004091820A5091830A20E630E0B901469FAC
:108450009001479F300D569F300D1124682F7727CC
:1084600067FD7095C9018257954F0E9465239C0155
:1084700090938D0A80938C0A80E0232B09F081E091
:108480000895FC01949108C08091C00085FFFCCF45
:108490009093C600319694919923B1F78CE095E0C2
:1084A00022E030E00E945F3E08952F923F924F926B
:1084B0005F926F927F928F929F92AF92BF92CF9274
:1084C000DF92EF92FF920F931F93DF93CF93CDB77D
:1084D000DEB728970FB6F894DEBF0FBECDBF9A83E4
:1084E00089838330910508F091C1FC01E051F84F78
:1084F000D4908C01000F111F000F111FF801E054E0
:10850000F84F80E090E0A0E0B0E080839183A28308
:10851000B38380EC97E064EC77E048EC57E02CEC18
:1085200037E00E94ED6BE981FA81EE0FFF1FEA57F9
:10853000FC4F0190F081E02DF7FD0EC0CF01880FB8
:10854000991F8E0F9F1F04571C4FD8016D917C916E
:108550008750984F0E947F8E69807A80660C771CC6
:10856000660C771CF301ED50F84FE590F5900591FE
:1085700014916D2D772767FD7095882777FD80957D
:10858000982F0E9472D61B012C01F301E359F54F7D
:10859000F887EF83C801B70120E030E040EC5FE3EB
:1085A0000E94B0D8A20191010E94B0D8AF81B885D5
:1085B0006D937D938D939C931397F301EE59FC4F2C
:1085C000FC83EB83608171818281938160939E0340
:1085D00070939F038093A0039093A10320E030E069
:1085E00040E752E40E94D7D57B018C018DE69AE0EA
:1085F00061E77AE045E75AE029E73AE0EBEECE2E74
:10860000E7E0DE2E0E94FD700E948B9093012054C3
:10861000384F3E832D8380E090E0A0E0B0E0F90188
:1086200080839183A283B38380EC97E064EC77E04E
:1086300048EC57E02CEC37E00E94ED6BF301E15081
:10864000F84F85909590A590B490C501B4019058CD
:10865000A20191010E94B0D8AF81B8856D937D933E
:108660008D939C93139760919E0370919F038091CB
:10867000A0039091A10320E030E040E752E40E9483
:10868000D7D57B018C018DE69AE061E77AE045E77A
:108690005AE029E73AE00E94FD700E948B90C501E4
:1086A000B401A50194010E94F7D4A20191010E9496
:1086B000B0D8EF81F8856083718382839383AB8127
:1086C000BC816D917D918D919C9120E030E040E0E6
:1086D0005FE30E94B0D860939E0370939F038093E2
:1086E000A0039093A10320E030E040E752E40E9411
:1086F000D7D57B018C018DE69AE061E77AE045E70A
:108700005AE029E73AE00E94FD700E948B90F30145
:10871000E55FF74F6591759185919491F301E05371
:10872000F84FA080B180C280D380A60195010E943D
:10873000F7D47B018C01CB01D801ED81FE818083D0
:108740009183A283B383F301E95EF74F659175913D
:10875000859194912CED822E27E0922E860C971C09
:10876000A60195010E94F7D4D4016D937D938D935A
:108770009C931397F301ED5DF74F6591759185918A
:108780009491EAE7F3E06E0E7F1EA60195010E9428
:10879000F7D4D3016D937D938D939C931397C70169
:1087A000D801EF81F88580839183A283B38380E031
:1087B00090E0A0E0B0E080939E0390939F03A0938D
:1087C000A003B093A1030E94A98FE981FA81E85127
:1087D000F84F81E08083A981BA81AA0FBB1FFD01F8
:1087E000EA57FC4F0190F081E02DF7FD0FC0CF015B
:1087F000880F991F8E0F9F1FAA0FBB1FA257BC4F38
:108800006D917C918750984F0E947F8E28960FB66D
:10881000F894DEBF0FBECDBFCF91DF911F910F91B6
:10882000FF90EF90DF90CF90BF90AF909F908F9090
:108830007F906F905F904F903F902F9008950F938F
:108840001F93CF93DF93C6E8D3E00EE813E02881AF
:10885000398137FD0CC0C901880F991F820F931F02
:10886000F801608171818750984F0E947F8E229617
:108870000C5F1F4FF3E0CC38DF0749F7DF91CF9152
:108880001F910F91089580918C0A90918D0A019605
:1088900060E070E04AE050E00E94D42108958091A9
:1088A0008C0A90918D0A019660E070E00E9474201D
:1088B0000895CF93DF93EC018091EB078093500AEA
:1088C00084E50E942042882309F46FC00E944F442F
:1088D0000E9444D6262F6093500A662309F465C08F
:1088E000E7E1F5E0949108C08091C00085FFFCCFDE
:1088F0009093C600319694919923B1F7C936D1056A
:1089000099F0CA36D10524F4C836D105F1F50FC067
:10891000CD36D10531F0CA3DD105B9F5EEE3F1E030
:1089200031C0E5E5F1E023C0ECE6F1E015C0E3E895
:10893000F1E007C08091C00085FFFCCF3196909395
:10894000C60090819923B1F720C08091C00085FFB7
:10895000FCCF31969093C60090819923B1F715C052
:108960008091C00085FFFCCF31969093C600908126
:108970009923B1F70AC08091C00085FFFCCF3196E2
:108980009093C60090819923B1F78CE095E0622F17
:1089900040E050E00E943D3D8091C00085FFFCCF4B
:1089A0008AE08093C60081E001C080E0DF91CF9132
:1089B0000895AF92BF92CF92DF92EF92FF920F9302
:1089C0001F93CF93DF9350ECE52E57E0F52ECDE6C5
:1089D000DAE000E010E0F801EF5DFB4F80810E94DB
:1089E0002042882339F10E944F445B016C01F80159
:1089F000E654F84F8081882311F061E002C0609155
:108A00007D0A70E0882777FD8095982F0E9472D6A6
:108A1000F70120813181428153810E94B0D89B01AE
:108A2000AC01C601B5010E94F7D4688379838A83BB
:108A30009B8309C0F70180819181A281B3818883E2
:108A40009983AA83BB830F5F1F4F84E090E0E80EF9
:108A5000F91E24960430110509F0BDCF86E40E946A
:108A600020428823E1F00E944F447B018C016093F7
:108A70007E0A70937F0A8093800A9093810A20E097
:108A800030E040E050E00E94DED7181644F4E09257
:108A90009E03F0929F030093A0031093A103DF9124
:108AA000CF911F910F91FF90EF90DF90CF90BF90EB
:108AB000AF9008950E94D94489E40E9420428823FF
:108AC00059F00E944F446093610A7093620A809348
:108AD000630A9093640A0CC080E090E0A0E0B0E0EC
:108AE0008093610A9093620AA093630AB093640A28
:108AF0008AE40E942042882359F00E944F446093E8
:108B0000650A7093660A8093670A9093680A0895CD
:108B100080E090E0A0E0B0E08093650A9093660A60
:108B2000A093670AB093680A0895EF92FF920F939B
:108B30001F9380911005882309F423C180910F05AC
:108B4000882309F41EC1E090C807F090C90700917E
:108B5000CA071091CB07C801B70120E030E040E020
:108B600050E00E94DED718160CF00BC1609112087D
:108B7000709113088091140890911508A80197012D
:108B80000E94D0D5882309F4FCC061E070E080E049
:108B900090E020E031E040E050E00E94D8D46093C3
:108BA000FD0760934B0A8091C0079091C107A09187
:108BB000C207B091C3078093FE079093FF07A0936D
:108BC0000008B09301088091C4079091C507A09157
:108BD000C607B091C7078093020890930308A0933B
:108BE0000408B09305082091C8073091C907409147
:108BF000CA075091CB07209306083093070840938B
:108C00000808509309088091CC079091CD07A09156
:108C1000CE07B091CF0780930A0890930B08A093DA
:108C20000C08B0930D08209312083093130840935A
:108C300014085093150880919E0390919F03A09172
:108C4000A003B091A10380930E0890930F08A09306
:108C50001008B09311088091531790915417909376
:108C60001708809316088091551790915617909386
:108C7000190880931808809157179091581790936E
:108C80001B0880931A088091591790915A17909356
:108C90001D0880931C08809155179091561790934A
:108CA0001F0880931E088091820A9091830A9093F6
:108CB0002108809320088091120C9091130C9093BE
:108CC0002308809322088091180C9091190C90939E
:108CD000250880932408A6E2B8E0EEE8FAE080E8F0
:108CE00091E001900D920197E1F78091EE0790914C
:108CF000EF07A091F007B091F1078093AA09909334
:108D0000AB09A093AC09B093AD098DE095E06EEA94
:108D100079E00E94B72C8091AF079091B007A091A5
:108D2000B107B091B2078093A6099093A709A093C9
:108D3000A809B093A9098DE095E06BE37AE04AE5D4
:108D40000E94B7298DE095E06DEF77E04FE452E0A7
:108D50000E9494308F5F9F4FA1F4EAE9F1E007C0D1
:108D60008091C00085FFFCCF31969093C600908122
:108D70009923B1F78091C00085FFFCCF8AE08093F2
:108D8000C6001F910F91FF90EF900895FC01949100
:108D900008C08091C00085FFFCCF9093C60031963B
:108DA00094919923B1F78CE095E02AE030E00E949D
:108DB0001F3D0895CF93DF93FC0180818B3309F42D
:108DC0006FC08091180C9091190C04970CF068C03A
:108DD0008091120C9091130C20E630E0829FE0010C
:108DE000839FD00D929FD00D1124C257D54FCE0135
:108DF000BF010E947023E7E1F5E0949108C08091E3
:108E0000C00085FFFCCF9093C600319694919923C2
:108E1000B1F7E3ECFAE0949108C08091C00085FFBF
:108E2000FCCF9093C600319694919923B1F7FE013F
:108E300007C08091C00085FFFCCF31969093C6009B
:108E400090819923B1F7E1ECFAE0949108C0809108
:108E5000C00085FFFCCF9093C60031969491992372
:108E6000B1F78091C00085FFFCCF8AE08093C600F7
:108E70008091120C9091130C019664E070E00E94B6
:108E8000B5D99093130C8093120C8091180C90918B
:108E9000190C01969093190C8093180C81E001C075
:108EA00080E0DF91CF910895EF92FF920F931F938F
:108EB000DF93CF93CDB7DEB76E970FB6F894DEBFD2
:108EC0000FBECDBF6091F6077091F7076115710570
:108ED00011F480E037C08E010F5F1F4FC8014DE1D4
:108EE00050E00E941B231E8EEE24FF24C801FC01CB
:108EF000EE0DFF1D1081112331F01A3021F008947E
:108F0000E11CF11CF4CFCE010196FC01EE0DFF1D1A
:108F100010820E94DA468823A1F0112371F0089490
:108F2000E11CF11C8091F6079091F7078E0D9F1DB3
:108F30009093F7078093F60704C01092F7071092FA
:108F4000F60781E06E960FB6F894DEBF0FBECDBF78
:108F5000CF91DF911F910F91FF90EF900895909323
:108F6000F7078093F6070E945447089580914C0AB2
:108F700090914D0A1816190614F080E0089580911A
:108F80001B0C90911C0C20E630E0AC01429FC0010C
:108F9000439F900D529F900D1124835E934F0E942A
:108FA000DA46882311F481E0089580911B0C90919A
:108FB0001C0C019690931C0C80931B0C80914C0A06
:108FC00090914D0A019790934D0A80934C0A81E04D
:108FD00008952F923F924F925F926F927F928F925D
:108FE0009F92AF92BF92CF92DF92EF92FF920F9338
:108FF0001F93DF93CF93CDB7DEB76E970FB6F8947C
:10900000DEBF0FBECDBF0E945447882309F415C2AE
:10901000F5C32D3071F02A3321F480910F0C882391
:1090200041F08091100C9091110C8F3591050CF44A
:10903000DFC1E091100CF091110C309709F417C3C7
:10904000A091120CB091130CAA9D7001AB9DF00C75
:10905000BA9DF00C1124EE0DFF1DE257F54F108262
:1090600080910F0C882309F0BEC110920F0CAC57F1
:10907000B54F1C9287010257154FC8016EE470E08E
:109080000E9465239C01009709F4F7C090938D0A14
:1090900080938C0A2F5F3F4F201B310B2E0D3F1DFD
:1090A000C9018257954F60E070E04AE050E00E94AD
:1090B000D4216093140C7093150C8093160C90932C
:1090C000170CC090510AD090520AE090530AF090C9
:1090D000540AA70196012F5F3F4F4F4F5F4F621712
:1090E00073078407950709F46AC38091120C909165
:1090F000130C9C012A9DC0012B9D900D3A9D900D53
:1091000011248257954F6FE779E00E942A23892B1B
:1091100009F055C3EDE1F5E0949108C08091C000DD
:1091200085FFFCCF9093C600319694919923B1F7B7
:10913000ECE4F9E0949108C08091C00085FFFCCF79
:109140009093C600319694919923B1F78CE095E005
:10915000B701A6012AE030E00E944F3D8091C00097
:1091600085FFFCCF73C0FE264F5FFC01E40FF11DAD
:10917000E257F54FE081EA32B1F730938D0A209340
:109180008C0AC901019660E070E00E9474200E9480
:109190003FD62F2D30E02617370709F45DC0EDE1EB
:1091A000F5E0949108C08091C00085FFFCCF9093BA
:1091B000C600319694919923B1F7EDE2F9E09491CC
:1091C00008C08091C00085FFFCCF9093C600319607
:1091D00094919923B1F74091510A5091520A6091AC
:1091E000530A7091540A8CE095E02AE030E00E9426
:1091F0004F3D8091C00085FFFCCF28C0EDE1F5E038
:10920000949108C08091C00085FFFCCF9093C60068
:10921000319694919923B1F7E3E0F9E0949108C075
:109220008091C00085FFFCCF9093C6003196949149
:109230009923B1F78CE095E0B701A6012AE030E070
:109240000E944F3D8091C00085FFFCCF8AE0809353
:10925000C6000E94F2414AC08091140C9091150CF6
:10926000A091160CB091170C8093510A9093520A5A
:10927000A093530AB093540A3EC0C8016AE270E05A
:109280000E946523009709F436C0EDE1F5E0949162
:1092900008C08091C00085FFFCCF9093C600319636
:1092A00094919923B1F7E9EDF8E0949108C0809189
:1092B000C00085FFFCCF9093C6003196949199230E
:1092C000B1F74091510A5091520A6091530A70913E
:1092D000540A8CE095E02AE030E00E944F3D8091F6
:1092E000C00085FFFCCF8AE08093C6001092110C6D
:1092F0001092100C83C28091120C9091130C8A9DD5
:1093000070018B9DF00C9A9DF00C1124870102577F
:10931000154FC80167E470E00E9465239C01009727
:1093200009F44BC090938D0A80938C0A2F5F3F4FB6
:10933000201B310B2E0D3F1DC9018257954F60E058
:1093400070E00E9474200E943FD664307105A8F539
:109350008091F8078823C9F480910D05882369F569
:10936000992DE6EDF8E008C08091C00085FFFCCFA4
:109370009093C600319694919923B1F78091C000E3
:1093800085FFFCCF7092C60018C0982DE0E6F8E08B
:1093900008C08091C00085FFFCCF9093C600319635
:1093A00094919923B1F78091C00085FFFCCF709212
:1093B000C60086E598E00E94C0BF8091120C909193
:1093C000130C019664E070E00E94B5D99093130CE1
:1093D0008093120C8091180C9091190C0196909327
:1093E000190C8093180C1092110C1092100C32C0B2
:1093F0002B3311F460920F0C80910F0C882351F5E0
:109400002091100C3091110C8091120C9091130C42
:109410008A9DF0018B9DF00D9A9DF00D1124E20FB5
:10942000F31FE257F54F80910E0C80832F5F3F4F63
:109430003093110C2093100C0DC0A0E6AA2EB12C75
:10944000E0E6F8E08490FAE07F2EE6EDF8E0949014
:1094500066246394809108059091090520910A057E
:1094600030910B05821B930B8F779070892B09F439
:10947000C0C18091180C9091190C04970CF0B9C1DF
:109480008CE095E00E945D3C282F80930E0C8A3082
:1094900009F0BFCDCECD8091100C9091110C892B8D
:1094A00009F0ACC10E94B647882309F0A7C180919A
:1094B000180C9091190C892B09F02FC110921A0CDD
:1094C0002CC14D3099F0433211F04A3321F4809190
:1094D0000F0C882359F08091100C9091110C8F354E
:1094E000910524F42F5F3F4F09F0F2C02091AF07A0
:1094F0003091B0074091B1075091B2078091A70712
:109500009091A807A091A907B091AA072817390739
:109510004A075B0708F49EC0932DE3E4F8E008C017
:109520008091C00085FFFCCF9093C6003196949146
:109530009923B1F78091C00085FFFCCF2092C6002F
:109540000E9404CF6093F2077093F3078093F407AF
:109550009093F5072091EE073091EF074091F007C7
:109560005091F107621B730B840B950B28EE33E0CF
:1095700040E050E00E94C8D9F22EE32ED42EC52E32
:10958000EDB7FEB738970FB6F894FEBF0FBEEDBF2C
:109590000DB71EB70F5F1F4FB282A182F801538231
:1095A0004282622F732F842F952F20E13EE040E00E
:1095B00050E00E94C8D9F801358324836F2D7E2D99
:1095C0008D2D9C2D2CE330E040E050E00E94C8D966
:1095D000CA01B9012CE330E040E050E00E94C8D954
:1095E000F801778366830E949423982DE7E1F5E0E4
:1095F0002DB73EB7285F3F4F0FB6F8943EBF0FBE62
:109600002DBF08C08091C00085FFFCCF9093C6009D
:10961000319694919923B1F7F50107C08091C0006C
:1096200085FFFCCF31969093C60090819923B1F7C6
:109630008091C00085FFFCCF2092C600C5010E942A
:10964000E3BF8DE095E00E94B3308DE095E061E0EE
:109650000E94443280910E0C833211F490921A0CC5
:109660002091100C3091110C2115310519F4109234
:109670000F0CC4C08091120C9091130C869DF001C8
:10968000879DF00D969DF00D1124E20FF31FE25718
:10969000F54F1082FC01EC57F54F90822091180C89
:1096A0003091190C2F5F3F4F3093190C2093180CF9
:1096B000019664E070E00E94B5D99093130C8093FA
:1096C000120C10920F0C1092110C1092100C3AC048
:1096D0004B3311F490920F0C80910F0C882391F56D
:1096E0002091100C3091110C8091120C9091130C60
:1096F000869DF001879DF00D969DF00D1124E20FDF
:10970000F31FE257F54F80910E0C80832F5F3F4F80
:109710003093110C2093100C15C0E0E66E2E712CC6
:1097200099249394E3E4F8E034907AE0272E5E01E4
:109730000894A11CB11C6FE2462E68E0562EE7E1AA
:10974000F5E084902091AF073091B0074091B107C8
:109750005091B2078091A7079091A807A091A907FF
:10976000B091AA07281739074A075B0708F046C0D7
:109770008091180C9091190C04970CF03FC08091C7
:109780001A0C8823D9F58091E3069091E406A09104
:10979000E506B091E6068093AF079093B007A093DB
:1097A000B107B093B2078BED96E00E947C839C01D9
:1097B000482F80930E0C8A3009F083CE97CE80918B
:1097C000120C9091130C8A9D80018B9D100D9A9D17
:1097D000100D1124C8018257954F6AE270E00E9473
:1097E00065239C01009709F409CDFF2440E0C801DE
:1097F000BCCC80910F05882309F04DCE6E960FB634
:10980000F894DEBF0FBECDBFCF91DF911F910F91B6
:10981000FF90EF90DF90CF90BF90AF909F908F9090
:109820007F906F905F904F903F902F900895AF92F0
:10983000BF92CF92DF92EF92FF920F931F93DF932D
:10984000CF93CDB7DEB7C055D0400FB6F894DEBF8A
:109850000FBECDBF8FE492E0EDEFF7E0DF019C019A
:109860001D9221503040E1F780E693E0EDE1FCE00D
:10987000DF019C011D9221503040E1F780911005DD
:10988000882321F48DE095E00E94643180911005D9
:10989000882309F459C3E7EBF1E007C08091C000C9
:1098A00085FFFCCF31969093C60090819923B1F744
:1098B0008091C00085FFFCCF8AE08093C600E2ED76
:1098C000F1E007C08091C00085FFFCCF31969093F6
:1098D000C60090819923B1F78091C00085FFFCCF2D
:1098E0008AE08093C6008CE095E06FE472E04AE085
:1098F00050E00E942C3D8091C00085FFFCCF8AE0A3
:109900008093C6008BE39AE06DEB7AE04FE050E085
:109910000E941B238DE095E06BE37AE00E94AC2966
:10992000882309F411C38DE095E06BE37AE041E010
:109930000E94B7298DE095E06DEF77E04FE452E0AB
:109940000E948F308DE095E00E94D228E9EDF1E091
:1099500007C08091C00085FFFCCF31969093C60070
:1099600090819923B1F78091C00085FFFCCF8AE0F8
:109970008093C6004091FD0750E060E070E08CE00D
:1099800095E02AE030E00E941F3D8091C00085FFF5
:10999000FCCF8AE08093C60040914B0A50E060E023
:1099A00070E08CE095E02AE030E00E941F3D80915D
:1099B000C00085FFFCCF8AE08093C6009091FD0730
:1099C000992309F4AFC280914B0A981709F0A2C2FB
:1099D0001598E6EEF1E007C08091C00085FFFCCF4E
:1099E00031969093C60090819923B1F78091C00081
:1099F00085FFFCCF8AE08093C6000EEF17E02AE0D7
:109A0000F22ED8014D915D916D917C918CE095E0A5
:109A100022E030E00E945F3E8091C00085FFFCCFD5
:109A2000F092C6000C5F1F4FB8E00E301B0749F7DD
:109A3000F80140815181628173818CE095E022E0E0
:109A400030E00E945F3E8091C00085FFFCCF8AE03D
:109A50008093C60006E118E09AE0F92ED8016D91D6
:109A60007C918CE095E04AE050E00E94843D80913A
:109A7000C00085FFFCCFF092C6000E5F1F4FB8E01C
:109A80000E311B0759F7F801608171818CE095E078
:109A90004AE050E00E94843D8091C00085FFFCCFE9
:109AA0008AE08093C600EDE0F2E007C08091C0003C
:109AB00085FFFCCF31969093C60090819923B1F732
:109AC0008091C00085FFFCCF8AE08093C600609142
:109AD0002008709121088CE095E04AE050E00E9457
:109AE000843D8091C00085FFFCCF8AE08093C60052
:109AF00060912208709123088CE095E04AE050E0E4
:109B00000E94843D8091C00085FFFCCF8AE0809355
:109B1000C60060912408709125088CE095E04AE029
:109B200050E00E94843D8091C00085FFFCCF8AE018
:109B30008093C60020E030E040E650E06AE0249FD9
:109B4000F001259FF00D349FF00D1124EA5DF74FD1
:109B500007C08091C00085FFFCCF31969093C6006E
:109B600090819923B1F78091C00085FFFCCF60936D
:109B7000C6002F5F3F4F2430310509F781E2E82E00
:109B8000F12CEC0EFD1E80E1D701E82F1D92EA9525
:109B9000E9F7D701E82F1D92EA95E9F7D701E82FF9
:109BA0001D92EA95E9F701E3C02ED12CCC0EDD1E03
:109BB000D601E82F1D92EA95E9F711E4A12EB12C08
:109BC000AC0EBD1ED5011D928A95E9F76091FE0786
:109BD0007091FF07809100089091010841E023E017
:109BE0008E010F5F1F4F0E94F21F6091020870915B
:109BF0000308809104089091050841E023E08E015C
:109C00000F5E1F4F0E94F21F6091060870910708B7
:109C1000809108089091090841E023E087010E94A3
:109C2000F21F6091060870910708809108089091D2
:109C3000090820E030E040EA50E40E94F7D441E017
:109C400023E085010E94F21F60910A0870910B08C1
:109C500080910C0890910D0841E023E086010E945C
:109C6000F21FEDB7FEB738970FB6F894FEBF0FBEE0
:109C7000EDBF31968DE19CE0ADB7BEB712969C93D7
:109C80008E93119781EB9AE093838283F582E4822D
:109C9000D782C6820E9494230F900F90EDB7FEB733
:109CA00031968DE79CE0ADB7BEB712969C938E932C
:109CB00011978AEA9AE093838283B582A4820E94F4
:109CC00094230F900F908DED9CE0EDB7FEB792833B
:109CD000818380EA9AE0948383830E94942300D056
:109CE000EDB7FEB731968DE39DE0ADB7BEB71296E6
:109CF0009C938E93119789E99AE093838283F582EE
:109D0000E4820E9494230F900F908DE99DE0EDB7BF
:109D1000FEB79283818388E89AE0948383830E94CC
:109D2000942385E090E090934D0A80934C0A05E0DF
:109D300010E00F900F900F900F90B0E6EB2EF12CEB
:109D400039C00E9DC0010F9D900D1E9D900D1124D8
:109D50000F5F1F4F20912008309121082E9DB001E8
:109D60002F9D700D3E9D700D11246A5D774F835EAF
:109D7000934F0E94702380914C0A90914D0A019656
:109D800090934D0A80934C0A809124089091250865
:109D90000197909325088093240880912008909142
:109DA0002108019664E070E00E94B5D990932108E3
:109DB0008093200880912408909125081816190690
:109DC0000CF4BFCF40914C0A50914D0A20E030E096
:109DD00060E670E0AAE01CC0269FF001279FF00D0E
:109DE000369FF00D1124E35EF34F07C08091C00051
:109DF00085FFFCCF31969093C60090819923B1F7EF
:109E00008091C00085FFFCCFA093C6002F5F3F4F1D
:109E1000241735070CF3E2E2F2E007C08091C0009E
:109E200085FFFCCF31969093C60090819923B1F7BE
:109E30008091C00085FFFCCF8AE08093C6004091EE
:109E4000AA095091AB096091AC097091AD098CE001
:109E500095E02AE030E00E941F3D8091C00085FF20
:109E6000FCCF8AE08093C600EEEAF9E007C080915B
:109E7000C00085FFFCCF31969093C6009081992356
:109E8000B1F78091C00085FFFCCF8AE08093C600C7
:109E90004091A6095091A7096091A8097091A9095C
:109EA0008CE095E02AE030E00E941F3D8091C000E8
:109EB00085FFFCCF8AE08093C6008091AA0990912B
:109EC000AB09A091AC09B091AD098093EE079093D6
:109ED000EF07A093F007B093F1078DE095E06EEAED
:109EE00079E041E021E00E94002D4091A6095091C7
:109EF000A7096091A8097091A9094093AF075093F1
:109F0000B0076093B1077093B2078BED96E00E94A3
:109F1000B77F1AC085E79AE09093F7078093F6071A
:109F20000E9454478FE492E0EDEFF7E0DF019C01DF
:109F30001D9221503040E1F78BE39AE061E77AE02F
:109F40004FE050E00E941B23C05BDF4F0FB6F89438
:109F5000DEBF0FBECDBFCF91DF911F910F91FF905C
:109F6000EF90DF90CF90BF90AF9008952F923F92E7
:109F70004F925F926F927F928F929F92AF92BF9219
:109F8000CF92DF92EF92FF920F931F93DF93CF93C5
:109F9000CDB7DEB7EE970FB6F894DEBF0FBECDBFDC
:109FA00087E40E942042882309F42FC20E944F4474
:109FB0000E943FD66430710509F441C065307105D7
:109FC00054F46230710541F1633071056CF577230B
:109FD000CCF40C9496646A35710509F4BBC16B35F9
:109FE000710534F46C31710511F00C9496646FC0F6
:109FF0006B35710509F4B2C16C35710511F00C9423
:10A000009664B1C18091F807882331F40E94D94445
:10A010000E9430410C94A4648091F807882321F4B5
:10A020000E945A4581E007C08091F807882339F4DF
:10A030000E945A4580E00E9472400C94A46487EE0E
:10A0400097E00E94C0BF80E50E942042882321F44F
:10A05000EE24FF24870106C00E944F440E9444D68C
:10A060007B018C0183E50E942042882361F00E94DD
:10A070004F4420E030E04AE754E40E94B0D80E9408
:10A0800044D67B018C010E948B900E9404CF5B011F
:10A090006C01AE0CBF1CC01ED11E0E9404CF609389
:10A0A000590A70935A0A80935B0A90935C0A06C01F
:10A0B0000E94759C0E940E400E9405C00E9404CF21
:10A0C0006A157B058C059D0598F30C949664809128
:10A0D0009E0390919F03A091A003B091A103809350
:10A0E000880A9093890AA0938A0AB0938B0A809178
:10A0F0007203909173039093BF078093BE0784E629
:10A1000090E090937303809372030E9404CF609356
:10A11000590A70935A0A80935B0A90935C0A81E013
:10A120000E94B08F8091C0079091C107A091C20793
:10A13000B091C30780936D0A90936E0AA0936F0A43
:10A14000B093700A8091C4079091C507A091C6078B
:10A15000B091C7078093710A9093720AA093730A13
:10A16000B093740A8091C8079091C907A091CA075B
:10A17000B091CB078093750A9093760AA093770AE3
:10A18000B093780A8091CC079091CD07A091CE072B
:10A19000B091CF078093790A90937A0AA0937B0AB3
:10A1A000B0937C0A80E090E0A0E0B0E080939E0352
:10A1B00090939F03A093A003B093A10388E50E940E
:10A1C0002042882361F489E50E942042882339F4E3
:10A1D0008AE50E942042882311F481E001C080E0DA
:10A1E0008093A203882329F488E50E9420428823D3
:10A1F00021F080E090E00E9455428091A2038823E4
:10A2000029F489E50E942042882321F081E090E032
:10A210000E94554288E50E9420428823D9F00E947E
:10A2200043446115710581059105A1F00E944F44D9
:10A230002091D0073091D1074091D2075091D30798
:10A240000E94F7D46093C0077093C1078093C20740
:10A250009093C30789E50E9420428823D9F00E9489
:10A2600043446115710581059105A1F00E944F4499
:10A270002091D4073091D5074091D6075091D70748
:10A280000E94F7D46093C4077093C5078093C607F4
:10A290009093C7078091A203882329F48AE50E943E
:10A2A0002042882321F082E090E00E9455428AE516
:10A2B0000E9420428823D9F00E9443446115710511
:10A2C00081059105A1F00E944F442091D80730915B
:10A2D000D9074091DA075091DB070E94F7D46093C9
:10A2E000C8077093C9078093CA079093CB0780EC87
:10A2F00097E064EC77E048EC57E02CEC37E00E9404
:10A30000ED6B80E00E94B08F8091880A9091890A5D
:10A31000A0918A0AB0918B0A80939E0390939F0329
:10A32000A093A003B093A1038091BE079091BF07B3
:10A3300090937303809372030E9404CF6093590A31
:10A3400070935A0A80935B0A90935C0A0E94A98FCB
:10A350000C94966410927D0A0C94966481E080932C
:10A360007D0A0C94966485E40E942042882311F4AF
:10A370000E948B9050ECE52E57E0F52E40EDC42E58
:10A3800047E0D42E00E010E0BB24B394F801EF5D69
:10A39000FB4F80810E942042882351F1033061F4F9
:10A3A0000E944F44F70160837183828393838CEC16
:10A3B00097E00E94CF6B1CC0023011F4B092EA0704
:10A3C0000E944F44F60120813181428153810E94D5
:10A3D000F7D4F701608371838283938380EC97E0E5
:10A3E00064EC77E048EC57E02CEC37E00E94ED6B32
:10A3F0000F5F1F4F24E030E0E20EF31EC20ED31EAB
:10A400000430110519F60C9496648DE40E942042E4
:10A41000882311F40C94B8630E944F440E943FD6E5
:10A420006237710511F40C94D15B633771050CF040
:10A430009BC06E31710509F492C26F3171050CF049
:10A4400042C06631710509F4ECC167317105E4F46D
:10A450006131710509F4A3C16231710534F46230D0
:10A46000710510F00C9496643BC16431710509F4D8
:10A47000A0C1653171050CF0CCC16231710511F0DC
:10A480000C9496640C94BA5A6931710509F4FFC1B1
:10A490006A31710554F46731710509F4C8C1683136
:10A4A000710511F00C949664DEC16B31710509F4ED
:10A4B00013C26B3171050CF4F0C16C31710511F0F0
:10A4C0000C9496640FC26435710511F40C94BA5A59
:10A4D0006535710514F56A32710509F4E0C36B3214
:10A4E000710554F46F31710509F42AC360327105A6
:10A4F00011F00C94966479C26235710511F40C94D4
:10A50000B15A6335710514F00C94B55A6135710573
:10A5100011F00C9496640C94965A6936710509F4FE
:10A5200039C46A36710584F46C35710511F40C94E4
:10A53000245B6836710509F4FCC36535710511F0BB
:10A540000C9496640C940D5B6B36710511F40C94AD
:10A55000905A6B36710514F40C945F5A6D36710580
:10A5600011F00C9496643AC56C3D710511F40C948D
:10A57000BB5E6D3D71050CF04FC06E3B710509F47B
:10A580008BC66F3B71051CF56737710509F4A4C0D4
:10A590006837710564F46337710511F40C94AA5B94
:10A5A0006537710511F00C9496640C94BA5B6937A9
:10A5B000710511F40C94CB5C6937710514F40C949B
:10A5C000C65C6C38710511F00C949664D2C36B3C78
:10A5D000710511F40C94015E6C3C710564F4683CE7
:10A5E000710511F40C94575D693C710511F00C94E0
:10A5F00096640C94DF5D6D3C710511F40C943F5E24
:10A600006D3C710514F40C941F5E6E3C710511F0E5
:10A610000C9496640C949D5E31E06F32730711F4D4
:10A620000C94296141E0603374073CF56A3F710581
:10A6300011F40C94EE606B3F710564F46D3D71058F
:10A6400011F40C94CA5E623E710511F00C9496648C
:10A650000C94D95E51E06C32750711F40C94DF5FF5
:10A6600081E06D32780711F40C94166068517140E6
:10A6700011F00C9496640C94315FE1E0673F7E0723
:10A6800011F40C947461F1E0683F7F079CF421E0C1
:10A69000653F720711F40C946C6131E0663F7307FB
:10A6A00014F00C9471616059714011F00C9496642F
:10A6B0000C94696153E0603A750709F406C283E0BF
:10A6C000673E780711F40C94A1636855724011F04D
:10A6D0000C9496640C947761E9E4F2E00C94D75CF6
:10A6E00086ED97E00E94C0BF80E50E94204288234B
:10A6F00021F4EE24FF24870106C00E944F440E94EB
:10A7000044D67B018C0183E50E942042882361F0BE
:10A710000E944F4420E030E04AE754E40E94B0D861
:10A720000E9444D67B018C010E948B900E9404CF32
:10A730006093590A70935A0A80935B0A90935C0A5B
:10A74000E114F1040105110501F10E9404CF5B0140
:10A750006C01AE0CBF1CC01ED11E0E9404CF6A1536
:10A760007B058C059D05A8F40E94D0A2882389F45E
:10A770000E94759C0E940E400E9405C0EECF0E9470
:10A78000759C0E940E400E9405C00E94D0A28823A2
:10A79000B1F387EC97E00E94C0BF0C9496648EEBF7
:10A7A00097E00E94C0BF5E985E9815985E980C94E2
:10A7B0009664EEEAF7E0949108C08091C00085FFAE
:10A7C000FCCF9093C600319694919923B1F7809174
:10A7D000C00085FFFCCF8AE08093C6008DE095E045
:10A7E0000E941336E0EAF7E0949108C08091C0001F
:10A7F00085FFFCCF9093C600319694919923B1F7D1
:10A800008091C00085FFFCCF8AE08093C6000C9445
:10A8100096648DE095E00E9464310E94174C0C9480
:10A8200096648DE095E00E946F280C949664809168
:10A830008C0A90918D0A04966AE270E00E9465236A
:10A84000FC01009711F03197108260918C0A709191
:10A850008D0A6C5F7F4F8DE095E041E021E00E9422
:10A86000002D0C9496648DE095E00E94842C8DE080
:10A8700095E00E9473280E9404CF6093EE077093C6
:10A88000EF078093F0079093F1070C9496648DE0A6
:10A8900095E00E947A280C94966480911005882394
:10A8A00011F40C94966483E50E942042882311F4ED
:10A8B0000C9496640E944344AB01BC014093AF07E3
:10A8C0005093B0078093B1077093B2078BED96E079
:10A8D0000E94B77F0C9496648DE095E00E94B82AA0
:10A8E0000C94966480918C0A90918D0A04966AE289
:10A8F00070E00E9465238C01009719F12091820A73
:10A900003091830A80E690E0FC012E9FC0012F9FCA
:10A91000900D3E9F900D11248257954F6EE470E08C
:10A920000E94652360E270E00E9465239C012F5F16
:10A930003F4F30938D0A20938C0A01501040F8014C
:10A94000108260918C0A70918D0A6C5F7F4F8DE050
:10A9500095E040E021E00E94002D0C9496648091E7
:10A960001005882311F40C9496648DE095E060E066
:10A970000E94272A80918C0A90918D0A04966AE29F
:10A9800070E00E9465238C01009719F12091820AE2
:10A990003091830A80E690E0AC01249FC001259F9E
:10A9A000900D349F900D11248257954F6EE470E006
:10A9B0000E94652360E270E00E9465239C012F5F86
:10A9C0003F4F30938D0A20938C0A01501040F801BC
:10A9D000108260918C0A70918D0A6C5F7F4F8DE0C0
:10A9E00095E00E94122B0C94966480910F058823A9
:10A9F00011F00E948B90E0908C0AF0908D0A24E078
:10AA000030E0E20EF31EC7016AE270E00E946523A7
:10AA10008C01C70161E270E00E946523009721F07C
:10AA20007C010894E11CF11C0115110521F0015075
:10AA30001040F801108280E50E942042182F80917A
:10AA40008C0A90918D0AE816F90608F410E08091BE
:10AA50001005882311F40C94966421E021278DE0E1
:10AA600095E0B70141E00E94002D83E50E9420425D
:10AA70008823B9F080918C0A90918D0A8E159F05DC
:10AA800080F40E944344AB01BC014093AF07509354
:10AA9000B0078093B1077093B2078BED96E00E94E8
:10AAA000B77F8DE095E00E947328112311F00C947C
:10AAB00096640E9404CF6093EE077093EF07809333
:10AAC000F0079093F1070C94966480918C0A909112
:10AAD0008D0A05966AE270E00E9465238C0100975A
:10AAE00019F12091820A3091830A80E690E0AC014E
:10AAF000249FC001259F900D349F900D11248257F3
:10AB0000954F6EE470E00E94652360E270E00E9461
:10AB100065239C012F5F3F4F30938D0A20938C0A51
:10AB200001501040F801108260918C0A70918D0ADA
:10AB30006B5F7F4F8DE095E00E9486300C949664A9
:10AB40000E9404CF6093F2077093F3078093F40799
:10AB50009093F5072091EE073091EF074091F007B1
:10AB60005091F107621B730B840B950B28EE33E0B9
:10AB700040E050E00E94C8D9F22EE32ED42EC52E1C
:10AB80002DB73EB7285030400FB6F8943EBF0FBEE9
:10AB90002DBF0DB71EB70F5F1F4FCE018196EDB7CA
:10ABA000FEB79283818381E997E0F80193838283E2
:10ABB0006F2D7E2D842F952F2CE330E040E050E068
:10ABC0000E94C8D9F801358324836F2D7E2D8D2DE9
:10ABD0009C2D2CE330E040E050E00E94C8D9F80101
:10ABE000778366830E949423E7E1F5E094912DB783
:10ABF0003EB7285F3F4F0FB6F8943EBF0FBE2DBF44
:10AC000008C08091C00085FFFCCF9093C6003196AC
:10AC100094919923B1F7FE01B19607C08091C000CD
:10AC200085FFFCCF31969093C60090819923B1F7B0
:10AC30008091C00085FFFCCF8AE08093C600CE01E2
:10AC400081960E94E3BF8091ED0F882311F40C944C
:10AC500096641092ED0F8091EB07082F10E0000F23
:10AC6000111F0D5A184EF80160817181882777FDF8
:10AC70008095982F0E9472D62091A7033091A80347
:10AC80004091A9035091AA030E94DED7181614F030
:10AC90000C949664F801118210820C94966483E5FA
:10ACA0000E942042882311F40C9496640E944F4421
:10ACB0000E943FD67B018C016B0180E50E942042FF
:10ACC000882369F0F7FC0BC0FFEFEF16F10409F0E1
:10ACD00034F40E944F440E943FD68B0102C00FEF14
:10ACE0001FEFE5E2F4E0808191818017910711F474
:10ACF0000C949664329624E0E539F207A1F704300B
:10AD0000110529F4D092ED07C092EC0704C017FF9B
:10AD100002C00C949664802F61E00E9431D0802F95
:10AD20006C2D0E94AED0802FB6010E94B3CF0C9440
:10AD3000966488E690E00E945944882311F00C94B0
:10AD4000966483E50E942042882379F00E944F4454
:10AD50002091500A022F10E0000F111F0D5A184EBB
:10AD60000E943FD6F801718360830E946A980C9418
:10AD7000966483E50E942042882311F40C94966423
:10AD80000E944F440E943FD6709356176093551708
:10AD90000C94966489E690E00E945944882311F04F
:10ADA0000C949664EBE8F7E0949108C08091C000A1
:10ADB00085FFFCCF9093C600319694919923B1F70B
:10ADC000E091500AF0E0EE0FFF1FEE0FFF1FE75A71
:10ADD000F84E40815181628173818CE095E021E0E1
:10ADE00030E00E945F3EE8E8F7E0949108C080916F
:10ADF000C00085FFFCCF9093C600319694919923B3
:10AE0000B1F7E091500AF0E0EE0FFF1FED5AF84E57
:10AE100060817181882777FD8095982F0E9472D676
:10AE2000AB01BC018CE095E021E030E00E945F3E88
:10AE3000E4E8F7E0949108C08091C00085FFFCCF62
:10AE40009093C600319694919923B1F740915F1782
:10AE50005091601760916117709162178CE095E0D6
:10AE600021E030E00E945F3EE1E8F7E0949108C005
:10AE70008091C00085FFFCCF9093C60031969491DD
:10AE80009923B1F76091551770915617882777FD70
:10AE90008095982F0E9472D6AB01BC018CE095E0A2
:10AEA00021E030E00E945F3EEEE7F7E0949108C0B9
:10AEB0008091C00085FFFCCF9093C600319694919D
:10AEC0009923B1F78CE095E060E070E04AE050E053
:10AED0000E94843DECE7F7E0949108C08091C000A7
:10AEE00085FFFCCF9093C600319694919923B1F7DA
:10AEF0004091591750915A1760915B1770915C17E8
:10AF00008CE095E021E030E00E945F3EE9E7F7E069
:10AF1000949108C08091C00085FFFCCF9093C6003B
:10AF2000319694919923B1F760915317709154170A
:10AF3000882777FD8095982F0E9472D6AB01BC01BF
:10AF40008CE095E021E030E00E945F3EE5E7F7E02D
:10AF5000949108C08091C00085FFFCCF9093C600FB
:10AF6000319694919923B1F78091500A0E94AF973E
:10AF7000BC018CE095E04AE050E00E94843DE0E7AF
:10AF8000F7E0949108C08091C00085FFFCCF9093BA
:10AF9000C600319694919923B1F78FEF9FEF0E94ED
:10AFA000AF97BC018CE095E04AE050E00E94843D00
:10AFB000E2E6F2E007C08091C00085FFFCCF319649
:10AFC0009093C60090819923B1F78091C00085FFCE
:10AFD000FCCF8AE08093C6000C94A4648DE690E0D8
:10AFE0000E945944882311F00C94966485E697E0FA
:10AFF0000E94C0BF1092ED0F83E50E94204288237B
:10B0000099F00E944F442091500A022F10E0000F47
:10B01000111F0D5A184E0E943FD6F80171836083AC
:10B0200081E08093990316C082E50E942042882324
:10B0300089F00E944F442091500A022F10E0000F27
:10B04000111F0D5A184E0E943FD6F801718360837C
:10B050001092990383E50E942042882351F00E94B8
:10B060004F446093A7037093A8038093A903909320
:10B07000AA0382E40E942042882351F00E944F4498
:10B080006093A3037093A4038093A5039093A603F6
:10B0900086E40E942042882369F00E944F44609316
:10B0A000AB037093AC038093AD039093AE0381E048
:10B0B0008093ED0F0E946A980E9404CF6B017C017F
:10B0C0002091500A022F10E01092FC07000F111F70
:10B0D000F801ED5AF84E60817181882777FD8095DF
:10B0E000982F0E9472D6000F111F075A184EF801B0
:10B0F00020813181428153810E94DED718160CF0E5
:10B1000066C081E08093FC0762C00E9404CF6C1986
:10B110007D098E099F09695E73408040904008F464
:10B120004FC09A2DE2E6F7E008C08091C00085FF8D
:10B13000FCCF9093C600319694919923B1F7E0919A
:10B14000500AF0E0EE0FFF1FEE0FFF1FE75AF84E18
:10B1500040815181628173818CE095E021E030E093
:10B160000E945F3E9B2DEEE5F7E008C08091C00095
:10B1700085FFFCCF9093C600319694919923B1F747
:10B180006091500A8CE095E070E04AE050E00E9447
:10B19000843DE2E6F2E007C08091C00085FFFCCF6D
:10B1A00031969093C60090819923B1F78091C000A9
:10B1B00085FFFCCF9092C6000E9404CF6B017C01FA
:10B1C0000E94759C0E940E400E9405C008C0E2E6E5
:10B1D000F7E0A490EEE5F7E0B4906AE0962E809157
:10B1E000FC070091500A8823E9F010E0000F111FBE
:10B1F000F801ED5AF84E60817181882777FD8095BE
:10B20000982F0E9472D6000F111F075A184EF8018E
:10B2100020813181428153810E94DED718160CF4BF
:10B2200074CF20C010E0000F111FF801ED5AF84E46
:10B2300060817181882777FD8095982F0E9472D652
:10B24000000F111F075A184EF801208131814281E9
:10B2500053810E94D0D588232CF4809199038823B0
:10B2600009F453CF80E597E00E94C0BF0E9404CF4D
:10B270006093EE077093EF078093F0079093F107C8
:10B280000E9404CF6093590A70935A0A80935B0A14
:10B2900090935C0A0C94966483E497E00E94C0BF8C
:10B2A00083E50E942042882361F00E944F440E945F
:10B2B0003FD6709356176093551781E0809399039A
:10B2C0000FC082E50E942042882351F00E944F4423
:10B2D0000E943FD6709356176093551710929903AA
:10B2E0000E9404CF7B018C011092FC0760915517DE
:10B2F00070915617882777FD8095982F0E9472D6F7
:10B3000020915F173091601740916117509162173B
:10B310000E94DED718160CF082C081E08093FC07F3
:10B320007EC00E9404CF6E197F09800B910B695E6D
:10B3300073408040904008F46BC0E091EB07F0E070
:10B34000EE0FFF1FEE0FFF1FE75AF84E40815181AD
:10B35000628173819B2DE0E4F7E008C08091C0001A
:10B3600085FFFCCF9093C600319694919923B1F755
:10B370008CE095E022E030E00E945F3E9C2DECE303
:10B38000F7E008C08091C00085FFFCCF9093C60015
:10B39000319694919923B1F76091EB078CE095E099
:10B3A00070E04AE050E00E94843D9D2DE8E3F7E024
:10B3B00008C08091C00085FFFCCF9093C6003196F5
:10B3C00094919923B1F740915F1750916017609164
:10B3D0006117709162178CE095E021E030E00E94E7
:10B3E0005F3EE2E6F2E007C08091C00085FFFCCF3F
:10B3F00031969093C60090819923B1F78091C00057
:10B4000085FFFCCFA092C6000E9404CF7B018C0177
:10B410000E94759C0E940E400E9405C00BC0E0E493
:10B42000F7E0B490ECE3F7E0C490E8E3F7E0D49001
:10B43000AAE0AA2E8091FC0720915517309156174B
:10B440008823A9F0B901882777FD8095982F0E945D
:10B4500072D620915F17309160174091611750911B
:10B4600062170E94DED718160CF45BCF18C0B90122
:10B47000882777FD8095982F0E9472D620915F17BC
:10B480003091601740916117509162170E94D0D59A
:10B4900088232CF480919903882309F442CF8EE20B
:10B4A00097E00E94C0BF0E9404CF6093590A709336
:10B4B0005A0A80935B0A90935C0A0C94966483E525
:10B4C0000E942042882321F10E944F4420E030E076
:10B4D00040E050E00E94D0D588231CF460E070E08A
:10B4E00011C00E944F4420E030E04FE753E40E9437
:10B4F000DED718161CF46FEF70E004C00E944F44B2
:10B500000E943FD67093ED076093EC070C9496640D
:10B510008FEF90E09093ED078093EC070C94966486
:10B520001092ED071092EC070C9496640E946B98B1
:10B530000E948B905E9A0E9499901092ED07109253
:10B54000EC0768EE73E080E090E00E9412CF10926A
:10B55000980387E197E00E94C0BF0E9405C00C9449
:10B5600096641092BD070C94966481E08093BD07A9
:10B570000C94966483E50E9420428823A1F00E94E7
:10B580004F4420E030E04AE754E40E94B0D80E94E3
:10B5900044D660939A0370939B0380939C0390938B
:10B5A0009D030C94966488E50E942042882311F044
:10B5B0000C94996489E50E942042882311F00C9430
:10B5C00099648AE50E942042882311F00C949964C2
:10B5D00085E40E942042882311F00C9499640E9413
:10B5E0008B905E9A0E9499900C9496645E9A109249
:10B5F000E80789E50E942042882319F05E9A10929C
:10B60000E9078AE50E942042882311F40C9496648D
:10B61000159A1092EA070C94966483E50E942042E2
:10B620000E944F4420E030E04AE754E40E94B0D842
:10B630000E9444D660935D0A70935E0A80935F0A0D
:10B640009093600A0C949664F1E96F2EFFE07F2ED0
:10B65000E1E82E2EEFE03E2E7DEC472E7FE0572EC8
:10B6600088249924F401EF5DFB4F80810E942042E1
:10B67000882309F45DC023E0821609F052C00E94BD
:10B680004F445B016C0120E030E040EA51E40E944D
:10B69000D0D588230CF03FC0F30160817181828195
:10B6A0009381A60195010E94D7D57B018C01609101
:10B6B000C50F7091C60F8091C70F9091C80FA80158
:10B6C00097010E94B0D86093C50F7093C60F809306
:10B6D000C70F9093C80FF1016081718182819381BE
:10B6E000A80197010E94B0D8F10160837183828321
:10B6F0009383F20160817181828193810E9470D66F
:10B70000A80197010E94B0D80E9444D6F20160833C
:10B71000718382839383F301A082B182C282D38238
:10B7200007C00E944F44F301608371838283938337
:10B730000894811C911C24E030E0620E731E220EDE
:10B74000331E420E531E34E08316910409F08ACF53
:10B750000C949664E7E4F6E0949108C08091C000F0
:10B7600085FFFCCF9093C600319694919923B1F751
:10B770000C94966480918C0A90918D0A05966AE2E9
:10B7800070E00E946523FC01009711F03197108250
:10B7900080918C0A90918D0A05960E94E3BF0C94CB
:10B7A0009664E4E4F6E0949108C08091C00085FFBF
:10B7B000FCCF9093C600319694919923B1F74091B4
:10B7C000C0075091C1076091C2077091C3078CE018
:10B7D00095E022E030E00E945F3EE1E4F6E09491E3
:10B7E00008C08091C00085FFFCCF9093C6003196C1
:10B7F00094919923B1F74091C4075091C507609186
:10B80000C6077091C7078CE095E022E030E00E9407
:10B810005F3EEEE3F6E0949108C08091C00085FFA2
:10B82000FCCF9093C600319694919923B1F7409143
:10B83000C8075091C9076091CA077091CB078CE087
:10B8400095E022E030E00E945F3EEBE3F6E0949169
:10B8500008C08091C00085FFFCCF9093C600319650
:10B8600094919923B1F74091CC075091CD07609105
:10B87000CE077091CF078CE095E022E030E00E9487
:10B880005F3EE0E3F6E0949108C08091C00085FF40
:10B89000FCCF9093C600319694919923B1F780E044
:10B8A0000E9456900E9472D62091910F3091920F73
:10B8B0004091930F5091940F0E94D7D5AB01BC01DA
:10B8C0008CE095E022E030E00E945F3EEDE2F6E0A1
:10B8D000949108C08091C00085FFFCCF9093C60072
:10B8E000319694919923B1F781E00E9456900E947D
:10B8F00072D62091950F3091960F4091970F5091ED
:10B90000980F0E94D7D5AB01BC018CE095E022E0F6
:10B9100030E00E945F3EEAE2F6E0949108C0809138
:10B92000C00085FFFCCF9093C60031969491992377
:10B93000B1F782E00E9456900E9472D62091990F32
:10B9400030919A0F40919B0F50919C0F0E94D7D538
:10B95000AB01BC018CE095E022E030E00E945F3E4C
:10B96000E2E6F2E007C08091C00085FFFCCF31968F
:10B970009093C60090819923B1F78091C00085FF14
:10B98000FCCF8AE08093C6000C94966480E00E940D
:10B99000B08F0C94966481E00E94B08F0C949664F2
:10B9A0008091C00085FFFCCF31969093C6009081B6
:10B9B0009923B1F78091C00085FFFCCF8AE0809386
:10B9C000C600E2E2F6E0949108C08091C00085FFD5
:10B9D000FCCF9093C600319694919923B1F7329998
:10B9E00003C0E3E6F2E00AC0E8E6F2E007C08091B7
:10B9F000C00085FFFCCF31969093C60090819923BB
:10BA0000B1F78091C00085FFFCCF8AE08093C6002B
:10BA1000EAE1F6E0949108C08091C00085FFFCCF78
:10BA20009093C600319694919923B1F7339903C04E
:10BA3000E3E6F2E00AC0E8E6F2E007C08091C00069
:10BA400085FFFCCF31969093C60090819923B1F782
:10BA50008091C00085FFFCCF8AE08093C600E2E1C0
:10BA6000F6E0949108C08091C00085FFFCCF9093D0
:10BA7000C600319694919923B1F7349903C0E3E657
:10BA8000F2E00AC0E8E6F2E007C08091C00085FF5E
:10BA9000FCCF31969093C60090819923B1F78091A5
:10BAA000C00085FFFCCF8AE08093C6003FC784E4D6
:10BAB0000E942042882309F439C70E944F4420E0A5
:10BAC00030E040E05FE30E94B0D87B018C0120E0D1
:10BAD00030E040E050E00E94D0D5882359F40F2E8A
:10BAE000F0E0CF2EF0E0DF2EF0E8EF2EFFE3FF2EA8
:10BAF000F02D11C0C801B701A80197010E94B0D86C
:10BB00009B01AC01CA012BED3FE049E450E40E94E7
:10BB1000B0D86B017C018091EB078093500A84E5DB
:10BB20000E942042882399F10E944F440E9444D6EB
:10BB3000262F6093500A6623D9F0E7E1F5E094914F
:10BB400008C08091C00085FFFCCF9093C60031965D
:10BB500094919923B1F7E2E7F2E007C08091C00029
:10BB600085FFFCCF31969093C60090819923B1F761
:10BB70008CE095E0622F40E050E00E943D3D8091D6
:10BB8000C00085FFFCCF8AE08093C600CFC68091BD
:10BB9000500A082F10E0000F111F000F111F0A5844
:10BBA0001C4F60E070E080E89FE3A70196010E94CF
:10BBB000D7D5F8016083718382839383B7C601E28E
:10BBC00014E051EAE52E5FE0F52EF80180810E9435
:10BBD0002042882349F00E944F440E9444D6F70136
:10BBE00060837183828393830F5F1F4F24E030E073
:10BBF000E20EF31E34E00532130739F70E94A46BFE
:10BC000095C601E214E041E8E42E4FE0F42EF8017D
:10BC100080810E942042882339F00E944F44F7011E
:10BC200060837183828393830F5F1F4F24E030E032
:10BC3000E20EF31E34E00532130749F777C683E5B9
:10BC40000E942042882351F00E944F446093B50F18
:10BC50007093B60F8093B70F9093B80F84E50E944E
:10BC60002042882309F462C60E944F446093B90FB2
:10BC70007093BA0F8093BB0F9093BC0F57C683E5A8
:10BC80000E942042882351F00E944F446093B10FDC
:10BC90007093B20F8093B30F9093B40F84E50E941A
:10BCA0002042882351F00E944F446093C90F709343
:10BCB000CA0F8093CB0F9093CC0F82E40E94204256
:10BCC000882361F00E944F440E9444D660937D0F08
:10BCD00070937E0F80937F0F9093800F88E50E9472
:10BCE0002042882351F00E944F446093BD0F70930F
:10BCF000BE0F8093BF0F9093C00F8AE50E94204231
:10BD0000882351F00E944F446093C10F7093C20F7B
:10BD10008093C30F9093C40F85E40E942042882330
:10BD200009F404C60E944F446093C50F7093C60F78
:10BD30008093C70F9093C80FF9C501E214E030ED6E
:10BD4000E32E37E0F32EF80180810E942042882301
:10BD500039F00E944F44F70160837183828393839B
:10BD60000F5F1F4F24E030E0E20EF31E34E0043298
:10BD7000130749F7DBC583E50E942042882309F4B5
:10BD8000D5C50E944F440E943FD6709373036093C1
:10BD90007203CCC583E50E942042882309F4C6C5FE
:10BDA0000E944F440E943FD67093750360937403C2
:10BDB000BDC580E50E942042882309F4B7C50E94D2
:10BDC0004F440E943FD67B0183E50E942042882396
:10BDD00019F40FEF1FEF05C00E944F440E943FD699
:10BDE0008B01C8010196039708F0A0C5E5E2F4E0D5
:10BDF000808191818E159F0509F498C5329644E0A3
:10BE0000E539F407A9F7F7FC91C50E948B90DE2C69
:10BE10008E2D60E00E9431D00115110541F00130F6
:10BE2000110579F05FEF0F3F1507A1F403C000E0A3
:10BE300010E010C08E2D0E94E1D000E010E0892BB0
:10BE400049F401E010E006C00E94759C0E940E407B
:10BE50000E9405C08D2D0E94E1D080179107A1F7A7
:10BE600065C580E50E942042882319F40FEF1FEF7B
:10BE700005C00E944F440E943FD68B0183E50E947B
:10BE80002042882309F446C00E944F440115110541
:10BE900051F40E943FD69B01AC0189EF97E0B901B4
:10BEA0000E947F8E43C5E7E1F5E0949108C0809140
:10BEB000C00085FFFCCF9093C600319694919923E2
:10BEC000B1F7E9E8F2E007C08091C00085FFFCCF40
:10BED00031969093C60090819923B1F78CE095E05C
:10BEE000B8014AE050E00E94843DE0E9F2E007C07A
:10BEF0008091C00085FFFCCF31969093C600908161
:10BF00009923B1F78091C00085FFFCCF8AE0809330
:10BF1000C6000CC517FD0AC5EEE9F2E007C0809126
:10BF2000C00085FFFCCF31969093C6009081992385
:10BF3000B1F7E1EAF2E007C08091C00085FFFCCFD5
:10BF400031969093C60090819923B1F78CE095E0EB
:10BF5000B8014AE050E00E94843DE9EAF2E007C0FF
:10BF60008091C00085FFFCCF31969093C6009081F0
:10BF70009923B1F7C801880F991F800F911F87502F
:10BF8000984F0E942A8EBC018CE095E04AE050E078
:10BF90000E94843DE2E6F2E007C08091C00085FF88
:10BFA000FCCF31969093C60090819923B1F7809190
:10BFB000C00085FFFCCF8AE08093C600B7C483E54C
:10BFC0000E942042882321F4BEE6CB2ED12C05C04E
:10BFD0000E944F440E943FD66B0180E50E942042A0
:10BFE000882319F468EE73E004C00E944F440E9455
:10BFF0003FD67B010027F7FC0095102F1C141D0471
:10C0000084F48BE1B60120E030E040E050E00E9493
:10C0100006D2C801B7010E9412CF8BE10E948FD1D6
:10C0200085C4C801B7010E9412CF80C480E50E9478
:10C030002042882351F00E944F446093B4037093D0
:10C04000B5038093B6039093B70389E40E9420421E
:10C05000882361F00E944F440E947A986093B8034D
:10C060007093B9038093BA039093BB0384E40E9456
:10C070002042882361F00E944F440E948898609378
:10C08000BC037093BD038093BE039093BF0383E40E
:10C090000E942042882351F00E944F446093C003C5
:10C0A0007093C1038093C2039093C3030E94989737
:10C0B000EEE9F2E007C08091C00085FFFCCF319629
:10C0C0009093C60090819923B1F7ECEAF2E007C0A3
:10C0D0008091C00085FFFCCF31969093C60090817F
:10C0E0009923B1F74091B4035091B5036091B60321
:10C0F0007091B7038CE095E022E030E00E945F3E53
:10C10000E0EBF2E007C08091C00085FFFCCF3196E4
:10C110009093C60090819923B1F76091B803709114
:10C12000B9038091BA039091BB030E948198AB013F
:10C13000BC018CE095E022E030E00E945F3EE4EB41
:10C14000F2E007C08091C00085FFFCCF319690934C
:10C15000C60090819923B1F76091BC037091BD0333
:10C160008091BE039091BF030E948F98AB01BC01E8
:10C170008CE095E022E030E00E945F3EE8EBF2E0E8
:10C1800007C08091C00085FFFCCF31969093C60018
:10C1900090819923B1F74091C0035091C103609100
:10C1A000C2037091C3038CE095E022E030E00E946E
:10C1B0005F3EE2E6F2E007C08091C00085FFFCCF61
:10C1C00031969093C60090819923B1F78091C00079
:10C1D00085FFFCCF8AE08093C600A8C383E40E9459
:10C1E0002042882349F00E944F440E943FD6DC0140
:10C1F000CB018F730E94B3BFEDEFF5E0949108C0BF
:10C200008091C00085FFFCCF9093C6003196949139
:10C210009923B1F76091B2197091B3198CE095E050
:10C220004AE050E00E94843DE2E6F2E007C08091DF
:10C23000C00085FFFCCF31969093C6009081992372
:10C24000B1F78091C00085FFFCCF8AE08093C600E3
:10C250006DC385E40E942042882319F4CC24DD2498
:10C2600012C00E944F440E943FD66B0177FF0BC063
:10C270000F2EF0E0EF2EF0E0FF2EFCE80F2FF2E49F
:10C280001F2FF02D0AC00F2EF0E0EF2EF0E0FF2E52
:10C29000F6E10F2FF3E41F2FF02D83E50E942042DB
:10C2A000882321F00E944F447B018C0183E40E948B
:10C2B0002042882319F425E030E005C00E944F4455
:10C2C0000E943FD69B01C801B701A6010E944A9E69
:10C2D0002DC30E948B902AC30E940D370E94BA384A
:10C2E00025C30E940D3722C30E94BA381FC3A090F5
:10C2F000C007B090C107C090C207D090C307A98201
:10C30000BA82CB82DC82E090C407F090C50700912E
:10C31000C6071091C707ED82FE820F831887209110
:10C32000C8073091C9074091CA075091CB072987A8
:10C330003A874B875C878091CC079091CD07A0917D
:10C34000CE07B091CF078D879E87AF87B88BA98A1C
:10C35000BA8ACB8ADC8AED8AFE8A0F8B188F298FE6
:10C360003A8F4B8F5C8F8D8F9E8FAF8FB8A385E4F4
:10C370000E942042882369F0ED84FE840F8518898D
:10C380000E944F449B01AC01C801B7010E94F7D441
:10C390000AC06D857E858F85988920E030E040E079
:10C3A00050E40E94F6D46D877E878F87988B6091CA
:10C3B0009E0370919F038091A0039091A10320E0C0
:10C3C00030E040E752E40E94D7D57B018C01CE01DA
:10C3D0000196BE016B5F7F4FAE01475F5F4F9E01CD
:10C3E000235F3F4FABEECA2EA7E0DA2E0E94FD700E
:10C3F0008AE50E942042882359F0E984FA840B855B
:10C400001C850E944F449B01AC01C801B70108C0C4
:10C4100069857A858B859C8520E030E040E251E497
:10C420000E94F7D469877A878B879C8760919E03E7
:10C4300070919F038091A0039091A10320E030E0D0
:10C4400040E752E40E94D7D57B018C01CE010196D2
:10C45000BE016B5F7F4FAE01475F5F4F9E01235F61
:10C460003F4FFBEECF2EF7E0DF2E0E94FD7088E5F8
:10C470000E942042882389F0E980FA800B811C8188
:10C480000E944F449B01AC01C801B7010E94F7D440
:10C4900069837A838B839C8308C080E090E0A0E46A
:10C4A000B0E489839A83AB83BC8389E50E942042F0
:10C4B000882339F00E944F446D837E838F83988751
:10C4C00008C080E090E0A0E4B0E48D839E83AF8359
:10C4D000B88760919E0370919F038091A003909113
:10C4E000A10320E030E040E752E40E94D7D57B0171
:10C4F0008C01CE010196BE016B5F7F4FAE01475F9D
:10C500005F4F9E01235F3F4FEBEECE2EE7E0DE2E26
:10C510000E94FD708CE40E942042882369F0ED8423
:10C52000FE840F8518890E944F449B01AC01C8010D
:10C53000B7010E94F7D40AC06D857E858F859889E2
:10C5400020E030E048EC52E40E94F6D46D877E870C
:10C550008F87988B60919E0370919F038091A003B9
:10C560009091A10320E030E040E752E40E94D7D54B
:10C570007B018C01CE010196BE016B5F7F4FAE0146
:10C58000475F5F4F9E01235F3F4FBBEECB2EB7E06F
:10C59000DB2E0E94FD700E948B905E9A64E670E034
:10C5A00080E090E00E9412CF8DEE95E00E94CFBF18
:10C5B00010E018C01F5F0E94759C0E940E400E94F0
:10C5C00005C0112379F40C9A149A63E070E080E0BE
:10C5D00090E00E9412CF149863E070E080E090E059
:10C5E0000E9412CF0E94D0A2882321F38CE40E94E3
:10C5F0002042882369F0ED84FE840F8518890E940B
:10C600004F449B01AC01C801B7010E94F6D40AC097
:10C610006D857E858F85988920E030E048EC52E476
:10C620000E94F7D46D877E878F87988B8D859E8536
:10C63000AF85B8898093CC079093CD07A093CE07A0
:10C64000B093CF078CEC97E00E94CF6BA9E04A2E05
:10C65000512C4C0E5D1EFDE06F2E712C6C0E7D1E5C
:10C6600060919E0370919F038091A0039091A1031C
:10C6700020E030E040E752E40E94D7D57B018C01F6
:10C68000CE010196BE016B5F7F4FA2019301EBEEDD
:10C69000CE2EE7E0DE2E0E94FD7051E1A52EB12CDA
:10C6A000AC0EBD1E45E1842E912C8C0E9D1E60911A
:10C6B0009E0370919F038091A0039091A10320E0BD
:10C6C00030E040E752E40E94D7D57B018C01C501E0
:10C6D000B401A20193010E94FD7039E1432E512C57
:10C6E0004C0E5D1E60919E0370919F038091A0038C
:10C6F0009091A10320E030E040E752E40E94D7D5BA
:10C700007B018C01C501B401A20193010E94FD705F
:10C7100060919E0370919F038091A0039091A1036B
:10C7200020E030E040E752E40E94D7D57B018C0145
:10C73000C501B401A2019E01235E3F4F0E94FD701E
:10C74000F5C01092F8070E94CDA28091550A9091F1
:10C75000560AA091570AB091580A8093510A9093B3
:10C76000520AA093530AB093540A0E94F241DEC0C9
:10C7700084E50E942042882309F48DC00E944F4422
:10C780000E9444D6262F6093500A6623B9F1E7E150
:10C79000F5E0949108C08091C00085FFFCCF909394
:10C7A000C600319694919923B1F7ECEBF2E007C003
:10C7B0008091C00085FFFCCF31969093C600908198
:10C7C0009923B1F78CE095E0622F40E050E00E94A1
:10C7D0003D3DEEEBF2E007C08091C00085FFFCCF4D
:10C7E00031969093C60090819923B1F78091C00053
:10C7F00085FFFCCF8AE08093C60098C086E40E9443
:10C8000020428823E1F00E944F447B018C01609319
:10C810007E0A70937F0A8093800A9093810A20E0B9
:10C8200030E040E050E00E94DED7181644F4E09279
:10C830009E03F0929F030093A0031093A103E7E1EE
:10C84000F5E0949108C08091C00085FFFCCF9093E3
:10C85000C600319694919923B1F7EFECF2E007C04E
:10C860008091C00085FFFCCF31969093C6009081E7
:10C870009923B1F76091EB078CE095E070E04AE016
:10C8800050E00E94843D8091C00085FFFCCF8AE08B
:10C890008093C6004BC0E7E1F5E0949108C0809119
:10C8A000C00085FFFCCF9093C600319694919923E8
:10C8B000B1F7EAEDF5E0949108C08091C00085FFE2
:10C8C000FCCF9093C600319694919923B1F72091B3
:10C8D000820A3091830A80E690E0289FF001299F28
:10C8E000F00D389FF00D1124E257F54F07C08091ED
:10C8F000C00085FFFCCF31969093C60090819923AC
:10C90000B1F7E8EDF5E0949108C08091C00085FF93
:10C91000FCCF9093C600319694919923B1F7809102
:10C92000C00085FFFCCF8AE08093C6000E94E53FEF
:10C930000BC00E948B9088E50E942042882311F052
:10C940000C94F65A0C94F95AEE960FB6F894DEBF92
:10C950000FBECDBFCF91DF911F910F91FF90EF9050
:10C96000DF90CF90BF90AF909F908F907F906F900F
:10C970005F904F903F902F900895CF93DF938091D9
:10C98000180C9091190C039714F40E94E9478DE05C
:10C9900095E060E00E9444328091180C9091190C4F
:10C9A000892B09F46FC080910D05882309F450C0CC
:10C9B0002091820A3091830A80E690E0289FE0016E
:10C9C000299FD00D389FD00D1124C257D54FCE01CD
:10C9D00069E979E00E942A23892BF9F48DE095E03A
:10C9E000BE010E94402A80910E05882319F00E9402
:10C9F000B64F32C0E6E9F9E0949108C08091C000DA
:10CA000085FFFCCF9093C600319694919923B1F79E
:10CA10008091C00085FFFCCF17C08DE095E060E0FD
:10CA20000E94272AE4E8F9E0949108C08091C000B0
:10CA300085FFFCCF9093C600319694919923B1F76E
:10CA40008091C00085FFFCCF8AE08093C60004C0BF
:10CA50000E94B64F0E9495458091180C9091190C38
:10CA600001979093190C8093180C8091820A9091F1
:10CA7000830A019664E070E00E94B5D99093830A1E
:10CA80008093820A0E94759C0E940E400E94EE963E
:10CA90000E9405C0DF91CF910895DF93CF9300D01E
:10CAA000CDB7DEB78CE095E040E052EC61E070E09D
:10CAB0000E94253CEBE6FAE0949108C08091C0000A
:10CAC00085FFFCCF9093C600319694919923B1F7DE
:10CAD0008091C00085FFFCCF8AE08093C60047E1CB
:10CAE00055E0FA01949108C08091C00085FFFCCF09
:10CAF0009093C600319694919923B1F784B7282F6B
:10CB000080FF15C0E3E6FAE0949108C08091C00070
:10CB100085FFFCCF9093C600319694919923B1F78D
:10CB20008091C00085FFFCCF8AE08093C60021FF82
:10CB300015C0E3E5FAE0949108C08091C00085FF3C
:10CB4000FCCF9093C600319694919923B1F78091D0
:10CB5000C00085FFFCCF8AE08093C60022FF15C08D
:10CB6000E2E4FAE0949108C08091C00085FFFCCF18
:10CB70009093C600319694919923B1F78091C000AB
:10CB800085FFFCCF8AE08093C60023FF15C0E2E357
:10CB9000FAE0949108C08091C00085FFFCCF90938B
:10CBA000C600319694919923B1F78091C00085FF1A
:10CBB000FCCF8AE08093C60025FF15C0E2E2FAE0D0
:10CBC000949108C08091C00085FFFCCF9093C6006F
:10CBD000319694919923B1F78091C00085FFFCCFE5
:10CBE0008AE08093C60014BEEAE1FAE0949108C09E
:10CBF0008091C00085FFFCCF9093C6003196949140
:10CC00009923B1F7E4E1FAE0949108C08091C00063
:10CC100085FFFCCF9093C600319694919923B1F78C
:10CC20008091C00085FFFCCF8AE08093C600FA01A6
:10CC30009491E7E1F5E008C08091C00085FFFCCF4A
:10CC40009093C600319694919923B1F7E4E0FAE00D
:10CC5000949108C08091C00085FFFCCF9093C600DE
:10CC6000319694919923B1F7EFEEF9E0949108C0D1
:10CC70008091C00085FFFCCF9093C60031969491BF
:10CC80009923B1F7E3EEF9E0949108C08091C000D8
:10CC900085FFFCCF9093C600319694919923B1F70C
:10CCA000EAEDF9E0949108C08091C00085FFFCCFC7
:10CCB0009093C600319694919923B1F78091C0006A
:10CCC00085FFFCCF8AE08093C600EFECF9E09491F9
:10CCD00008C08091C00085FFFCCF9093C6003196BC
:10CCE00094919923B1F7E3ECF9E0949108C0809115
:10CCF000C00085FFFCCF9093C60031969491992394
:10CD0000B1F78091C00085FFFCCF8AE08093C60018
:10CD1000FA019491E7E1F5E008C08091C00085FF39
:10CD2000FCCF9093C600319694919923B1F7E4EB30
:10CD3000F9E0949108C08091C00085FFFCCF9093EA
:10CD4000C600319694919923B1F720910F1B309131
:10CD5000101BCE0101962115310519F485519B4117
:10CD600002C0821B930B9A83898369817A818CE04C
:10CD700095E04AE050E00E94843DEDE9F9E09491AD
:10CD800008C08091C00085FFFCCF9093C60031960B
:10CD900094919923B1F78CE095E060ED74E04AE05E
:10CDA00050E00E94843D8091C00085FFFCCF8AE066
:10CDB0008093C6001092840A1092850A1092860A07
:10CDC0001092870A0E940D370E94BA380E94B49BC5
:10CDD0000E943A6E0E94B98F0E941F440E94ECC0CC
:10CDE00080E197E220E931E0F9013197F1F701970D
:10CDF000D9F70E94174C0F900F90CF91DF910895B3
:10CE00002F923F924F925F926F927F928F929F925A
:10CE1000AF92BF92CF92DF92EF92FF920F931F9348
:10CE2000DF93CF93CDB7DEB7CD55D0400FB6F89492
:10CE3000DEBF0FBECDBF2F969FAF8EAF2F976196EF
:10CE40007FAF6EAF61972A0162962FAF62976396AC
:10CE50000FAF63976496EFAE64976896ACAEBDAEC5
:10CE6000CEAEDFAE6897E22EFF24EE0CFF1CEE0C78
:10CE7000FF1C9A012E0D3F1D2D963FAF2EAF2D9713
:10CE8000D9016D907D908D909C90FC01EE0DFF1D61
:10CE9000C401B30120813181428153810E94F7D4C2
:10CEA00069AF7AAF8BAF9CAF10E0000F111F000F7E
:10CEB000111FF201E00FF11F2B96FFAFEEAF2B9782
:10CEC000A080B180C280D3802F96EEADFFAD2F97AA
:10CED000E00FF11FC601B5012081318142815381EC
:10CEE0000E94F7D46DAB7EAB8FAB98AF64962FAD3D
:10CEF0006497E22FF0E0EE0FFF1FEE0FFF1F2F965B
:10CF0000AEADBFAD2F97AE0FBF1F4D915D916D912F
:10CF10007C9129964CAF5DAF6EAF7FAF299761963C
:10CF20006EAD7FAD6197E60FF71F608171818281E1
:10CF3000938129962CAD3DAD4EAD5FAD29970E94F2
:10CF4000F6D469AB7AAB8BAB9CAB6196AEADBFADA3
:10CF500061971C968D919D910D90BC91A02D259669
:10CF60008CAF9DAFAEAFBFAF25972F96AEADBFAD27
:10CF70002F971C962D913D914D915C911F97219675
:10CF80002CAF3DAF4EAF5FAF2197A4019301505836
:10CF90002DA73EA74FA758ABB601A501705849A7CA
:10CFA0005AA76BA77CA761966EAD7FAD6197E60E21
:10CFB000F71ED7016D917D918D919C9129AD3AAD70
:10CFC0004BAD5CAD0E94F6D43B014C016196EEADD9
:10CFD000FFAD61970E0F1F1FD8016D917D918D914F
:10CFE0009C912DA93EA94FA958AD0E94F6D45B0192
:10CFF0006C016DA57EA58FA598A9A60195010E943B
:10D00000B0D87B018C0169A57AA58BA59CA5A4014C
:10D0100093010E94B0D89B01AC01C801B7010E94E6
:10D02000F6D41B012C016DA57EA58FA598A9A4019E
:10D0300093010E94B0D87B018C0169A57AA58BA5CC
:10D040009CA5A60195010E94B0D89B01AC01C80126
:10D05000B7010E94F7D49B01AC01C201B1010E944B
:10D060006AD55B016C0120E030E040E050E00E94B6
:10D07000D0D5882354F4C601B5012BED3FE049EC2F
:10D0800050E40E94F7D45B016C01E7968FADE797FF
:10D09000882351F0C601B5012BED3FE049EC50E487
:10D0A0000E94F6D45B016C01C601B501E6962CAD79
:10D0B0003DAD4EAD5FADE6970E94B0D829A93AA923
:10D0C0004BA95CA95F770E94EBD77B018C012FE60F
:10D0D00032E143E85AE30E94D0D587FDF6C1C8018A
:10D0E000B7010E94ADD60E9444D678A76FA3672BE4
:10D0F00021F4E1E0F0E0F8A7EFA32FA138A5B901F2
:10D1000080E090E00E9470D67B018C01C601B501E1
:10D11000A80197010E94D7D56BA37CA38DA39EA3E2
:10D1200069A97AA98BA99CA9A80197010E94D7D5C2
:10D130006F8F78A389A39AA325966CAD7DAD8EAD34
:10D140009FAD259721962CAD3DAD4EAD5FAD21979E
:10D150000E94F6D4A80197010E94D7D56B8F7C8FCF
:10D160008D8F9E8F6BA17CA18DA19EA120E030E0D0
:10D1700040E05FEB0E94B0D82BA13CA14DA15EA185
:10D180000E94B0D820E030E040E85FE30E94F7D48E
:10D190006F8B788F898F9A8F64963FAD6497E32F5A
:10D1A000F0E0EE0FFF1FEE0FFF1F9E012F5F3F4FBE
:10D1B000E20FF31F29964CAD5DAD6EAD7FAD2997A3
:10D1C00040835183628373832F96AEADBFAD2F979B
:10D1D0001C964D915D916D917C911F974D875E8757
:10D1E0006F87788B41E050E05A8B498B66246296BA
:10D1F0007FAD6297672F70E0660F771F660F771F0E
:10D20000C901860F971F6A969FAF8EAF6A97639684
:10D21000BFAD6397AB2FB0E0AA0FBB1FAA0FBB1F18
:10D2200021E030E02C0F3D1F2A0F3B1F6C963FAFD3
:10D230002EAF6C976E96FFAFEEAF6E971AC138E1C6
:10D2400036150CF446C06DA57EA58FA598A92BA117
:10D250003CA14DA15EA10E94B0D87B018C0169A5C3
:10D260007AA58BA59CA52F89388D498D5A8D0E9452
:10D27000B0D89B01AC01C801B7010E94F7D47B0173
:10D280008C016DA57EA58FA598A92F89388D498D14
:10D290005A8D0E94B0D85B016C0169A57AA58BA557
:10D2A0009CA52BA13CA14DA15EA10E94B0D89B01E1
:10D2B000AC01C601B5010E94F6D46DA77EA78FA769
:10D2C00098AB6394C701D80189A79AA7ABA7BCA75D
:10D2D00065C049895A89BA0180E090E00E9470D601
:10D2E0002BA13CA14DA15EA10E94B0D87B018C0175
:10D2F000C8010E94D4D56B8B7C8B8D8B9E8BB70124
:10D30000C8010E9413D93B014C012D96AEADBFADB3
:10D310002D97ED90FD900D911C9117FB109517F92D
:10D3200010952B96EEADFFAD2B972080318042807B
:10D330005380C801B7012B893C894D895E890E94C1
:10D34000B0D85B016C01C201B101A40193010E943C
:10D35000B0D89B01AC01C601B5010E94F7D46DA7FE
:10D360007EA78FA798ABC801B701A40193010E94C3
:10D37000B0D87B018C01C201B1012B893C894D8958
:10D380005E890E94B0D89B01AC01C801B7010E9420
:10D39000F6D469A77AA78BA79CA7662469AD7AAD56
:10D3A0008BAD9CAD2DA53EA54FA558A90E94F7D4E5
:10D3B0006A96AEADBFAD6A976D937D938D939C9346
:10D3C00013976DA97EA98FA998AD29A53AA54BA55C
:10D3D0005CA50E94F7D46C96EEADFFAD6C976083B0
:10D3E0007183828393836E96AEADBFAD6E976D9160
:10D3F0007D918D919C912F8D38A149A15AA10E94B8
:10D40000F7D46E96EEADFFAD6E9760837183828325
:10D4100093836D857E858F8598892B8D3C8D4D8D71
:10D420005E8D0E94F7D46D877E878F87988BCE01A3
:10D4300001960E94623ECE010196BE016B5F7F4F56
:10D44000AE01475F5F4F9E01235F3F4F6896ECAC94
:10D45000FDAC0EAD1FAD6897F7E7CF2ED12CCC0EEB
:10D46000DD1E0E94FD7029893A892F5F3F4F3A8B5C
:10D47000298B49895A896FA178A54617570708F45F
:10D48000DECE61964EAD5FAD6197485F5F4F6196AE
:10D490002EAD3FAD6197245F3F4F61968EAD9FAD3E
:10D4A0006197DC0114966196BFAFAEAF6197BD0185
:10D4B0006896ECACFDAC0EAD1FAD6897E7E7CE2EDD
:10D4C000D12CCC0EDD1E0E94FD70C35ADF4F0FB66B
:10D4D000F894DEBF0FBECDBFCF91DF911F910F91AA
:10D4E000FF90EF90DF90CF90BF90AF909F908F9084
:10D4F0007F906F905F904F903F902F9008953F9254
:10D500004F925F926F927F928F929F92AF92BF9253
:10D51000CF92DF92EF92FF920F931F93CF93DF93FF
:10D520008091ED0F882309F4F6C08090A7039090B6
:10D53000A803A090A903B090AA036091531770911B
:10D540005417882777FD8095982F0E9472D620E087
:10D5500030E040E050E40E94F7D4A50194010E941D
:10D56000D0D587FDD8C03090BF140F2EF0E04F2EDD
:10D57000F0E05F2EF0E06F2EF0E07F2EF02DCDE496
:10D58000D0E058C0232D30E02C9FF0012D9FF00DEE
:10D590003C9FF00D1124E251F04F80819181A281D6
:10D5A000B3810097A105B10581F484819581A6819D
:10D5B000B7810097A105B10541F480859185A285C9
:10D5C000B3850097A105B10591F12C9F60012D9FB6
:10D5D000D00C3C9FD00C11248EEE9FE0C80ED91EBB
:10D5E000F60164857585868597850E9472D67B01D4
:10D5F0008C01F60160897189828993890E9470D6B5
:10D600009B01AC01C801B7010E94D7D5F60122A148
:10D6100033A144A155A10E94B0D87B018C01A30184
:10D6200092010E94DED7181614F4270138013394B2
:10D63000FFE03F228091BE14381609F0A3CFC3014A
:10D64000B2012091AB033091AC034091AD035091F6
:10D65000AE030E94B0D89B01AC01C501B4010E9489
:10D66000F7D47B018C01A50194010E94D0D587FDE0
:10D6700002C0470158011091A3030091A403F09048
:10D68000A503E090A603C501B401212F302F4F2D33
:10D690005E2D0E94DED7181634F4812F902FAF2D07
:10D6A000BE2D4C015D014090D4145090D514609073
:10D6B000D6147090D714C301B201A50194010E9441
:10D6C000DED71816C4F4C501B40120E037ED43EAF3
:10D6D0005CE30E94B0D87B018C01C301B20128E455
:10D6E00031EE4AE75FE30E94B0D8A80197010E949B
:10D6F000F7D44B015C018092D4149092D514A0927F
:10D70000D614B092D714C501B4010E943FD67093CD
:10D71000541760935317DF91CF911F910F91FF9092
:10D72000EF90DF90CF90BF90AF909F908F907F90C1
:10D730006F905F904F903F9008958091BE149091AC
:10D74000BF14891B8F7008950F931F93CF93DF939E
:10D75000C0E0D0E08E010353104FFE01EF55F04FB3
:10D7600060817181828193810E9470D6FE01EF56A3
:10D77000F04F20813181428153810E94B0D80E94B4
:10D7800044D6F80160837183828393832496C031E9
:10D79000D10501F7DF91CF911F910F910895FC0101
:10D7A000608171818281938120919D0F30919E0FC4
:10D7B00040919F0F5091A00F0E94B0D80E9480D836
:10D7C0006093E90F7093EA0F8093EB0F9093EC0F47
:10D7D00089EE9FE00E94459008958F929F92AF92AC
:10D7E000BF92CF92DF92EF92FF920F931F93FC01B3
:10D7F0008B015A014901608171818281938120915D
:10D80000910F3091920F4091930F5091940F0E947D
:10D81000B0D80E9480D83DEDC32E3FE0D32E609358
:10D82000DD0F7093DE0F8093DF0F9093E00FF80110
:10D8300060817181828193812091950F3091960F43
:10D840004091970F5091980F0E94B0D80E9480D8B5
:10D8500024E0E22EF12CEC0CFD1C6093E10FF701AB
:10D86000718382839383F5016081718182819381C9
:10D870002091990F30919A0F40919B0F50919C0FDE
:10D880000E94B0D80E9480D88601085F1F4F609325
:10D89000E50FF801718382839383F40160817181C4
:10D8A0008281938120919D0F30919E0F40919F0F17
:10D8B0005091A00F0E94B0D80E9480D8F6013C96EB
:10D8C0006093E90F718382839383C601B701A80136
:10D8D0009F010E940B9080E090E0A0E0B0E0809378
:10D8E000C0149093C114A093C214B093C314809336
:10D8F000C4149093C514A093C614B093C714809316
:10D90000C8149093C914A093CA14B093CB148093F5
:10D91000CC149093CD14A093CE14B093CF148093D5
:10D92000D0149093D114A093D214B093D3141F9118
:10D930000F91FF90EF90DF90CF90BF90AF909F90AE
:10D940008F9008958F929F92AF92BF92CF92DF9265
:10D95000EF92FF920F931F93CF93DF93EC016B0134
:10D96000009709F45CC08FA9882309F058C0EEA085
:10D97000FFA008A519A5FB01B6A0A7A090A481A4AB
:10D98000C801B7012B2D3A2D492D582D0E94D0D515
:10D9900088230CF044C0C801B701A80197010E9478
:10D9A000B0D87B018C016AA97BA98CA99DA990584C
:10D9B00020E030E040E050EC0E94B0D82EA53FA51A
:10D9C00048A959A90E94B0D89B01AC01C801B70170
:10D9D0000E94F7D40E941DD97B018C016B2D7A2DFA
:10D9E000892D982D9701A8010E94D0D5882324F471
:10D9F000EB2CFA2C092D182D6B2D7A2D892D982DB5
:10DA00009701A8010E94D0D5882349F0C701D80109
:10DA1000F60186A397A3A0A7B1A781E086ABDF910B
:10DA2000CF911F910F91FF90EF90DF90CF90BF901B
:10DA3000AF909F908F900895EF92FF920F931F9356
:10DA4000CF93DF93F090BF1400E010E020E030E0CF
:10DA50004DE4E42E12C0FE9CE0011124C251D04FCF
:10DA6000C901B801AE010E94A26C8F2D8F5F803179
:10DA700009F480E0F82E98018E018091BE14F8160A
:10DA800051F7C901B80140E050E00E94A26CDF915B
:10DA9000CF911F910F91FF90EF900895AF92BF9299
:10DAA000CF92DF92EF92FF920F931F93CF93DF936A
:10DAB000EB018A016115710509F466C04115510534
:10DAC00009F462C0DAA4CBA4BCA4ADA46EA17FA16A
:10DAD00088A599A52D2D3C2D4B2D5A2D0E94D0D5D2
:10DAE000882309F451C08FA9882309F043C0F801A5
:10DAF000E6A0F7A000A511A56D2D7C2D8B2D9A2DEC
:10DB0000A80197010E94DED71816A4F5C801B70135
:10DB1000A80197010E94B0D87B018C016AA97BA95A
:10DB20008CA99DA9905820E030E040E050EC0E9484
:10DB3000B0D82EA53FA548A959A90E94B0D89B01ED
:10DB4000AC01C801B7010E94F7D40E941DD97B0126
:10DB50008C016D2D7C2D8B2D9A2D9701A8010E9493
:10DB6000D0D5882324F4ED2CFC2C0B2D1A2DC701C5
:10DB7000D80104C08D2D9C2DAB2DBA2D8EA39FA353
:10DB8000A8A7B9A781E08EABDF91CF911F910F912C
:10DB9000FF90EF90DF90CF90BF90AF900895CF921D
:10DBA000DF92EF92FF920F93DF93CF9300D0CDB728
:10DBB000DEB78091BE148FB7F894F090BF148FBF7A
:10DBC0008091BE1490E040968F1991098F709070EB
:10DBD000049704F10091BE1403500F70CC24DD248F
:10DBE00040E050E06DE4E62E13C0802F002309F4DE
:10DBF00080E1082F01500E9DC00111248251904FE9
:10DC00009A838983B6010E944E6DA601C980DA808D
:10DC10000F1559F70F900F90CF91DF910F91FF9053
:10DC2000EF90DF90CF9008956091EC079091BF1432
:10DC30008091BE149817B9F04091BF14242F30E0A2
:10DC40008DE490E0289FF001299FF00D389FF00DA2
:10DC50001124EA5CFF4E608102C04F5F4F708091DB
:10DC6000BE144817D1F784E070E00E94B3CF0E9441
:10DC70007F6A08951092BE141092BF1480E1EDEDFA
:10DC8000FFE0DF011D928A95E9F780E090E0A0E0D7
:10DC9000B0E08093C4149093C514A093C614B093BD
:10DCA000C7148093C8149093C914A093CA14B09356
:10DCB000CB148093CC149093CD14A093CE14B09336
:10DCC000CF148093D0149093D114A093D214B09316
:10DCD000D3148093C0149093C114A093C214B09332
:10DCE000C31408952F923F924F925F926F927F924A
:10DCF0008F929F92AF92BF92CF92DF92EF92FF925C
:10DD00000F931F93DF93CF93CDB7DEB766970FB610
:10DD1000F894DEBF0FBECDBF9E8B8D8B6A017B0159
:10DD200048015901DC01D8966D917D918D919C91AE
:10DD3000DB970E9470D6698B7A8B8B8B9C8BA701AB
:10DD400096010E94B0D80E94BDD50E9444D66D8332
:10DD50007E838F83988769897A898B899C89A501BD
:10DD600094010E94B0D80E94BDD50E9444D6698318
:10DD70007A838B839C832D813E814F815885283700
:10DD800031054105510540F448E750E060E070E09E
:10DD90004D835E836F83788769817A818B819C81D3
:10DDA000683771058105910540F488E790E0A0E0AF
:10DDB000B0E089839A83AB83BC83AD89BE89AC5BB9
:10DDC000BF4FAD90BD90CD90DC901397A454B04060
:10DDD000BE8BAD8B6D817E818F8198850E9470D6C0
:10DDE0006D877E878F87988BC601B5010E9472D69A
:10DDF0001B012C0120E030E040E050E00E94D0D533
:10DE0000882321F4E0E070E060E028C069897A8925
:10DE10008B899C899B01AC010E94B0D87B018C014D
:10DE20006D857E858F8598899B01AC010E94B0D855
:10DE30009B01AC01C801B7010E94F6D47B018C01A3
:10DE4000C201B101A20191010E94F7D49B01AC0172
:10DE5000C801B7010E94D7D5E62F692F2E2F372F83
:10DE6000482F562FB901CA010E94BDD50E943FD646
:10DE70003B014C0169817A818B819C810E9470D623
:10DE800069877A878B879C8766277727CB016A19F2
:10DE90007B098C099D090E9472D65B016C0120E010
:10DEA00030E040E050E00E94D0D5882321F4E0E04B
:10DEB00070E060E028C069857A858B859C859B0130
:10DEC000AC010E94B0D87B018C0169897A898B8969
:10DED0009C899B01AC010E94B0D89B01AC01C80198
:10DEE000B7010E94F6D47B018C01C601B501A601E1
:10DEF00095010E94F7D49B01AC01C801B7010E94B3
:10DF0000D7D5E62F692F2E2F372F482F562FB9013F
:10DF1000CA010E94ADD6ED89FE89A088B188C28869
:10DF2000D38886017501E618F708080919090E94C7
:10DF30003FD6A8019701261B370B480B590B57FFFB
:10DF400071C0C201B10120E030E040E050E00E9429
:10DF5000D0D5882321F4E0E070E060E044C0C20145
:10DF6000B101A20191010E94F7D47B018C01C6018D
:10DF7000B5010E9470D69B01AC01C801B7010E9497
:10DF8000B0D87B018C016D857E858F8598899B013A
:10DF9000AC010E94B0D89B01AC01C801B7010E943E
:10DFA000F6D47B018C0169857A858B859C859B01E4
:10DFB000AC010E94B0D89B01AC01C801B7010E941E
:10DFC000F7D47B018C01C201B10120E030E040E8D0
:10DFD00050E40E94B0D89B01AC01C801B7010E9477
:10DFE000D7D5E62F692F2E2F372F482F562FB9015F
:10DFF000CA010E94BDD50E943FD6AC01CB01DA0117
:10E000003C014D0197FE03C06624772443016A1446
:10E010007B048C049D0410F03501460120E030E0C3
:10E0200040E050E09FB7F8946D897E89645B7F4F34
:10E03000DB018C91AC54B040BE8BAD8B882321F5B5
:10E04000FD01648A758A868A978A260D371D481DC8
:10E05000591D58962D933D934D935C935B972D815D
:10E060003E814F815885DC962D933D934D935C9373
:10E07000DF97A05CBF4F29813A814B815C812D9352
:10E080003D934D935C9313979FBF66960FB6F8949C
:10E09000DEBF0FBECDBFCF91DF911F910F91FF90DB
:10E0A000EF90DF90CF90BF90AF909F908F907F9038
:10E0B0006F905F904F903F902F9008954F925F9296
:10E0C0007F928F929F92AF92BF92CF92DF92EF9208
:10E0D000FF920F931F93CF93DF937090BF14C0E014
:10E0E000D0E07DE4472E512C46C02097B1F18EA997
:10E0F000882361F4849CF001859CF00D949CF00DC4
:10E100001124E251F04F86A9882339F1EAA0FBA03F
:10E110000CA11DA16EA17FA188A599A5A8019701B9
:10E120000E94D7D55B016C01849CF001859CF00DA9
:10E13000949CF00D1124E251F04F66A177A180A5C7
:10E1400091A5A80197010E94D7D58B019C01CE0112
:10E15000B601A5010E94726E1EAA739480E1781622
:10E1600009F47724849CE001859CD00D949CD00D0B
:10E170001124C251D04F872C992487FC9094809110
:10E18000BE1490E08816990609F0AFCF2097F1F001
:10E19000EAA0FBA00CA11DA16EA17FA188A599A555
:10E1A000A80197010E94D7D55B016C016DEC7CEC56
:10E1B0008CE49DE3A80197010E94D7D58B019C01B7
:10E1C000CE01B601A5010E94726E1EAADF91CF9109
:10E1D0001F910F91FF90EF90DF90CF90BF90AF9085
:10E1E0009F908F907F905F904F9008950E94CF6D89
:10E1F0000E941C6D0E945E7008952F923F924F9274
:10E200005F926F927F928F929F92AF92BF92CF92C6
:10E21000DF92EF92FF920F931F93DF93CF93CDB7CF
:10E22000DEB7CC59D0400FB6F894DEBF0FBECDBFDD
:10E230005C014B013A012901C756DF4FE882C959F9
:10E24000D040C656DF4FF882CA59D040C556DF4F7E
:10E250000883CB59D040C456DF4F1883CC59D040E7
:10E26000E796DFAECEAEE7978091BE148F5F803128
:10E2700009F480E0282F332727FD309538A72FA3F6
:10E2800006C00E94759C0E940E400E9405C08091AD
:10E29000BF1490E04FA158A58417950791F36091A2
:10E2A000910F7091920F8091930F9091940FE5963A
:10E2B0006CAF7DAF8EAF9FAFE597D5012D913D91AE
:10E2C0004D915C910E94B0D80E9480D8CD57DF4F0D
:10E2D0006883C358D040CC57DF4F7883C458D040B0
:10E2E000CB57DF4F8883C558D040CA57DF4F98833C
:10E2F000C658D0402091950F3091960F4091970FBE
:10E300005091980FE1962CAF3DAF4EAF5FAFE197C4
:10E31000CA01B901D4012D913D914D915C910E94AA
:10E32000B0D80E9480D8C957DF4F6883C758D04003
:10E33000C857DF4F7883C858D040C757DF4F88830E
:10E34000C958D040C657DF4F9883CA58D040209153
:10E35000990F30919A0F40919B0F50919C0FAD9661
:10E360002CAF3DAF4EAF5FAFAD97CA01B901D3013E
:10E370002D913D914D915C910E94B0D80E9480D822
:10E38000C557DF4F6883CB58D040C457DF4F7883E1
:10E39000CC58D040C357DF4F8883CD58D040C257A8
:10E3A000DF4F9883CE58D04020919D0F30919E0F23
:10E3B00040919F0F5091A00FA9962CAF3DAF4EAF4B
:10E3C0005FAFA997CA01B901D2012D913D914D913D
:10E3D0005C910E94B0D80E9480D8C157DF4F6883FB
:10E3E000CF58D040C057DF4F7883C059D040CF5668
:10E3F000DF4F8883C159D040CE56DF4F9883C25932
:10E40000D0408091BE14E82FF0E0A596FFAFEEAFAC
:10E41000A5978DE490E09F01289FF001299FF00DC2
:10E42000389FF00D1124E251F04FE45BFF4F108252
:10E43000EC54F0404091DD0F5091DE0F6091DF0F02
:10E440007091E00FA3964CAF5DAF6EAF7FAFA39717
:10E45000CD57DF4F88819981AA81BB81C358D040B5
:10E46000841B950BA60BB70B6F968CAF9DAFAEAF11
:10E47000BFAF6F9780839183A283B383B7FF0BC035
:10E48000B095A095909581959F4FAF4FBF4F8083DA
:10E490009183A283B3832091E10F3091E20F4091E9
:10E4A000E30F5091E40F6B962CAF3DAF4EAF5FAFD3
:10E4B0006B97C957DF4F688179818A819B81C758E3
:10E4C000D040621B730B840B950B67966CAF7DAFCE
:10E4D0008EAF9FAF67978DE490E0A596AEADBFADD0
:10E4E000A597A89FF001A99FF00DB89FF00D1124EA
:10E4F000E251F04F67962CAD3DAD4EAD5FAD6797E5
:10E50000248335834683578357FF0DC0DA01C90141
:10E51000B095A095909581959F4FAF4FBF4F848345
:10E520009583A683B7834091E50F5091E60F6091E4
:10E53000E70F7091E80F63964CAF5DAF6EAF7FAFA2
:10E540006397C557DF4F88819981AA81BB81CB58DA
:10E55000D040841B950BA60BB70B2F968CAF9DAFAD
:10E56000AEAFBFAF2F978DE490E0A596AEADBFAD37
:10E57000A597A89FF001A99FF00DB89FF00D112459
:10E58000E251F04F2F962CAD3DAD4EAD5FAD2F97C4
:10E59000208731874287538757FF0DC0DA01C901B1
:10E5A000B095A095909581959F4FAF4FBF4F8087B5
:10E5B0009187A287B3872090E90F3090EA0F4090AF
:10E5C000EB0F5090EC0FC157DF4F488159816A81A2
:10E5D0007B81CF58D04042195309640975092B96A5
:10E5E0004CAF5DAF6EAF7FAF2B97E091EB07F0E0E4
:10E5F000EE0FFF1FEE0FFF1FEA58FC4F6081718185
:10E600008281938127966CAF7DAF8EAF9FAF2797A6
:10E61000809174039091750323969FAF8EAF2397DB
:10E620002B966CAD7DAD8EAD9FAD2B9797FF07C040
:10E6300090958095709561957F4F8F4F9F4F0E9469
:10E6400072D627962CAD3DAD4EAD5FAD27970E949B
:10E65000B0D80E943FD62396AEADBFAD23979D01A3
:10E66000442737FD4095542F0E9482D924E630E09C
:10E6700040E050E00E94EAD98DE490E0A5966EADAE
:10E680007FADA597689FF001699FF00D789FF00D11
:10E690001124E251F04FDF011C96248711963C9320
:10E6A000119712964C93129713965C93E080F18029
:10E6B000028113816480758086809780A084B184F4
:10E6C000C284D384C901DA018A159B05AC05BD0556
:10E6D00014F4D601C50186159705A805B90514F4EB
:10E6E000D401C3019C01AD018E159F05A007B107A0
:10E6F00014F4A80197018DE490E0A596AEADBFADEE
:10E70000A597A89FB001A99F700DB89F700D112407
:10E710006251704FFB01208B318B428B538B263023
:10E7200031054105510510F40C94977CE85BFF4FCF
:10E730008091EC079091ED07AA2797FDA095BA2F3D
:10E7400080839183A283B383DB0190961C92CD5783
:10E75000DF4F288139814A815B81C358D040A3961D
:10E760008CAD9DADAEADBFADA397281739074A0755
:10E770005B0724F481E0DB0190968C93C957DF4F4F
:10E78000288139814A815B81C758D0406B966CAD36
:10E790007DAD8EAD9FAD6B9726173707480759079C
:10E7A00094F48DE490E0A596AEADBFADA597A89F7B
:10E7B000F001A99FF00DB89FF00D1124E251F04F28
:10E7C00080A1826080A3C557DF4F288139814A81AB
:10E7D0005B81CB58D04063966CAD7DAD8EAD9FAD67
:10E7E0006397261737074807590794F48DE490E09C
:10E7F000A596AEADBFADA597A89FF001A99FF00D5E
:10E80000B89FF00D1124E251F04F80A1846080A3E5
:10E81000C157DF4F288139814A815B81CF58D04071
:10E82000221533054405550594F48DE490E0A59632
:10E830004EAD5FADA597489FF001499FF00D589FE1
:10E84000F00D1124E251F04F80A1886080A38DE487
:10E8500090E0A5966EAD7FADA597689FF001699F8A
:10E86000F00D789FF00D1124E251F04FE796AEAD18
:10E87000BFADE7978C9181A3208131814281538183
:10E8800021962CAF3DAF4EAF5FAF219721153105DB
:10E890004105510509F05E988DE490E0A5964EADD6
:10E8A0005FADA597489FF001499FF00D589FF00D6F
:10E8B0001124E251F04F6480758086809780611446
:10E8C00071048104910409F05E988DE490E0A596AE
:10E8D0006EAD7FADA597689FF001699FF00D789FA1
:10E8E000F00D1124E251F04FA084B184C284D3848E
:10E8F000A114B104C104D10409F015988DE490E08D
:10E90000A596AEADBFADA597A89FF001A99FF00D4C
:10E91000B89FF00D1124E251F04F84859585A685AE
:10E92000B7850097A105B10551F05E982090B10F11
:10E930003090B20F4090B30F5090B40F08C02090A9
:10E94000C90F3090CA0F4090CB0F5090CC0FC756D4
:10E95000DF4F6881C959D040C656DF4F7881CA5908
:10E96000D040C556DF4F8881CB59D040C456DF4FC9
:10E970009881CC59D040A20191010E94D0D587FD49
:10E9800016C0C756DF4F8881C959D040C656DF4FE1
:10E990009881CA59D040C556DF4FA881CB59D04085
:10E9A000C456DF4FB881CC59D0401C012D016F9661
:10E9B0006CAD7DAD8EAD9FAD6F970E9472D6E59622
:10E9C0002CAD3DAD4EAD5FADE5970E94D7D5C1589A
:10E9D000DF4F6883CF57D040C058DF4F7883C0588F
:10E9E000D040CF57DF4F8883C158D040CE57DF4F3C
:10E9F0009883C258D040AC01CB01DA0189839A8355
:10EA0000AB83BC8367966CAD7DAD8EAD9FAD6797D4
:10EA10000E9472D6E1962CAD3DAD4EAD5FADE19753
:10EA20000E94D7D5EC966FAFEC97ED967FAFED9740
:10EA3000EE968FAFEE97EF969FAFEF97AC01CB01BD
:10EA4000DA018D839E83AF83B8872F966CAD7DAD41
:10EA50008EAD9FAD2F970E9472D6AD962CAD3DAD79
:10EA60004EAD5FADAD970E94D7D5E8966FAFE897F2
:10EA7000E9967FAFE997EA968FAFEA97EB969FAF5B
:10EA8000EB97AC01CB01DA0189879A87AB87BC870A
:10EA90002B966CAD7DAD8EAD9FAD2B970E9472D63F
:10EAA000A9962CAD3DAD4EAD5FADA9970E94D7D5CF
:10EAB00027962CAD3DAD4EAD5FAD27970E94B0D8E7
:10EAC0007B018C012396EEADFFAD2397BF01882714
:10EAD00077FD8095982F0E9472D69B01AC01C801EA
:10EAE000B7010E94B0D820E030E048EC52E40E9428
:10EAF000D7D59B01AC016D877E878F87988B219638
:10EB00006CAD7DAD8EAD9FAD2197663071058105F1
:10EB100091051CF576E06716710481049104ECF40C
:10EB200086E0A816B104C104D104BCF48DE490E0E1
:10EB3000A596AEADBFADA597A89FF001A99FF00D1A
:10EB4000B89FF00D1124E251F04FDA01C901BF77EF
:10EB500086A797A7A0ABB1AB5DC0C158DF4F288196
:10EB6000CF57D040C058DF4F3881C058D040CF5722
:10EB7000DF4F4881C158D040CE57DF4F5881C2582F
:10EB8000D040B901CA010E9467D93B014C01EC9603
:10EB90002FADEC97ED963FADED97EE964FADEE971E
:10EBA000EF965FADEF97B901CA010E9467D95B018B
:10EBB0006C01E8962FADE897E9963FADE997EA96A4
:10EBC0004FADEA97EB965FADEB97B901CA010E9492
:10EBD00067D97B018C01C401B301A60195010E9494
:10EBE000F7D4A80197010E94F7D40E941DD92DE403
:10EBF00030E0A5964EAD5FADA597429FF001439FD3
:10EC0000F00D529FF00D1124E251F04F66A777A747
:10EC100080AB91AB8DE490E0A5966EAD7FADA597EE
:10EC2000689FF001699FF00D789FF00D1124E2516B
:10EC3000F04F86A597A5A0A9B1A989AF9AAFABAFB0
:10EC4000BCAF60E070E080E89FE329AD3AAD4BAD2A
:10EC50005CAD0E94D7D59B01AC01C201B1010E94FD
:10EC6000B0D82B013C018091BE149091BF14A82F05
:10EC7000B0E05096A91BB109AF70B070BEA3ADA3B0
:10EC8000A230B1050CF451C05D01CC24B7FCC09496
:10EC9000DC2CC601B5010E9472D620E030E040E0D5
:10ECA00051E40E94D0D588230CF03FC060E074E2AC
:10ECB00084E799E4A30192010E94D7D50E9480D8ED
:10ECC0007B018C0160917D0F70917E0F80917F0F91
:10ECD0009091800FE616F7060807190730F56E19B0
:10ECE0007F09800B910B660F771F881F991FA60164
:10ECF00095010E94C8D9CA01B9010E9470D60E942C
:10ED000080D89B01AC012E0D3F1D401F511FCA0131
:10ED1000B9010E9470D69B01AC0160E074E284E707
:10ED200099E40E94D7D52B013C018DE490E0A59693
:10ED3000EEADFFADA597E89F8001E99F100DF89F0C
:10ED4000100D11240251104F69AD7AAD8BAD9CAD01
:10ED5000A30192010E94B0D8D80192966D937D9341
:10ED60008D939C93959750966D917D918D919C91EB
:10ED700053970E9470D6A30192010E94B0D80E94BE
:10ED8000BDD50E9444D6F80160AF71AF82AF93AF9A
:10ED9000CD56DF4F1882C359D040CC56DF4F188272
:10EDA000C459D04020E8222E9FE3392E882499248C
:10EDB000E1E0F0E0EC0FFD1FE80DF91DC301B20129
:10EDC00020813181428153810E94B0D8E1E1F0E09D
:10EDD000EC0FFD1FE80DF91D60837183828393831F
:10EDE0005B016C01E894D7F8F401EF57F04FE08035
:10EDF000F18002811381C601B501A80197010E942B
:10EE0000DED71816CCF4C801B701A60195010E94FF
:10EE1000D7D56B017C01CD56DF4F6881C359D040F7
:10EE2000CC56DF4F7881C459D040C101A70196016B
:10EE30000E94D0D588236CF4CD56DF4F8881C3590A
:10EE4000D040CC56DF4F9881C459D040D1016C01DD
:10EE50007D0124E030E0820E931E30E183169104A0
:10EE600071F0D701C601CD56DF4FC882C359D040DB
:10EE7000CC56DF4F9883C459D0401D0199CFC701AC
:10EE8000B60120E030E040E85FE30E94D0D588235F
:10EE90000CF04CC08E010F5E1F4F81E2A82EB12CEA
:10EEA000AC0EBD1ED8016D917D918D919C91A701F5
:10EEB00096010E94B0D8F801619371938193919368
:10EEC0008F01EA15FB0571F78DE490E0A5962EAD54
:10EED0003FADA597289F8001299F100D389F100DE9
:10EEE00011240251104FD80192966D917D918D9110
:10EEF0009C919597A70196010E94B0D8F80162A352
:10EF000073A384A395A360AD71AD82AD93AD0E9450
:10EF100070D6A70196010E94B0D80E9444D6D801AD
:10EF2000D8966D937D938D939C93DB978DE490E0C1
:10EF3000A596EEADFFADA597E89F8001E99F100D66
:10EF4000F89F100D11240251104FD80150966D9169
:10EF50007D918D919C9153970E9470D6F80126A5C2
:10EF600037A540A951A90E94D7D51B012C01F80152
:10EF700080819181A281B3810097A105B10549F5F6
:10EF800084819581A681B7810097A105B10509F516
:10EF900080859185A285B3850097A105B105C9F447
:10EFA000C201B1012091B90F3091BA0F4091BB0F4E
:10EFB0005091BC0F0E94B0D80E94BDD50C5B1F4F72
:10EFC0000E9444D6D8016D937D938D939C931397A3
:10EFD00071C1C201B1012091B50F3091B60F4091BE
:10EFE000B70F5091B80F0E94B0D80E94BDD50E94B3
:10EFF00044D62DE430E0A596EEADFFADA597E29F97
:10F000006001E39FD00CF29FD00C11242EEE3FE064
:10F01000C20ED31EB4E46B2E712C6C0C7D1CD3017C
:10F020006D937D938D939C9313978090CD0F9090CB
:10F03000CE0FA090CF0FB090D00F0E9470D67B0162
:10F040008C01F60160817181828193810E9472D668
:10F050009B01AC01C801B7010E94B0D87B018C01B3
:10F06000D60150966D917D918D919C9153970E9400
:10F0700070D69B01AC01C801B7010E94D7D57B01B6
:10F080008C01C501B4010E9470D69B01AC01C8017E
:10F09000B7010E94DED718162CF4F301808291820A
:10F0A000A282B3828090D10F9090D20FA090D30F04
:10F0B000B090D40F8DE490E0A5962EAD3FADA5970E
:10F0C000289F6001299FD00C389FD00C11244EEE50
:10F0D0005FE0C40ED51EA4E46A2E712C6C0C7D1C5E
:10F0E000D3016D917D918D919C910E9470D67B0191
:10F0F0008C01F60164817581868197810E9472D6A8
:10F100009B01AC01C801B7010E94B0D87B018C0102
:10F11000D60150966D917D918D919C9153970E944F
:10F1200070D69B01AC01C801B7010E94D7D57B0105
:10F130008C01C501B4010E9470D69B01AC01C801CD
:10F14000B7010E94DED718162CF4F3018082918259
:10F15000A282B3828090D90F9090DA0FA090DB0F3B
:10F16000B090DC0F8DE490E0A5962EAD3FADA59755
:10F17000289F6001299FD00C389FD00C11244EEE9F
:10F180005FE0C40ED51EF4E46F2E712C6C0C7D1C58
:10F19000D3016D917D918D919C910E9470D67B01E0
:10F1A0008C01F60164857585868597850E9472D6E7
:10F1B0009B01AC01C801B7010E94B0D87B018C0152
:10F1C000D60150966D917D918D919C9153970E949F
:10F1D00070D69B01AC01C801B7010E94D7D57B0155
:10F1E0008C01C501B4010E9470D69B01AC01C8011D
:10F1F000B7010E94DED718162CF4F30180829182A9
:10F20000A282B3828090D50F9090D60FA090D70F96
:10F21000B090D80F8DE490E0A5962EAD3FADA597A8
:10F22000289F6001299FD00C389FD00C11244EEEEE
:10F230005FE0C40ED51EE4E46E2E712C6C0C7D1CB8
:10F24000D3016D917D918D919C910E9470D67B012F
:10F250008C01F60160857185828593850E9472D646
:10F260009B01AC01C801B7010E94B0D87B018C01A1
:10F27000D60150966D917D918D919C9153970E94EE
:10F2800070D69B01AC01C801B7010E94D7D57B01A4
:10F290008C01C501B4010E9470D69B01AC01C8016C
:10F2A000B7010E94DED718162CF4F30180829182F8
:10F2B000A282B3828DE490E0A5962EAD3FADA597D6
:10F2C000289F6001299FD00C389FD00C11244EEE4E
:10F2D0005FE0C40ED51EF601EC5BFF4F60817181CB
:10F2E000828193810E9470D67B018C01A2019101E1
:10F2F0000E94D7D5D601D2966D937D938D939C9322
:10F30000D597C801B7012DEB37E346E051E40E94E1
:10F31000B0D80E943FD6F601648F758F868F978F85
:10F320006090BD0F7090BE0F8090BF0F9090C00F87
:10F33000C401B30120E030E040E05FE30E94B0D8B8
:10F340005B016C01298D3A8D4B8D5C8D2DAB3EABF5
:10F350004FAB58AF4091C10F5091C20F6091C30F96
:10F360007091C40F49AB5AAB6BAB7CABCB01BA010C
:10F3700020E030E040E05FE30E94B0D87B018C01E8
:10F380006DA97EA98FA998AD9F77A80197010E94CA
:10F39000DED7181644F4C601B501A80197010E94F2
:10F3A000D0D5882314F4860175016D8D7E8D8F8DE7
:10F3B00098A16DA77EA78FA798AB8091C50F90915C
:10F3C000C60FA091C70FB091C80F89A79AA7ABA786
:10F3D000BCA7BC01CD0120E030E040E05FE30E942B
:10F3E000B0D81B012C016DA57EA58FA598A99F778C
:10F3F000A20191010E94DED7181644F4C801B7019A
:10F40000A20191010E94D0D5882314F4170128018C
:10F410008DE490E0A596AEADBFADA597A89FF00195
:10F42000A99FF00DB89FF00D1124E251F04F22A1D9
:10F4300033A144A155A129A33AA34BA35CA3C201C4
:10F44000B1010E94D0D587FD04C029A03AA04BA0ED
:10F450005CA04DA15EA1423051050CF405C1509154
:10F46000C014CB56DF4F5883C559D0406091C114AA
:10F47000CA56DF4F6883C659D0407091C214C9562E
:10F48000DF4F7883C759D0408091C314C856DF4FEF
:10F490008883C859D040652FCA56DF4F7881C65936
:10F4A000D040C956DF4F8881C759D040C856DF4F7A
:10F4B0009881C859D04027E137EB41ED58E30E94CD
:10F4C000DED718160CF0D0C069897A898B899C899F
:10F4D0002091C4143091C5144091C6145091C714A2
:10F4E0000E94F6D49B01AC010E94B0D87B018C0134
:10F4F0006D897E898F89988D2091C8143091C914A7
:10F500004091CA145091CB140E94F6D49B01AC01D7
:10F510000E94B0D89B01AC01C801B7010E94F7D48A
:10F520000E941DD97B018C01A40193010E94DED7AA
:10F5300018165CF00F2EF0E06F2EF0E07F2EF0E852
:10F540008F2EFFE39F2EF02D08C0C401B301A80148
:10F5500097010E94D7D53B014C016DA97EA98FA9C7
:10F5600098AD2091CC143091CD144091CE1450918F
:10F57000CF140E94F6D47B018C01E89417F9C801DE
:10F58000B70129A93AA94BA95CA90E94DED7181690
:10F5900094F469A97AA98BA99CA9A80197010E9452
:10F5A000D7D55B016C01C401B301A60195010E948E
:10F5B000D0D5882314F4640153016DA57EA58FA5D1
:10F5C00098A92091D0143091D1144091D214509127
:10F5D000D3140E94F6D47B018C01E89417F9C8017A
:10F5E000B70129A53AA54BA55CA50E94DED7181640
:10F5F00094F469A57AA58BA59CA5A80197010E9402
:10F60000D7D57B018C01C601B501A80197010E94E5
:10F61000D0D5882314F48601750169A17AA18BA144
:10F620009CA1A80197010E94B0D87B018C01CB5608
:10F63000DF4F6881C559D040CA56DF4F7881C6591F
:10F64000D040C956DF4F8881C759D040C856DF4FD8
:10F650009881C859D040A80197010E94D0D587FD54
:10F6600019C0D801C70102C0D201C101CB56DF4F7A
:10F670008883C559D040CA56DF4F9883C659D040B9
:10F68000C956DF4FA883C759D040C856DF4FB8834B
:10F69000C859D0408DE490E0A596AEADBFADA5971A
:10F6A000A89F8001A99F100DB89F100D1124025131
:10F6B000104FCB56DF4F8881C559D040CA56DF4F17
:10F6C0009881C659D040C956DF4FA881C759D0404C
:10F6D000C856DF4FB881C859D040F80182A793A718
:10F6E000A4A7B5A762A973A984A995A9905820E0F9
:10F6F00030E040E050EC0E94B0D8D8019E962D91A9
:10F700003D914D915C91D1970E94B0D82BE037ED9F
:10F7100043E25BE30E94F7D40E941DD9F62EE72E48
:10F72000D82EC92ECB56DF4F6881C559D040CA5656
:10F73000DF4F7881C659D040C956DF4F8881C759FD
:10F74000D040C856DF4F9881C859D0402F2D3E2D4C
:10F750004D2D5C2D0E94D0D587FD14C0CB56DF4FB8
:10F76000F882C559D040CA56DF4FE882C659D0400A
:10F77000C956DF4FD882C759D040C856DF4FC8821C
:10F78000C859D0408DE490E0A596EEADFFADA597A9
:10F79000E89F8001E99F100DF89F100D1124025180
:10F7A000104FCB56DF4F8881C559D040CA56DF4F26
:10F7B0009881C659D040C956DF4FA881C759D0405B
:10F7C000C856DF4FB881C859D040F80186A397A327
:10F7D000A0A7B1A762A173A184A195A12F2D3E2D51
:10F7E0004D2D5C2D0E94D0D518162CF081E0D8014B
:10F7F000D7968C9302C0F80117AA8DE490E0A596E5
:10F800002EAD3FADA597289FF001299FF00D389FA1
:10F81000F00D1124E251F04F81E086ABA4ECB4E18D
:10F82000FE01719680E101900D928150E1F78DE427
:10F8300090E0A5964EAD5FADA597489F6001499FAA
:10F84000D00C589FD00C11246EEE7FE0C60ED71E50
:10F85000D6019296ED90FD900D911C919597E092B6
:10F86000C014F092C1140093C2141093C31496965E
:10F870006D917D918D919C919997A80197010E941E
:10F88000D7D54B015C01C201B101A80197010E94CB
:10F89000D7D58B019C01C601B501A4010E94726EEF
:10F8A000BFA1B093BE14C157DF4F288139814A816F
:10F8B0005B81CF58D0402093E90F3093EA0F4093FB
:10F8C000EB0F5093EC0FC557DF4F488159816A8188
:10F8D0007B81CB58D0404093E50F5093E60F609367
:10F8E000E70F7093E80FC957DF4F688179818A81EC
:10F8F0009B81C758D0406093E10F7093E20F8093D3
:10F90000E30F9093E40FCD57DF4F88819981AA814F
:10F91000BB81C358D0408093DD0F9093DE0FA0933E
:10F92000DF0FB093E00F0E94F6700E94B38FC456B1
:10F93000DF4F0FB6F894DEBF0FBECDBFCF91DF9182
:10F940001F910F91FF90EF90DF90CF90BF90AF90FD
:10F950009F908F907F906F905F904F903F902F90EF
:10F960000895FF920F931F93CF93DF938B010E9413
:10F9700004CFEB01FF24FA9409C00E9404CF6C1B52
:10F980007D0B6017710710F080E008C0FEBC0DB45D
:10F9900007FEFDCF8EB58F3F81F781E0DF91CF91DC
:10F9A0001F910F91FF900895FC014281242F30E0B8
:10F9B000C9019595879580658CBD40FF02C080E0A8
:10F9C00004C080E0463009F081E08DBD808160E0B8
:10F9D0000E94AED00895DF92EF92FF920F931F9393
:10F9E000CF93DF93EC01D62E79018A010E94D47C5B
:10F9F000CE016CE271E00E94B17C8D2D80648EBDE1
:10FA00000DB407FEFDCF28E130E0D801C701022E7A
:10FA100004C0B695A795979587950A94D2F78EBDA1
:10FA20000DB407FEFDCF285030408FEF283F380738
:10FA300061F7DD2011F485E906C088E0D81611F4DD
:10FA400087E801C08FEF8EBD0DB407FEFDCF8CE0BF
:10FA5000D81631F48FEF8EBD0DB407FEFDCF8EB5F5
:10FA60009FEF2FEF2EBD0DB407FEFDCF8EB587FFA4
:10FA700004C0992311F09150F5CF8B83DF91CF9182
:10FA80001F910F91FF90EF90DF900895FC0180810E
:10FA900061E00E94AED00895DC016EBDFA0120E065
:10FAA00030E00DB407FEFDCF80818EBD0DB407FEA2
:10FAB000FDCF81818EBD2E5F3F4F329682E0203098
:10FAC000380779F70DB407FEFDCF8FEF8EBD0DB46B
:10FAD00007FEFDCF8FEF8EBD0DB407FEFDCF8FEF7C
:10FAE0008EBD0DB407FEFDCF8EB513968C93139784
:10FAF0008F71853011F481E0089583E111968C9324
:10FB00001197CD010E94467D80E00895CF92DF924B
:10FB1000EF92FF920F931F93CF93DF93EC017A0143
:10FB20008B0169018C81833039F059E0EE0CFF1CA8
:10FB3000001F111F5A95D1F7CE0168E1A801970166
:10FB40000E94EB7C882311F086E023C0CE016EEF8B
:10FB5000A6010E944C7D8823E9F0CE0168E572E0A1
:10FB60000E94B17C882311F487E113C0CE016DE0BF
:10FB700020E030E040E050E00E94EB7C882341F43C
:10FB80008FEF8EBD0DB407FEFDCF8EB5882379F0C3
:10FB900086E18983CE010E94467D80E0DF91CF918E
:10FBA0001F910F91FF90EF90DF90CF900895CE01BD
:10FBB0000E94467D81E0F2CFBF92CF92DF92EF921A
:10FBC000FF920F931F93CF93DF93EC016B017A01A8
:10FBD0000E9404CF8B01BB24BA9409C00E9404CFB9
:10FBE000601B710B6D52714010F081E10BC0BEBC07
:10FBF0000DB407FEFDCF8EB58B838F3F79F38E3F1B
:10FC000039F08FE08983CE010E94467D80E02FC0CD
:10FC1000D7011197EF28D9F08FEF8EBD20E030E0AB
:10FC20009FEF0BC00DB407FEFDCF8EB5F601E20FBE
:10FC3000F31F80839EBD2F5F3F4F2A173B0790F332
:10FC40000DB407FEFDCF8EB5AC0DBD1D8C938FEFAF
:10FC50008EBD0DB407FEFDCF8EB58FEF8EBD0DB4FA
:10FC600007FEFDCF8EB5CE010E94467D81E0DF917B
:10FC7000CF911F910F91FF90EF90DF90CF90BF90A9
:10FC80000895CF92DF92EF92FF920F931F93CF933D
:10FC9000DF93EC017A018B0169018C81833039F0AB
:10FCA000A9E0EE0CFF1C001F111FAA95D1F7CE0191
:10FCB00061E1A80197010E94EB7C882339F084E080
:10FCC0008983CE010E94467D80E006C0CE01B60148
:10FCD00040E052E00E94DC7DDF91CF911F910F91B7
:10FCE000FF90EF90DF90CF900895BF92CF92DF9278
:10FCF000EF92FF920F931F93CF93DF93EC01B62EF9
:10FD00001C82198248830E9404CF6B01888161E0C4
:10FD10000E9431D0CE010E94467D86E060E00E94C4
:10FD200031D085E061E00E9431D087E061E00E943F
:10FD300031D084E061E00E9431D084E061E00E9433
:10FD4000AED085E08A8382E58CBD1DBC80E09FEF4C
:10FD50009EBD0DB407FEFDCF8F5F8A30C9F709C085
:10FD60000E9404CF6C197D09615D774010F081E03D
:10FD70005EC0CE0160E020E030E040E050E00E9454
:10FD8000EB7C182F8B83813059F7CE0168E02AEA8B
:10FD900031E040E050E00E94EB7C82FF02C01C8317
:10FDA00011C080E02FEF2EBD0DB407FEFDCF9EB534
:10FDB0008F5F8430C1F79B839A3A11F082E037C09D
:10FDC00082E08C838C81823021F0EE24FF24870135
:10FDD0000FC0E12CF12C012D00E4102F09C00E946E
:10FDE00004CF6C197D09615D774010F08AE01FC077
:10FDF000CE0167E320E030E040E050E00E94EB7C81
:10FE0000CE0169E2A80197010E94EB7C8B838823D5
:10FE100031F78C81823029F5CE016AE320E030E0B1
:10FE200040E050E00E94EB7C882331F088E0898339
:10FE3000CE010E94467D21C08FEF8EBD0DB407FE1E
:10FE4000FDCF8EB5807C803C11F483E08C8380E014
:10FE50009FEF9EBD0DB407FEFDCF2EB58F5F8330A3
:10FE6000C1F7CE010E94467D86E08B1518F488E12B
:10FE7000898303C0BA8281E001C080E0DF91CF9125
:10FE80001F910F91FF90EF90DF90CF90BF9008955A
:10FE9000CF93DF93EB01DC0190E020E03EE28C9118
:10FEA000803269F0283029F4FE01E90FF11D30831A
:10FEB0009F5FFE01E90FF11D8C9180839F5F2F5F93
:10FEC00011962B3061F7C90FD11D1882DF91CF91A8
:10FED00008950F931F93CF93DF93DC01EB018A0109
:10FEE00080E090E020E2FE01E80FF91F20830196F8
:10FEF0008B309105C1F757E040E024C0622F2E32CD
:10FF000019F08EEC9AE007C05A3051F15AE048E0FF
:10FF100018C0321729F1FC01019634913323C9F737
:10FF20005417F0F02132E0F02F37D0F4822F8156B1
:10FF30008A3110F4622F6052FE01E40FF11D6083DC
:10FF40004F5F11962C91222311F02F32B9F6F80150
:10FF5000B183A08390E08881803219F091E001C0E4
:10FF600090E0892FDF91CF911F910F9108956F92AB
:10FF70007F928F929F92AF92BF92CF92DF92EF9239
:10FF8000FF920F931F93CF93DF93EC017A018B01C4
:10FF90002B81222309F480C089899A89AB89BC8985
:10FFA00084179507A607B70708F476C085C0E11443
:10FFB000F1040105110551F41C821D821E821F826D
:10FFC000188619861A861B8681E067C028853985C0
:10FFD0004A855B85E98DFA8D858590E009962150EB
:10FFE00030404040504039014A01082E04C09694E8
:10FFF0008794779467940A94D2F72F5F3F4F4F4FBF
:020000021000EC
:100000005F4F0894E108F1080109110957016801DF
:1000100004C0D694C794B794A7948A95D2F708944D
:10002000E11CF11C011D111DA614B704C804D9045C
:1000300028F0211531054105510549F48D899E8926
:10004000AF89B88D8C839D83AE83BF8316C0A618FD
:10005000B708C808D90811C04C815D816E817F81C5
:10006000898D9A8D94010E94668B0894A108B1082D
:10007000C108D108882331F40FC084E0882E912C68
:100080008C0E9D1EA114B104C104D10429F7E88689
:10009000F9860A871B8798CF80E0DF91CF911F9167
:1000A0000F91FF90EF90DF90CF90BF90AF909F9017
:1000B0008F907F906F900895223009F078CFE7CF2E
:1000C000CF93DF93EC018C859D85AE85BF8540E0A5
:1000D000611141E0BC01CD010E943C89882319F4E3
:1000E00020E030E00AC08889282F30E095E0220F18
:1000F000331F9A95E1F722523B4EC901DF91CF9110
:1001000008950F931F93CF93DF938C01FC0183819C
:100110008823E1F1818187FF36C0C80161E00E9438
:100120006080EC01009791F18881853E79F1F801BA
:100130008381823040F481899289A389B4898C8F2C
:100140009D8FAE8FBF8FF80185899689A789B08D65
:100150009B8F8A8FCD01AA27BB279D8B8C8BE0912B
:10016000D814F091D914309751F0BE016A5E7F4FD8
:10017000CE0148960995888D998D9B8B8A8BF801C5
:1001800081818F7781830E94018904C081E0F80119
:10019000808380E0DF91CF911F910F9108950F939D
:1001A0001F938C010E948180F80113821F910F918F
:1001B0000895FC018381882319F0CF010E94CF802C
:1001C0000895CF93DF93FC01EB018381882391F0A5
:1001D0008250823020F48FE28883198209C0CF01D7
:1001E00060E00E946080009729F0BE010E94487F75
:1001F00081E001C080E0DF91CF9108956F927F92FE
:100200008F929F92AF92BF92CF92DF92EF92FF9226
:100210000F931F93DF93CF9300D000D0CDB7DEB7FD
:100220007C015A016B01DC0113968C91139781308C
:1002300009F091C011968C9181FF8DC0A0C00097EC
:10024000A105B10511F481E087C0F70160847184D4
:1002500082849384C701B601A5010E94B77F8823D9
:1002600009F479C0D70159968D919C915A97A114A0
:10027000B104C104D10489F455964D915D916D91FD
:100280007C9158970E94DC8B882309F464C0F701A5
:10029000158A168A178A108E44C0D70114964D917C
:1002A0005D916D917C9117979E012F5F3F4F0E944A
:1002B000668B882309F44FC0D7015996ED91FC91C4
:1002C0005A9749815A816B817C818789803149F4B1
:1002D000483FBFEF5B07B0E06B07B0E07B0748F03B
:1002E00020C0483F8FEF58078FEF68078FE07807EF
:1002F000C0F4CF010E94DC8B882369F1D7011496EA
:100300004D915D916D917C91179759968D919C912E
:100310005A970FEF1FEF2FEF3FE00E94DF8A8823ED
:10032000D1F0F701A18AB28AC38AD48A8181806818
:100330008183C7010E948180882369F0B601A501ED
:100340006A147B048C049D0410F4B401A301C7015A
:100350000E94B77F01C080E00F900F900F900F9028
:10036000CF91DF911F910F91FF90EF90DF90CF9091
:10037000BF90AF909F908F907F906F900895F701FE
:1003800081899289A389B48984179507A607B7073D
:1003900008F055CFE0CFCF93DF93EC0140E050E081
:1003A00060E070E00E94FE80882369F0CE0161E089
:1003B0000E946080FC01009731F085EE80831B82F3
:1003C0000E94018901C080E0DF91CF9108952F92B2
:1003D0003F924F925F926F927F928F929F92AF92D5
:1003E000BF92CF92DF92EF92FF920F931F93CF9322
:1003F000DF93EC012A018B81882309F4B6C089813F
:1004000080FFB3C0C8C025014E185F083B0174E0EF
:10041000272E312C2C0E3D1E4201A1C02885398586
:100420004A855B856FEFA62E61E0B62EA222B3222D
:100430008B8179018A0199E016950795F794E794E5
:100440009A95D1F7E98DFA8D823049F4428D538D1A
:10045000648D758D4E0D5F1D601F711F3FC0D48070
:10046000DA94DE20A114B104D9F4DD20C9F42115F9
:1004700031054105510549F48D899E89AF89B88DB3
:100480008C839D83AE83BF830BC04C815D816E8165
:100490007F81CF0191010E94668B882309F465C09A
:1004A000E98DFA8D4C815D816E817F814250504093
:1004B00060407040058404C0440F551F661F771FBD
:1004C0000A94D2F786859785A089B189480F591F6C
:1004D0006A1F7B1F4D0D511D611D711D80E092E053
:1004E0008A199B0984018815990508F48C0182E01A
:1004F0000030180709F067C08091DA149091DB147E
:10050000A091DC14B091DD14481759076A077B07E6
:1005100009F459C08091DE169091DF1693010E9474
:10052000417E882349F421C0950122523B4EC301EC
:10053000B901A8010E945123600E711E980140E08C
:1005400050E088859985AA85BB85820F931FA41FDB
:10055000B51F88879987AA87BB87801A910A81145B
:10056000910409F05BCFA20102C04FEF5FEFCA0117
:10057000DF91CF911F910F91FF90EF90DF90CF907F
:10058000BF90AF909F908F907F906F905F904F90B3
:100590003F902F900895A988BA88CB88DC88E8849A
:1005A000F9840A851B859A0140E050E0D601C50117
:1005B0008E199F09A00BB10B281739074A075B0753
:1005C00008F021CF23CFCB01BA0140E00E943C8943
:1005D000882309F0A9CFC9CFCF92DF92EF92FF9283
:1005E0000F931F93CF93DF937C01EB018A01FC01F2
:1005F0008381823008F46FC080859185A285B385A0
:100600008F719070A070B0700097A105B10509F0CE
:1006100062C06DC0F8011082EDE0CE2ED12CC70172
:10062000BE0140E250E00E94E7819C0180329105CA
:1006300021F0009709F04FC050C04881442309F4CD
:100640004CC0453E61F34E3251F38B858F738F3032
:10065000E9F501151105D1F18A8D9B8D892BB1F535
:10066000842F90E08F719070009781F18330910515
:100670006CF58C9D90018D9D300D9C9D300D11244D
:100680002D503040F801E20FF31F898180838B8168
:1006900081838D8182838F818383898584838E8505
:1006A0008583888986838A8987838C8980878E89D8
:1006B0008187888D82878C8D83878E8D84878881C2
:1006C00086FF04C0F801E20FF31F15868B8583FDBA
:1006D000A6CF822F03C08FEF01C080E0DF91CF91C2
:1006E0001F910F91FF90EF90DF90CF9008954115EB
:1006F000510509F08FCF90CFDF93CF930F92CDB7F5
:10070000DEB7BE016F5F7F4F41E050E00E94E7819E
:10071000019719F02FEF3FEF03C08981282F30E0B8
:10072000C9010F90CF91DF910895EF92FF920F933F
:100730001F93CF93DF93EC018B81823038F1E884F3
:10074000F9840A851B85CE010E947C8397FD1EC01B
:1007500088859985AA85BB854F96A11DB11D88877F
:100760009987AA87BB87A5E016950795F794E79424
:10077000AA95D1F72E2D30E02F703070F5E0220FC2
:10078000331FFA95E1F722523B4E02C020E030E0E1
:10079000C901DF91CF911F910F91FF90EF900895C4
:1007A0000F931F93CF93DF93EC018B018B818823F1
:1007B00009F040C0FB018789803109F041C082E027
:1007C0008B831D8A1E8A1F8A188E808D918DA0E0D2
:1007D000B0E045E0880F991FAA1FBB1F4A95D1F7CB
:1007E000898B9A8BAB8BBC8B13C083E08B83F80116
:1007F000428D538D648D758D4D8B5E8B6F8B788F95
:100800009E012F5E3F4FC8010E943A8C882391F0D1
:100810001A8F098F81E089831C821D821E821F82AC
:10082000188619861A861B861C861D861E861F86BC
:10083000188A01C080E0DF91CF911F910F91089538
:100840008032C1F7D2CF1F93CF93DF93EC01142FE7
:10085000262F30E0F90175E0EE0FFF1F7A95E1F7E2
:10086000E252FB4E8385817121F0842F827109F061
:1008700069C08091DA149091DB14A091DC14B091DE
:10088000DD148C879D87AE87BF87688BF90165E093
:10089000EE0FFF1F6A95E1F7E252FB4E84899589BE
:1008A000A0E0B0E0DC01992788278D8B9E8BAF8B71
:1008B000B88F228D338DA90160E070E0482B592B51
:1008C0006A2B7B2B4D8B5E8B6F8B788F838590E0B3
:1008D00088719070009751F4848D958DA68DB78D99
:1008E000898B9A8BAB8BBC8B81E00CC0409751F508
:1008F0009E012F5E3F4F898D9A8D0E943A8C8823EE
:1009000009F184E08B83812F8F7089831C821D8283
:100910001E821F82188619861A861B8614FF18C02D
:10092000CE0140E050E060E070E00E94FE8088234D
:1009300079F40AC049895A896B897C89CE010E9461
:10094000B77F02C01B8280E0DF91CF911F91089595
:1009500015FDF0CF81E0F8CFCF93DF93EC019C0140
:100960002C5F3F4F898D9A8D41E050E060E070E050
:100970000E94A68C8823A1F08D899E89AF89B88DAD
:100980000097A105B10559F48C819D81AE81BF818D
:100990008D8B9E8BAF8BB88F89818068898381E036
:1009A000DF91CF9108952F923F924F925F927F9265
:1009B0008F929F92AF92BF92CF92DF92EF92FF926F
:1009C0000F931F93DF93CF9300D000D000D0CDB70B
:1009D000DEB76C01162F072F5E834D83DC01139663
:1009E0008C911397813009F06FC111968C9181FF22
:1009F0006BC188C1F60141895289638974898085F8
:100A00009185A285B38584179507A607B70731F0AE
:100A1000C6010E94B77F882309F456C1812F902F09
:100A20009C0119014D805E8013C1D6015996ED914C
:100A3000FC915A97DA01C90149E0B695A7959795B7
:100A400087954A95D1F774807A9478228FEF882E13
:100A500081E0982E82229322772009F053C08114DE
:100A6000910409F04FC0D60114964D915D916D919E
:100A70007C911797411551056105710581F45596D3
:100A80008D919D910D90BC91A02D0097A105B10570
:100A900061F1F60184839583A683B78333C0CF01C8
:100AA0009E012F5F3F4F0E94668B882309F40CC183
:100AB00029813A814B815C81D6015996ED91FC9157
:100AC0005A978789803149F4283FBFEF3B07B0E050
:100AD0004B07B0E05B0778F008C0283FEFEF3E0718
:100AE000EFEF4E07EFE05E0730F0C6010E94AC84E6
:100AF000882341F4E9C0D60114962D933D934D937C
:100B00005C93179780E092E0881999095201841547
:100B1000950508F45C01D6015996ED91FC915A9720
:100B20001496ED90FD900D911C9117978EEF9FEF0D
:100B3000AFEFBFEFE80EF91E0A1F1B1F058404C0AC
:100B4000EE0CFF1C001F111F0A94D2F786859785B3
:100B5000A089B189E80EF91E0A1F1B1FE70CF11CC2
:100B6000011D111D90E0A91692E0B90639F580919A
:100B7000DA149091DB14A091DC14B091DD148E1581
:100B80009F05A007B10771F41092E0168FEF9FEF59
:100B9000AFEFBFEF8093DA149093DB14A093DC14D3
:100BA000B093DD148091DE169091DF16B801A70195
:100BB00091010E94867D8823B9F586C08114910435
:100BC00019F5D60118962D913D914D915C911B9789
:100BD00051968D919D910D90BC91A02D28173907AC
:100BE0004A075B0788F00E940189882309F46CC0DA
:100BF00081E08093E016E092DA14F092DB14009327
:100C0000DC141093DD1408C0C801B70141E00E9454
:100C10003C89882309F458C0940122523B4EC901F3
:100C2000B101A5010E945123950140E050E0F60179
:100C300080859185A285B385820F931FA41FB51F60
:100C400080879187A287B3872A0C3B1C4A185B08D0
:100C5000D60118962D913D914D915C911B974114B1
:100C6000510409F0E2CE51968D919D910D90BC9169
:100C7000A02D82179307A407B50748F4F601218B2E
:100C8000328B438B548B81818068818311C080912A
:100C9000D8149091D914892B59F08D819E81892B7C
:100CA00039F0D60111968C911197806811968C932A
:100CB000F601818183FF05C0C6010E9481808823DF
:100CC00019F04D815E8105C081E0D6018C934FEF14
:100CD0005FEFCA0126960FB6F894DEBF0FBECDBFF8
:100CE000CF91DF911F910F91FF90EF90DF90CF9008
:100CF000BF90AF909F908F907F905F904F903F906C
:100D00002F90089582FD76CE89CEDF92EF92FF92EA
:100D10000F931F93CF93DF93EC0189899A89AB8955
:100D2000BC89805E9F4FAF41B04008F071C0CE01DA
:100D30000E94AC84882309F46BC00E940189882337
:100D400009F466C0E98DFA8DEC80FD800E811F816B
:100D50008EEF9FEFAFEFBFEFE80EF91E0A1F1B1FCC
:100D6000058404C0EE0CFF1C001F111F0A94D2F76B
:100D700086859785A089B189E80EF91E0A1F1B1F79
:100D800081E08093E016E092DA14F092DB14009395
:100D9000DC141093DD1480E092E0EEEDF4E1DF016D
:100DA0009C011D9221503040E1F7DD24D39411C005
:100DB000B801A7014D0D511D611D711D8091DE16F9
:100DC0009091DF162EED34E10E94867D882301F19B
:100DD000D394E98DFA8D8481D81650F320E032E067
:100DE00040E050E0058404C0220F331F441F551F0C
:100DF0000A94D2F789899A89AB89BC89820F931F9B
:100E0000A41FB51F898B9A8BAB8BBC8B81E001C073
:100E100080E0DF91CF911F910F91FF90EF90DF90D5
:100E200008958F929F92AF92BF92CF92DF92EF92EE
:100E3000FF920F931F93CF93DF936C01EB01942EDE
:100E4000852EA22E898D9A8DD6015A969C938E93CB
:100E50005997CB0140E050E060E070E00E94B77F1E
:100E6000BB2438C0CE010E949583FC01009709F491
:100E700093C055E016950795F794E7945A95D1F7E6
:100E80001E2D1F708081882311F0853EC9F4BB2080
:100E900099F42091DA143091DB144091DC145091D4
:100EA000DD14D6011C962D933D934D935C931F97B3
:100EB00050961C93BB24B3948081882359F418C0A6
:100EC000892D982DBF014BE050E00E9444230097EC
:100ED00009F470C0E884F9840A851B8589899A8998
:100EE000AB89BC89E816F9060A071B0708F4BACFD4
:100EF000A6FE52C0A1FE50C0BB2051F0F6011089E1
:100F0000C60161E00E946080EC01009769F444C072
:100F10008B81823009F440C0CE010E9485868823EF
:100F2000D9F110E0CEEDD4E180E2DE011D928A9588
:100F3000E9F7DE01292D382DC901FC018BE0019074
:100F40000D928150E1F7E091D814F091D9143097C7
:100F500039F0BE01625F7F4FCE014096099508C00F
:100F600081E298E2998B888B80E098E09F878E875A
:100F7000888999899B8B8A8B998F888F8E859F858D
:100F80009F8B8E8B0E940189882331F0C601612FCF
:100F90004A2D0E94238401C080E0DF91CF911F91F0
:100FA0000F91FF90EF90DF90CF90BF90AF909F9008
:100FB0008F900895A7FEEACFEFCF2F923F924F92E6
:100FC0005F926F927F928F929F92AF92BF92CF92D9
:100FD000DF92EF92FF920F931F93DF93CF93CDB7E2
:100FE000DEB7C654D0400FB6F894DEBF0FBECDBFFB
:100FF0003C016B01DE01AE5BBF4F11965C934E93DB
:1010000025962FAF25971C861F861FA21AA661154D
:10101000710509F480C0FC018381882309F07BC03D
:10102000FA0180818F32F1F08601ECE0EE2EF12C96
:10103000EC0EFD1E72E4A72EB12CAC0EBD1E4E01AF
:101040000894811C911C2796FFAEEEAE279767E2AD
:10105000262E312C2C0E3D1E270124C01196B18363
:10106000A08301C0FD01A081B1818C918F32B1F3C9
:10107000D60113968C91139782508230A8F28E017C
:10108000095D1F4F59966D917C915A97C8010E9436
:10109000D083882351F63FC0342D252D8701832F1F
:1010A000922F7C01F50180819181B401A5010E94FC
:1010B000697F882329F42FC03196D501ED93FC93E5
:1010C000D501ED91FC9180818F32B1F38823C9F075
:1010D000C701B801A40121E00E9411878823D9F03B
:1010E0000C151D0519F0C8010E94CF802796EEADA2
:1010F000FFAD2797EE16FF0679F6C101322D292F95
:10110000CDCFC301B801A40125962FAD25970E942C
:101110001187182F01C010E0CE0187960E94D98058
:10112000CE010C960E94D980812FCA5BDF4F0FB68B
:10113000F894DEBF0FBECDBFCF91DF911F910F910D
:10114000FF90EF90DF90CF90BF90AF909F908F90E7
:101150007F906F905F904F903F902F9008950F93E6
:101160001F93DF93CF93CDB7DEB76B970FB6F8948D
:10117000DEBF0FBECDBF9C01AB0119821C828E0168
:101180000F5F1F4FC801B90122E00E94DD8788234D
:1011900011F410E004C0C8010E94CB81182FCE01C9
:1011A00001960E94D980812F6B960FB6F894DEBF0E
:1011B0000FBECDBFCF91DF911F910F910895DB013D
:1011C0000D900020E9F71197A61BB70B0496AD010F
:1011D0000E94D3840895DF93CF930F92CDB7DEB7EB
:1011E00069830496BE016F5F7F4F41E050E00E942B
:1011F000D3840F90CF91DF91089504960E94D384F9
:1012000008958091E016882399F14091DA14509165
:10121000DB146091DC147091DD148091DE169091E6
:10122000DF162EED34E10E94867D882319F140916E
:10123000E1165091E2166091E3167091E4164115A3
:1012400051056105710591F08091DE169091DF16D0
:101250002EED34E10E94867D882361F01092E11624
:101260001092E2161092E3161092E4161092E01615
:1012700081E0089580E00895DF92EF92FF920F934E
:101280001F937B018C01D42E8091DA149091DB1492
:10129000A091DC14B091DD148E159F05A007B10755
:1012A000C1F00E9401898823E1F08091DE169091BF
:1012B000DF16B801A7012EED34E10E94417E88239C
:1012C00081F0E092DA14F092DB140093DC141093B6
:1012D000DD14DD2011F481E005C081E08093E0168B
:1012E00001C080E01F910F91FF90EF90DF90089573
:1012F0008F929F92AF92BF92CF92DF92EF92FF9226
:101300000F931F93CF93DF936C01142F7093DF160D
:101310006093DE16FC01178A82E090E0A0E0B0E066
:1013200080839183A283B3831092E0161092E1161A
:101330001092E2161092E3161092E4168FEF9FEFD0
:10134000AFEFBFEF8093DA149093DB14A093DC141B
:10135000B093DD14442321F488249924540140C01F
:10136000453008F01EC160E070E080E090E040E0B1
:101370000E943C89882309F414C1C12FD0E0219731
:10138000FE0174E0EE0FFF1F7A95E1F7E252FB4E8B
:10139000E254FE4F8081EE5BF14090E08F779070D9
:1013A000892B09F0FEC0E653FE4F80819181A28116
:1013B000B38184369105A105B10508F4F2C064E05B
:1013C000CC0FDD1F6A95E1F7CC55D94E8880998006
:1013D000AA80BB8081149104A104B10409F4E1C086
:1013E000C501B40140E00E943C89882309F4D9C0BA
:1013F0008091E9149091EA148050924009F0D1C094
:101400002091EE14222309F4CCC08091EC14909129
:10141000ED14892B09F4C5C08091EB14882309F4DD
:10142000C0C0F601228B8091EB148483158661E0A5
:1014300070E007C04F5FF60145874150483008F023
:10144000B0C0F6014585848190E09B01042E02C066
:10145000220F331F0A94E2F78217930759F720915E
:10146000F4143091F5142115310519F040E050E0E5
:1014700008C0209102153091031540910415509138
:101480000515F6012583368347835087E090EC14D9
:10149000F090ED1400E010E0E80CF91C0A1D1B1D93
:1014A000E38AF48A058B168B8091EF149091F014E7
:1014B000918F808F6091EE1470E080E090E00E9448
:1014C00082D96E0D7F1D801F911FF601628F738F71
:1014D000848F958F2091EF143091F01455E0220FF6
:1014E000331F5A95E1F721503E4F232F332726957E
:1014F00040E050E0260F371F481F591F26873787C7
:10150000408B518B8091F1149091F214009719F057
:10151000A0E0B0E008C08091FE149091FF14A0916B
:101520000015B091011585017401E21AF30A040B4C
:10153000150BA8019701280F391F4A1F5B1FF601E1
:10154000058404C056954795379527950A94D2F798
:101550002187328743875487253FFFE03F07F0E02C
:101560004F07F0E05F0720F48CE0F601878B19C08D
:10157000255F3F4F4040504018F480E1F6010EC017
:1015800080910A1590910B15A0910C15B0910D1535
:10159000F601828F938FA48FB58F80E2878B81E0D5
:1015A00001C080E0DF91CF911F910F91FF90EF90EC
:1015B000DF90CF90BF90AF909F908F9008956F92E3
:1015C0007F928F929F92AF92BF92CF92DF92EF92D3
:1015D000FF920F931F93CF93DF93EC015A016B019E
:1015E00038014901423051056105710508F45EC0BA
:1015F00089859A85AB85BC850196A11DB11D84178F
:101600009507A607B70708F451C08F89803129F4E0
:10161000E52EF62E072F11270CC0803209F046C0A8
:101620007A018B0187E016950795F794E7948A95E0
:10163000D1F78B899C89AD89BE89E80EF91E0A1FF6
:101640001B1FC801B70141E00E943C89882371F14A
:101650008F89803149F4F501F070EE0FFF1FE252DF
:10166000FB4E718260820DC0F501EF77F070EE0FD6
:10167000FF1FEE0FFF1FE252FB4E608271828282DB
:1016800093828A89823080F08D819E81AF81B88576
:10169000E80EF91E0A1F1B1FE092E116F092E216F7
:1016A0000093E3161093E41681E001C080E0DF911F
:1016B000CF911F910F91FF90EF90DF90CF90BF904F
:1016C000AF909F908F907F906F900895CF92DF9210
:1016D000EF92FF920F931F93CF93DF93EC017A0168
:1016E0008B01690189859A85AB85BC850196A11D11
:1016F000B11D84179507A607B70708F453C08F8953
:10170000803129F45527412F302F2F2D0CC08032E6
:1017100009F048C09A01AB0167E0569547953795A7
:1017200027956A95D1F78B899C89AD89BE89280F49
:10173000391F4A1F5B1F8091DA149091DB14A0912E
:10174000DC14B091DD14281739074A075B0739F01C
:10175000CA01B90140E00E943C89882319F18F89B0
:10176000803159F4F701F070EE0FFF1FE252FB4E8B
:1017700080819181A0E0B0E00EC0F701EF77F070BA
:10178000EE0FFF1FEE0FFF1FE252FB4E8081918193
:10179000A281B381BF70F60180839183A283B3835A
:1017A00081E001C080E0DF91CF911F910F91FF9008
:1017B000EF90DF90CF900895AF92BF92CF92DF92DB
:1017C000EF92FF920F931F93DF93CF9300D000D03F
:1017D000CDB7DEB76C017A018B0182E090E0A0E02A
:1017E000B0E0F60180839183A283B3835E01089405
:1017F000A11CB11CC601B801A70195010E94668B0E
:10180000882341F1C601B801A70100E010E020E003
:1018100030E00E94DF8A8823E9F0E980FA800B81BA
:101820001C81F6018789803151F4F8EFEF16FFEF44
:10183000FF06F0E00F07F0E01F07E0F209C088EFB5
:10184000E8168FEFF8068FEF08078FE0180790F281
:1018500081E001C080E00F900F900F900F90CF912A
:10186000DF911F910F91FF90EF90DF90CF90BF908D
:10187000AF9008954F925F926F927F928F929F9256
:10188000AF92BF92CF92DF92EF92FF920F931F938E
:10189000DF93CF9300D000D0CDB7DEB76C01498382
:1018A0005A836B837C833901EE24FF2487012E0148
:1018B0000894411C511C812CE2E09E2EA12CB12CDD
:1018C00049815A816B817C81C60192010E94668B9D
:1018D000882339F1D501C401F601058404C0880FBD
:1018E000991FAA1FBB1F0A94D2F7E80EF91E0A1F00
:1018F0001B1F29813A814B815C818789803131F4BA
:10190000285F3F4F40405040D8F205C0285F3F4F0E
:101910004F4F5F40A8F2F301E082F182028313830C
:1019200081E00F900F900F900F90CF91DF911F915A
:101930000F91FF90EF90DF90CF90BF90AF909F906E
:101940008F907F906F905F904F9008952F923F926D
:101950004F925F926F927F928F929F92AF92BF92BF
:10196000CF92DF92EF92FF920F931F93DF93CF936B
:10197000CDB7DEB72F970FB6F894DEBF0FBECDBF41
:101980001C014A875B876C877D873F872E87DC0138
:1019900019968D919D910D90BC91A02D0196A11D40
:1019A000B11D8E839F83A887B987F90100811181BA
:1019B00022813381011511052105310549F04801C6
:1019C00059010894811C911CA11CB11C1D8210C0DE
:1019D000D1018D909D90AD90BC901D828A859B8594
:1019E000AC85BD850197A105B10511F491E09D83FA
:1019F000750164014424552432018E010F5F1F4F8D
:101A0000F10181859285A385B485481659066A0639
:101A10007B0608F090C08E819F81A885B9858C15C2
:101A20009D05AE05BF0550F4A2E08A2E912CA12C95
:101A3000B12CF2E0CF2ED12CE12CF12CC101B70159
:101A4000A60198010E94668B882309F474C08981DD
:101A50009A81AB81BC81A70196012F5F3F4F4F4F09
:101A60005F4F0097A105B10519F049015A010DC05A
:101A7000281939094A095B098A859B85AC85BD858A
:101A8000281739074A075B0759F00894411C511C75
:101A9000611C711C0894C11CD11CE11CF11CB0CF4D
:101AA000C101A601B7010FEF1FEF2FEF3FE00E942A
:101AB000DF8A882399F43FC0260137010894410842
:101AC000510861087108C101B301A20197018601A3
:101AD0000E94DF8A882379F1730162018C149D04CE
:101AE000AE04BF0448F3AE85BF854D915D916D9105
:101AF0007C91411551056105710539F0C1019501D0
:101B000084010E94DF8A8823B1F0EE85FF85808200
:101B10009182A282B382FD81FF2359F00894811C37
:101B2000911CA11CB11CD1018D929D92AD92BC92D1
:101B3000139781E001C080E02F960FB6F894DEBFC6
:101B40000FBECDBFCF91DF911F910F91FF90EF900E
:101B5000DF90CF90BF90AF909F908F907F906F90CD
:101B60005F904F903F902F900895FC018091E51673
:101B70008C3090F480838F5F8093E516815090E0E5
:101B8000FC01EE0FFF1FE80FF91FEA51F94E88EB39
:101B90009BE09283818308958FEF80830895FC01F9
:101BA00020812C30B8F58181992787FD909548E8F0
:101BB00050E0481B590B440F551F440F551F641725
:101BC000750784F08281992787FD909548E552E05A
:101BD000481B590B440F551F440F551F64177507B9
:101BE0000CF4AB0142505040CA01AA2797FDA095C2
:101BF000BA2F880F991FAA1FBB1F4FB7F89430E068
:101C0000F901EE0FFF1FE20FF31FEA51F94E928325
